:100000000C94A90D0C94D10D0C94D10D0C94D10D20
:100010000C94D10D0C94D10D0C94D10D0C94D10DE8
:100020000C94D10D0C94D10D0C94D10D0C94B6619F
:100030000C944C650C94E3610C94D10D0C944B170B
:100040000C9439170C94D10D0C94D10D0C94D10D46
:100050000C94D10D0C94D10D0C94D10D0C94D10DA8
:100060000C940C650C94A7170C944E620C941B63B3
:100070000C94D10D0C94D10D0C94D10D0C94D10D88
:100080000C94D10D0C94D10D0C94D10D0C6710670C
:100090001867226739675367686777678C67A36754
:1000A000AD67CB67D167D667DC67E2673C684668B7
:1000B000EB67F167F76700680468096811682368EF
:1000C00029682F6834681467146819681E685370AB
:1000D0006C617368008040000000000000000000B8
:1000E0000000000000000000000000000000000010
:1000F0000000000000000000000000000000000000
:1001000000000000000000000000000000000000EF
:1001100000000000000000000000000000000000DF
:10012000000080C0E0E0F0F8F8FCFCFCF8F8F8F023
:1001300040000000000080808000000000000000FF
:1001400000000000000000000000000080C0C0E0CF
:10015000E0E0F0F0F0E0C00000000000C0F8FFFFB9
:100160009F8783838383838383838383838383833F
:1001700083838383838383830383808383838383D2
:10018000838383838383838383838383838383833F
:100190008383C3E3733F1F0000000080E0F0F8FC9E
:1001A000FEFFFFFFFF7F3F1F1F0F0783C3E1E1E05B
:1001B000E0C0000E1F3F7F7FFFF3E0E08000000003
:1001C0000000000000000080F0FCFEFFFFFFFF7F4A
:1001D0003F0F0301010100000080F0FEFFFFC7C1D7
:1001E000C1C1C1C1C1C1C1C1C1C1C1C1C1C1C1C1FF
:1001F000C1C1C1C1C101C1F0FEFF3F0F070F0D0D0D
:100200000D1D191919193131313171616161E1C166
:10021000C1C18100000080E0F8FCFFFFFFFF2F1745
:100220000F038180C0E0F0F8FCFEFFFFFFFFFFFF3F
:100230007F010000000000000001010307070E1EFF
:100240001C3870E0F0F8FEFFFF7F1F0F0300010075
:10025000000000000000000000000000000000009E
:10026000000000000000000000000000000000008E
:10027000000000000000000000000000000000007E
:10028000000000000000000000000000000000006E
:1002900000000000007EFFFFFFFFFFFFFBF8FCFCFB
:1002A000FEFF7F3F1F0F07C3FFFFFFFFFFFF7F071B
:1002B0000000000000000000000000000000C0E09E
:1002C000F8FEFFFF7F1F0F1F3D7CF8F8F0E0800075
:1002D000000000000000000000000000000000001E
:1002E000000000000000000000000000000000000E
:1002F00000000000000000000000000000000000FE
:1003000000000000000000000000000000000000ED
:1003100000000000000000010101010103070707C0
:100320000301000000E0FCFFFFFFFFFF1F030000D0
:10033000000000000000000000C0F078DE27130974
:100340000E0703000000000000000001030F7FFF04
:10035000FC7878F800000000000000000000008039
:10036000808080808080808000808000808000008D
:1003700000000000008080808080808080808080FD
:1003800080808080808080000000000000000000ED
:10039000000000000000000000000000000000005D
:1003A000000080F0FEFFFFFFFF3F0F010000000094
:1003B00000000000C0E0381E0F0300010000000034
:1003C000000000000000000000000000000000002D
:1003D0000000030301000000000000000000000E08
:1003E0000E02020202020303000F0F000F0F0808A3
:1003F00008080808080F0F08080808080F0F000071
:1004000000000F0F000000000000000000000000CE
:1004100000000000000000000000000000000000DC
:10042000C0F8BFFFFFFF1F7F0100000000000000B9
:1004300000F0FCFF7F7830000000000000000000AA
:1004400000000000000000000000000000000000AC
:10045000000000000000000000000000000000009C
:10046000000000000000000000000000000000008C
:10047000000000000000000000000000000000007C
:10048000000000000000000000000000000000006C
:100490000000000000000000000000000000301C10
:1004A000070E0F0701000000000000000000000020
:1004B000000000000000000000000000000000003C
:1004C000000000000000000000000000000000002C
:1004D00000000000000000001B1E272D36394B4E87
:1004E000636C7278878D939CB1B4C6C9D2D8E1E4AD
:1004F00001020304010302040402030104030201D4
:1005000003010200040506076D656E75537461638F
:100510006B206F766572666C6F77006D656E7553D4
:100520007461636B20756E646572666C6F770070C2
:100530007265737320616E79204B657900414C457B
:100540005254004D455353414745004C4F41444997
:100550004E47002020202020202020202020202066
:1005600020202020202020202000506C6561736511
:1005700020526573657420537769746368657300EE
:100580005377697463686573205761726E696E672B
:1005900000204F6C642056657273696F6E2045456C
:1005A00050524F4D202020434845434B2053455443
:1005B00054494E47532F43414C494200416C6172AC
:1005C0006D732044697361626C6564005265736584
:1005D00074207468726F74746C65005468726F7400
:1005E000746C65206E6F742069646C650050726570
:1005F000737320616E79206B657920746F20736B43
:10060000697000414C45525400454550524F4D20B1
:100610006C6F77206D656D004F46464142535255D1
:1006200073525525454C73454C2554487354482501
:10063000414C73414C2550312050312550322050CF
:1006400032255033205033250054485252554445EA
:100650004C4549443049443149443241494C47456D
:100660004154524E535731535732535733535734E3
:1006700053573553573653573753573853573953C2
:100680005741535742535743004F4646004F4E2061
:10069000002D2D2D004348002D2D2D2000525544B6
:1006A00020454C45205448522041494C20005031AF
:1006B000202050322020503320204D4158204655D4
:1006C0004C4C4359433143594332435943335050BF
:1006D0004D3150504D3250504D3350504D3450509C
:1006E0004D3550504D3650504D3750504D38434891
:1006F0003120434832204348332043483420434884
:100700003520434836204348372043483820434863
:10071000392043483130434831314348313243482E
:100720003133434831344348313543483136002D65
:100730002D2D2D00564552533A2056312E35353049
:10074000302D6572657A00444154453A2031312E8E
:1007500030322E323031320054494D453A2031305A
:100760003A31303A3338002053564E3A20657239C8
:10077000782D7237303800204D4F443A20204E48B3
:100780005420200012081200081C0808081C080049
:1007900000082200490022080000000000227F22F9
:1007A0000000000822004900220800000822004939
:1007B000002208000000227F220000000000082222
:1007C00000490022080000081C0808081C08005402
:1007D000307141D82AC023C651A84EA5463F48E4EF
:1007E00048C01C7B1EB11E511FCC2054546D0045C7
:1007F0007870457846466E654D6564437273005463
:100800004F540053544B1153542500544D4511542B
:1008100053570053544154005B4D454E555D207471
:100820006F207265667265736800537461636B0F45
:100830006200746D61696E0F6D7300746D723120AA
:100840004A69747465720F757300746D72314C610E
:1008500074206D696E0F757300746D72314C617424
:10086000206D61780F7573005354415432004D6F01
:1008700064650042616E6447617000506F74536339
:10088000726F6C6C00416C61726D205761726E69A1
:100890006E67004D656D6F7279205761726E696E7B
:1008A000670054524530313241470054524530318F
:1008B0003241470044656661756C7420537700537C
:1008C0007769746368205761726E696E6700546857
:1008D000726F74746C65205761726E696E67005335
:1008E000706C617368204E616D650053706C61734C
:1008F000682073637265656E004F4646004C6967F9
:100900006874206F6E2053746B204D76004C6967BD
:100910006874206F6666206166746572004C696752
:1009200068742073776974636800466C617368202B
:100930006F6E2062656570004265657020636F753B
:100940006E74646F776E004D696E757465206265B4
:100950006570005468726F74746C6520726576659A
:100960007273650053494E474F534D5046494C549E
:100970000046696C7465722041444300496E6163AE
:1009800074697669747920616C61726D004261747A
:1009900074657279207761726E696E6700436F6E5D
:1009A0007472617374004861707469632053747267
:1009B000656E67746800537065616B65722050697D
:1009C00074636800426565706572506953706B723C
:1009D00000536F756E64204D6F64650051756965D5
:1009E00074204E6F4B6579207853686F727453682A
:1009F0006F7274204E6F726D20204C6F6E672020D6
:100A0000784C6F6E672000426565706572004F77A5
:100A10006E6572204E616D6500524144494F20530E
:100A2000455455500043616C004D756C7469706C91
:100A30006965720063683163683263683363683480
:100A4000006F6666202B3D203A3D006D6F64650A9D
:100A500025207372632020737700536C61766500E4
:100A6000545241494E4552000003030303005645CA
:100A70005253494F4E005472696D2D202B00204D6A
:100A8000656E75204578697420446F776E2020204C
:100A900055705269676874204C656674004449411A
:100AA0004700424700414E41005B4D454E555D2099
:100AB0005748454E20444F4E45004D4F5645205314
:100AC0005449434B532F504F545300534554204DDA
:100AD0004944504F494E54005B4D454E555D20549E
:100AE0004F205354415254005354415254204341D7
:100AF0004C4942524154494F4E0043414C494252A5
:100B00004154494F4E0066726565004D4F44454C57
:100B100053454C0044454C455445204D4F44454CAD
:100B20000F5B4D454E555D005432546854726967F1
:100B300000547261696E657200452E204C696D69C2
:100B4000747300504F534E454700536869667420D4
:100B500053656C004C50342F4C5035202044534D7D
:100B6000326F6E6C792044534D322F44534D5800F0
:100B700044534D20547970650053656E642052785B
:100B8000204E756D626572205B4D454E555D00507F
:100B9000504D2046724C656E0D6D536563002052BA
:100BA000784E756D0034434820364348203843481A
:100BB00020313043483132434831344348313643A1
:100BC0004800755300755365630050504D20202038
:100BD00050585820202044534D32202050504D3141
:100BE00036200050726F746F0052455441313233D9
:100BF000004265657020436E74005472696D205325
:100C00007700457870202020457846696E654669F2
:100C10006E6520204D656469756D436F6172736503
:100C2000005472696D20496E6300542D4578706FD1
:100C300000542D5472696D00436F756E7420446FBB
:100C4000776E436F756E7420557020200054696D67
:100C500065722000547269676765720054696D653A
:100C600072004E616D6500534554555000000901F6
:100C70000000000000000602004475706C696361AA
:100C800074696E67206D6F64656C005B4D454E55F1
:100C90005D20205B455849545D005945530B4E4F2C
:100CA0000044454C455445204D4F44454C00445567
:100CB000504C4943415445204D4F44454C00204140
:100CC00042434445464748494A4B4C4D4E4F50518C
:100CD00052535455565758595A6162636465666752
:100CE00068696A6B6C6D6E6F70717273747576770C
:100CF00078797A303132333435363738395F2D2EC2
:100D0000006578702020252020737731207377329A
:100D1000004558504F2F4452000003445220486968
:100D20006768004452204C6F77004452204D69643C
:100D3000004472537732004472537731005765692B
:100D4000676874004578706F004558504F2F4452C3
:100D500000002B2A52004D495845520050726573CD
:100D600073205B455849545D20746F2061626F7237
:100D700074004D6178206D697865727320726561C9
:100D800063683A200044454C455445204D4958205D
:100D90005B4D454E555D00536C6F772020557000BC
:100DA000536C6F772020446F776E0044656C6179D7
:100DB0002055700044656C617920446F776E004166
:100DC000646420202020204D756C7469706C795209
:100DD00065706C61636520004D756C747078004FB0
:100DE0004646005761726E696E6700537769746397
:100DF0006800437572766573004F4E204F4646007B
:100E00005472696D004F46464F4E2000466C4D6F40
:100E100064657472696D004F666673657400466D33
:100E20005472696D56616C00576569676874005348
:100E30006F757263650045444954204D4958200040
:100E4000494E53455254204D495820002D2D2D2DEB
:100E5000202020763E6F66732020763C6F667320DC
:100E6000207C767C3E6F66737C767C3C6F6673413B
:100E70004E44202020204F522020202020584F5226
:100E80002020202076313D3D7632207631213D767E
:100E9000322076313E7632202076313C7632202068
:100EA00076313E3D76322076313C3D76322000531D
:100EB0005700435553544F4D2053574954434845C9
:100EC0005300000253414645545920535749544357
:100ED000484553000002434F5059205452494D2079
:100EE0005B4D454E555D002D2D2D494E56004C490C
:100EF0004D49545300000303030303030303030397
:100F0000030303030303004356004355525645535E
:100F10000050524553455400454449542D3E00432A
:100F2000555256450009002D2D2D494E56004F466D
:100F3000464F4E20002D2D2D783E30783C307C7869
:100F40007C663E30663C307C667C633120633220B8
:100F50006333206334206335206336206337206396
:100F6000382063392063313063313163313263318A
:100F70003363313463313563313600454550524F68
:100F80004D206F766572666C6F7700454550524F05
:100F90004D206F766572666C6F770067656E77724D
:100FA000697465206572726F7200454550524F4DED
:100FB00020466F726D617474696E670042616420CF
:100FC000454570726F6D2044617461004D4F44451A
:100FD0004C2020202020004D4520202020202020B3
:100FE000200050085000000000000000006F0000CA
:100FF00007000700147F147F14242A7F2A1223136A
:1010000008646236495522500005030000001C2286
:1010100041000041221C0014083E081408083E0844
:101020000800503000000808080808006060000050
:101030002010080402003E49453E0000427F400067
:10104000625149460041494936001814127F002771
:10105000454539003E4949320001790503003649CA
:101060004936000649291E00003636000000563673
:10107000000008142241141414141441221408000E
:10108000020151090600060909067E0909097E7F49
:10109000494949363E414141227F4141221C7F4915
:1010A0004949417F090909013E4149497A7F0808B8
:1010B000087F00417F41002040413F017F0814220A
:1010C000417F404040407F020C027F7F0408107F38
:1010D0003E4141413E7F090909063E4151215E7F63
:1010E00009192946264949493201017F01013F403A
:1010F00040403F1F2040201F3F4030403F631408C6
:10110000146307087008076151494543007F414156
:101110000002040810200041417F00040201020483
:101120004040404040000102040020545454787F65
:10113000484444383844444420384444487F385470
:10114000545418087E0901020C5252523E7F080482
:10115000047800447D40002040443D007F10284436
:101160000000417F40007C041804787C0804047867
:1011700038444444387C14141408081414187C7C33
:10118000080404084854545420043F4440203C4080
:1011900040207C1C2040201C3C4020403C44281027
:1011A00028440C5050503C4464544C440008364190
:1011B0000000007F000000413608000808221C08DB
:1011C000081C220808A06080000000000000000049
:1011D000000000000000FFFF0000000000001F3FB3
:1011E00000003F1F00003030FFFF3030FFFF303085
:1011F0003078CCCCFFFFCCCC8C0C060F0F86C0E037
:1012000070381C0C3CFEC7E3F33B1E0C00000000D2
:10121000333B1F0F000000000000F0F81C0E070316
:101220000000000003070E1CF8F000003030E0C0A2
:10123000FCFCC0E03030C0C0C0C0FCFCC0C0C0C0BE
:1012400000000000000000000000C0C0C0C0C0C01E
:10125000C0C0C0C00000000000000000000000008E
:101260000080C0E070381C0C00000000000000008E
:1012700000000000000038380000000000000000FE
:1012800000000000000003033F3F03033F3F030350
:101290000C0C0C0C3F3F0C0C07030C0E0703010059
:1012A000183C3C180F1F383133331E1E33330000F7
:1012B0000000000000000000000003070E1C383092
:1012C0000000000030381C0E07030000030301007B
:1012D0000F0F00010303000000000F0F00000000CB
:1012E0000000333B1F0F0000000000000000000062
:1012F000000000000000183C3C18000000000C0E2C
:1013000007030100000000000000FCFE87C3E37734
:10131000FEFC00000C0EFFFF0000000000000C0EA1
:101320000783C3E77E3C00000303C3C3C3E7FE3C5F
:101330000000C0E070381C0EFFFF00003F3F333359
:101340003373E3C30000FCFEC7C3C3C78E0C0000A9
:101350000303C3E3733B1F0F00003CFEE7C3C3E777
:10136000FE3C00003C7EE7C3C3E7FEFC0000183CE7
:101370003C18000000000000183C3C180000000071
:101380000000C0E0F0381C0E070330303030303041
:101390003030303003070E1C38F0E0C000000C0E77
:1013A00007030383C3E77E3C00000F1F3B31303847
:1013B0001F0F000030303F3F3030000000003C3E47
:1013C00037333130303000003030303030391F0F9B
:1013D00000000303030303033F3F00000C1C3830ED
:1013E00030381F0F00000F1F383030391F0F00003A
:1013F00000003F3F0000000000000F1F393030396F
:101400001F0F0000000030381C0E07030000060FFD
:101410000F06000000000000333B1F0F000000001B
:101420000000000103070E1C38300303030303030D
:101430000303030330381C0E070301000000000003
:10144000000033330100000000003C7EE7C3C3E727
:101450007E3CF0F8DCCEC7C7CEDCF8F0FFFFC3C39C
:10146000C3C3C3E7FE3CFCFE0703030303070E0CE4
:10147000FFFF030303070E1CF8F0FFFFC3C3C3C342
:10148000C3C30303FFFFC3C3C3C3C3C30303FCFE40
:101490000703C3C3C3C7CECCFFFFC0C0C0C0C0C01A
:1014A000FFFF00000303FFFF030300000000000034
:1014B0000303FFFF0303FFFFC0E0F0381C0E070328
:1014C000FFFF0000000000000000FFFF0E1CF8F806
:1014D0001C0EFFFFFFFF3870E0C08000FFFFFCFE26
:1014E000070303030307FEFC0000000000000000E8
:1014F00000003F3F0000000000003F3F3F3F303012
:10150000303030391F0F0F1F3830303030381C0C5E
:101510003F3F303030381C0E07033F3F3030303013
:10152000303030303F3F00000000000000000F1F4F
:101530003830303030303F3F3F3F00000000000087
:101540003F3F000030303F3F303000000C1C38304F
:1015500030381F0F00003F3F000103070E1C3830DA
:101560003F3F30303030303030303F3F00000000FF
:1015700000003F3F3F3F0000000103033F3F0F1FBC
:101580003830303030381F0FFFFFC3C3C3C3C3E749
:101590007E3CFCFE070303030307FEFCFFFFC3C3FF
:1015A000C3C3C3E77E3C3C7EE7C3C3C3C3C78E0C43
:1015B00003030303FFFF03030303FFFF0000000017
:1015C0000000FFFFFFFF000000000000FFFFFFFF23
:1015D000000000000000FFFF0F1F38F0E0E0F038CF
:1015E0001F0F3F7FE0C08080C0E07F3F0303038385
:1015F000C3E3733B1F0F0000FFFF0303030300005F
:101600000C1C3870E0C080000000000003030303DE
:10161000FFFF000030381C0E07070E1C383000009A
:1016200000000000000000003F3F0000000000003C
:1016300000000F1F383033371E1C3F333F3F000080
:1016400003070E1C38300C1C3830303030391F0F77
:10165000000000003F3F000000000F1F3830303016
:1016600030381F0F03070E1C38381C0E07030F1FDE
:1016700038381F1F38381F0F3C3E0703010103078E
:101680003E3C000000013F3F010000003C3E37337C
:1016900031303030303000003F3F303030300000EB
:1016A00000000000000103070E0C00003030303055
:1016B0003F3F00000000000000000000000030304C
:1016C0003030303030303030000003070E1C3830FE
:1016D00000000000303030303070E0C0FFFFC0E06C
:1016E00070303070E0C0C0E070303030303000001A
:1016F000C0E070303070E0C0FFFFC0E070303030CC
:101700003070E0C0C0C0FCFEC7C303070E0CF0F889
:101710009C0C0C0C0C0CFCFCFFFFC0E0703030701B
:10172000E0C000003030F3F30000000000000000D3
:101730003030F3F30000FFFF0080C0E070300000A5
:1017400000000303FFFF00000000F0F03070E0E055
:101750007070E0C0F0F0C0E070303070E0C0C0E009
:10176000703030303070E0C0000000000000000039
:1017700000000C1E3F33333333333F3F3F3F3030A5
:10178000303030381F0F0F1F3830303030381C0CDD
:101790000F1F3830303030303F3F0F1F3B33333373
:1017A0003333030300003F3F00000000000000014E
:1017B00033333333333B1F0F3F3F00000000000043
:1017C0003F3F000030303F3F303000000C1C3830CD
:1017D00030381F0F00003F3F03070F1C3830000058
:1017E000000030303F3F303000003F3F0000030337
:1017F00000003F3F3F3F0000000000003F3F0F1F41
:101800003830303030381F0FF0F03030303030F0BA
:10181000E0C0C0E0F0303030E0C0F0F0F0F0C0E008
:1018200070303070E0C0C0E0F03030303030000058
:101830003030FFFF303000000000F0F0000000000A
:101840000000F0F0F0F0000000000000F0F0F0F018
:10185000000000000000F0F03070E0C08080C0E0C8
:101860007030F0F0800000000000F0F030303030D8
:1018700030B0F0F070300000C0E03C3E07030000E4
:1018800000000000FFFF00000000000003073E3CD6
:10189000E0C00000C0C0C0C00C1CF8F0E0C0C0E058
:1018A000F0F81C0CC0C0C0C03F3F03030303030398
:1018B000010000010303030303033F3F3F3F000018
:1018C000000000000000303133333333333F1E0C4F
:1018D00000000F1F383030381C0C0F1F38303038E4
:1018E0001C0C3F3F03070E1C38381C0E07030F1F4C
:1018F00038381C1C38381F0F30381C0F07070F1CD6
:101900003830000133333333333B1F0F30383C3E24
:10191000373331303030000000010F1F3830000005
:10192000000000003F3F00000000000030381F0FA3
:1019300001000000000000000C0E07030100000180
:1019400003070E0C00000000408008042010020174
:101950000000891112239B322446AD573665BF74AF
:10196000488CC19D5AAFD3BE6CCAE5DB7EE9F7F85F
:101970008110080193331A22A5562C47B7753E648F
:10198000C99C408DDBBF52AEEDDA64CBFFF976E83F
:1019900002218B30100299132667AF763444BD556F
:1019A0004AADC3BC588ED19F6EEBE7FA7CC8F5D91F
:1019B00083310A2091121803A7772E66B5543C454F
:1019C000CBBD42ACD99E508FEFFB66EAFDD874C9FF
:1019D00004428D5316619F702004A9153227BB362F
:1019E0004CCEC5DF5EEDD7FC6888E1997AABF3BADF
:1019F00085520C4397711E60A1142805B3373A260F
:101A0000CDDE44CFDFFD56ECE9986089FBBB72AABE
:101A100006638F7214409D512225AB343006B917EE
:101A20004EEFC7FE5CCCD5DD6AA9E3B8788AF19B9E
:101A300087730E6295501C41A3352A24B1163807CE
:101A4000CFFF46EEDDDC54CDEBB962A8F99A708B7E
:101A5000088481951AA793B62CC2A5D33EE1B7F0AE
:101A60004008C919522BDB3A644EED5F766DFF7C5E
:101A7000899400859BB712A6ADD224C3BFF136E08E
:101A8000C1184809D33B5A2AE55E6C4FF77D7E6C3E
:101A90000AA583B4188691972EE3A7F23CC0B5D16E
:101AA0004229CB38500AD91B666FEF7E744CFD5D1E
:101AB0008BB502A499961087AFF326E2BDD034C14E
:101AC000C3394A28D11A580BE77F6E6EF55C7C4DFE
:101AD0000CC685D71EE597F42880A1913AA3B3B22E
:101AE000444ACD5B5669DF78600CE91D722FFB3EDE
:101AF0008DD604C79FF516E4A9902081BBB332A20E
:101B0000C55A4C4BD7795E68E11C680DF33F7A2EBD
:101B10000EE787F61CC495D52AA1A3B03882B193ED
:101B2000466BCF7A5448DD59622DEB3C700EF91F9D
:101B30008FF706E69DD414C5ABB122A0B9923083CD
:101B4000C77B4E6AD5585C49E33D6A2CF11E780F7D
:101B5000301911241FBECFEFD0E1DEBFCDBF11E0A1
:101B6000A0E0B1E0EEE7F2ED02C005900D92A832E0
:101B7000B107D9F71EE0A8E2B1E001C01D92AA3575
:101B8000B107E1F71BE1C2E5DBE104C02297FE01EA
:101B90000E94F868C035D107C9F70E9462180C94FA
:101BA0003D690C94000030919B0422B780919B0406
:101BB0003817C9F7932F80E030E0282B392BC90163
:101BC000089529E2820290011124359527953595D3
:101BD000279587FD815C86FB880F880B80F9992704
:101BE00087FD9095281B390BC9010895F894209121
:101BF000B70D3091B80D7894C9010895482F50E081
:101C00009A01220F331F63E0440F551F6A95E1F7D5
:101C1000240F351F2E553E4FC901089590E09C01B9
:101C2000220F331F220F331F280F391F2E513D4F14
:101C3000C9010895AF92BF92CF92DF92EF92FF92C7
:101C40000F931F93CF93DF93C82E162FEA01F22E26
:101C5000D02E57FF10C022FF02C08CE101C08FE0E0
:101C60009C2D981B892F612F4DE22F2D0E94255A04
:101C7000D095C195DF4F2D2D2F218C2D612F4AE35B
:101C80000E94255A8F2D90E0B4E0AB2EB12CA822F3
:101C9000B922F2FE02C0E2E001C0E0E0CE016CE356
:101CA00070E00E94A6689B01442737FD4095542FA1
:101CB0000F2D00618E2F8C0D612FA2E0EA2E0E9465
:101CC000255CA114B10411F0ECE101C0E1E1CE0109
:101CD0006CE370E00E94A6689C01442737FD4095A4
:101CE000542F0D2D00618E2F8C0D612FF2E0EF2E01
:101CF0000E94255CDF91CF911F910F91FF90EF9093
:101D0000DF90CF90BF90AF9008950F931F93062F51
:101D1000122F206250E00E945B5D17FD07C080918A
:101D2000890D602F46E7212F0E94255A1F910F91A0
:101D30000895242F409108010E94850E08950F9365
:101D4000022F442319F44FE257E020C04530A8F495
:101D5000E0916C01F0E0EE0FFF1FEE0FFF1F3197D7
:101D6000E40FF11DE051FB4F449150E0440F551F2B
:101D7000440F551F4756594F09C0453250F450E0A3
:101D8000440F551F440F551F4656594F24E00E94DB
:101D9000E85A0F910895FF920F931F93182FF62E74
:101DA000022F442321F448E956E024E00EC08A5E65
:101DB0004A3008F485506F2D50E0202F0E945B5D63
:101DC000812F6F2D45E956E022E00E94E85A1F91CD
:101DD0000F91FF9008950F931F93DF93CF9300D03F
:101DE000CDB7DEB7382F162F942F022F442329F0BA
:101DF000463139F04A3E81F408C08A5F41E956E035
:101E000007C08A5F4DE856E003C08A5F49E856E0A4
:101E1000202F0E94185B28C04095441F4427441F70
:101E200081E2841B482F832F39839A830E94255A8D
:101E30003981832F8A5F9A81E92FFF27E7FDF0958B
:101E4000F7FF03C0F095E195FF4FFF27E7FDF09501
:101E50003197AF01440F551F4E0F5F1F475B594F1E
:101E6000612F23E00E94E85A0F900F90CF91DF91ED
:101E70001F910F91089589E496E00895DF92EF9203
:101E8000FF920F931F93D82EE62EF42E10919301FC
:101E9000E12FFF27E7FDF095F7FF03C0F095E195EF
:101EA000FF4FE031A4F483E0E802F0011124E85E82
:101EB000F94F8D2D6E2DAF0123E00F2D0E94E85AB2
:101EC0001F3F3CF58D2D86506E2D41E21FC08D2D9C
:101ED0008650E53264F411161CF4412F4F5002C0B5
:101EE000412F415F6E2D2F2D0E94EB0E12C0111657
:101EF0001CF4412F445202C0412F4C5D6E2D2F2DFA
:101F00000E94EB0E8D2D8E5E6E2D4DE62F2D0E94C4
:101F1000255A1F910F91FF90EF90DF9008958C301C
:101F200038F4E82FF0E0EE0FFF1FEB52FB4F2AC012
:101F3000803198F4E82FF0E0DF01AA0FBB1FAE5804
:101F4000BB4FEE0FFF1FEE5BFE4F2D913C911197A3
:101F500080819181281B390B0AC0843158F4E82F05
:101F6000F0E0EE0FFF1FEE58FB4F20813181220F72
:101F7000331F0DC0843248F4E82FF0E0EE0FFF1F4E
:101F8000E554FB4F2081318102C020E030E0C901DF
:101F90000895AF92BF92DF92EF92FF920F931F933B
:101FA000DF93CF9300D0CDB7DEB7F82E463008F0E0
:101FB000DEC0882309F4DEC0863119F08A3E19F4A8
:101FC000D6C061E0D7C0992787FD90959C0197FF07
:101FD00004C022273327281B390B2A307CF41F1416
:101FE0004CF02DE030E0A901481B590BCA010E94BA
:101FF000C55EBAC00D960E94C55EBBC02A50A22E17
:10200000BB249501220F331F2A0D3B1D28573E4F3D
:10201000F901E85AFD4F5081552309F4A8C0453015
:1020200029F4F501EA59FB4F80819CC0F901EA5A75
:10203000FD4FD080295A3D4FF901E080553008F41A
:10204000A6C0583060F08D2D81504A8359830E947C
:102050008F0F8C018E2D81500E948F0FA2C020E027
:1020600030E000E010E0583088F4553088F5523008
:1020700009F462C0533020F4513009F06EC057C0EB
:102080005330D1F0543009F068C01CC05A3009F404
:102090004EC05B3038F4583009F43FC0593009F075
:1020A0005CC040C05C3009F44CC05C3008F444C0F3
:1020B0005D3009F052C04AC017FF39C01095019534
:1020C0001F4F35C017FF38C0109501951F4F34C002
:1020D000142F1F5F8D2D60E0412F0E94C90F082F24
:1020E0008E2D60E0412F0E94C90FF501EE0FFF1FFA
:1020F000EA0DFB1DE052FC4F9081953029F400233E
:1021000061F1882341F52AC0963029F4002319F59E
:10211000882319F120C0802721C081E0021713070E
:10212000E1F41CC081E002171307C1F416C081E07E
:10213000201731079CF011C081E00217130774F0DB
:102140000CC081E0021713074CF407C081E0201790
:10215000310724F402C081E001C080E0F501EA59B2
:10216000FB4F80831F142CF061E0682703C060E000
:1021700001C0682F862F0F900F90CF91DF911F9194
:102180000F91FF90EF90DF90BF90AF9008958D2D4D
:1021900081504A8359830E948F0F8C018E2D0E949B
:1021A000E10D9C014A8159815ECF86B380958E777F
:1021B00008950E94D5108823E1F70E94345E0895A7
:1021C0008091590160E040E00E94C90F882331F4FA
:1021D0008091830490918404009711F0C79A089528
:1021E000C79808950F931F93CF93DF93EC018B0152
:1021F0000E94BB5982E260E043E056E024E00E9486
:10220000185B80E2BE010E943F5B88E2B8010E9439
:102210003F5B80E36DEE75E00E943F5B0E94C55D11
:10222000809156010E94BB5D0E94D910DF91CF9131
:102230001F910F9108950F93AB0160E123E000E03F
:102240000E94E85A0F910895DF92EF92FF920F9348
:102250001F93CF93DF9380916B0181FD83C080E852
:1022600095E06AE675E00E94F21090918301892F53
:10227000887341F0883131F0883221F0803311F0D9
:10228000883329F4892F877C88608093830100E05C
:1022900010E065E1E62EF12C08C0C701801B910912
:1022A0000E94C55E110F182B0F5F0830B0F3D0905D
:1022B0008301D12680E060E143E555E026E100E0BE
:1022C0000E94E85ACD2DD0E0CE0180FF05C082E00B
:1022D00069E476E00E941B11C1FF05C087E16CE450
:1022E00076E00E941B11C2FF05C08CE26FE476E02D
:1022F0000E941B11CE01887390700097B1F0012FDE
:1023000013FF05C081E462E576E00E941B1104FF23
:1023100005C081E465E576E00E941B1105FF05C05C
:1023200081E468E576E00E941B11C6FF05C086E5E2
:102330006BE576E00E941B11D7FE05C08BE66EE5CB
:1023400076E00E941B110E94C55D809183011817E1
:1023500049F00E94D510882329F40E94E01000E083
:1023600010E09BCFDF91CF911F910F91FF90EF90E5
:10237000DF9008951F93CF93DF930E94D51020E044
:1023800030E011E0482F50E02F5F3F4FBA01022E9E
:1023900002C0759567950A94E2F760FD03C01F5F60
:1023A000183091F71150163030F5812F0E943654B5
:1023B000882309F110935501812F0E943A5481E03E
:1023C0000E9409550E94BB5986E160E04BE455E04C
:1023D00024E00E94185BC8E8D1E01AE04991812FFF
:1023E00068E124E00E94255A155F1837B9F70E946A
:1023F000C55D0E94D910DF91CF911F910895CF93B1
:10240000DF93EC010E94BB5982E260E043E455E0B7
:1024100024E00E94185B88E1BE010E943F5B0E949D
:10242000C55D809156010E94BB5DDF91CF910895FB
:102430001F93CF93DF93EC01162F0E94BB5982E2CA
:1024400060E04DE355E024E00E94185B88E1BE01A6
:102450000E943F5B8CE168E34FE255E00E94475BDE
:102460000E94C55D112319F48091560101C089E1D4
:102470000E94BB5D82E10E9460680E94D9100E94A8
:10248000D5108823C9F480914B0E833019F4A89598
:1024900010924B0E8091590160E040E00E94C90FFC
:1024A000882331F480917001882311F4112311F0F5
:1024B000C79AE5CFC798E3CFDF91CF911F910895D9
:1024C00080916504882351F081E995E060E00E94E5
:1024D0001812809165048E7F809365040895809121
:1024E0006B0187FD07C0887329F48CEB95E060E0F1
:1024F0000E941812089580916B0182FD0AC00E940B
:102500002A56883C910528F489E096E060E00E9414
:1025100018120895EF92FF92CF93DF93A82FAF7018
:10252000A65090919A01923074F0292F332727FDFD
:10253000309521503040C1E0D0E002C0CC0FDD1F0B
:102540002A95E2F79C2FA83008F09CC06A2F659569
:1025500070E0FB01EE0FFF1FE050FF4F0190F08194
:10256000E02DB081992379F4CB2FDD27C7FDD095DD
:10257000D7FF03C0D095C195DF4F9C2FC7FD9D5F4E
:10258000959595959F5F40916C0150E0417050701A
:1025900022E030E0241B350B2617370769F4209121
:1025A00099012F7009F473C021E094E030916E011D
:1025B00030FF03C0919501C020E04B2F552747FD08
:1025C0005095C92FDD27C7FDD095A0FF03C0C40FCC
:1025D000D51F04C0BA016C1B7D0BEB01209729F0BD
:1025E0007E019F2D9B2797FF0BC0222349F4BB231D
:1025F00039F010820E94245F86E10E94606841C029
:10260000CE0184589F4F893F9105B8F4C08386E07E
:102610000E940955CE0183589F4F8B3F910588F545
:10262000D7FF03C0D095C195DF4FD595C795D595F8
:10263000C795BE01645C462F1FC01C161D0614F40E
:102640008DE701C083E8808386E00E940955CE01B2
:1026500083589F4F8B3F9105A0F4CE01D7FF03C055
:10266000909581959F4F64E070E00E94A6687095F8
:1026700061957F4F462F445C8DE294E065E10E94B6
:10268000ED6680E0DF91CF91FF90EF90089520E01C
:102690008DCF8F929F92AF92BF92CF92DF92EF92A7
:1026A000FF920F931F93CF93DF93182FEB015A01E3
:1026B0006901802E84FF06C01F70106694E0992E79
:1026C00005E003C085E0982E04E0802F806618178F
:1026D00061F0802F8064181741F0809104058823F1
:1026E00069F0133611F0133449F47E010894E11CAB
:1026F000F11C83E10E946068892D18C0992D9066B5
:10270000191761F0992D9064191741F0882309F485
:1027100074C0123619F0123409F06FC07E010894AB
:10272000E108F10884E10E946068802F90E00E9437
:10273000C55E882351F0EE24FF24EC1AFD0A892D92
:102740000E94245F802F0E94245FA114B10491F4A1
:1027500081E0C816D10471F4103661F410920405BA
:1027600001E0E02EF12C209711F0EE24FF2480E60A
:102770000E94245F2091800430918104E21AF30AC0
:10278000CE14DF0444F4812F0E94245F83E10E9471
:10279000606876010AC0EA14FB043CF4812F0E94B1
:1027A000245F84E10E9460687501EC16FD06A9F0C3
:1027B000E114F10451F4812F0E94155FD7FF02C08C
:1027C00083E101C084E10E946068882D83700E94CB
:1027D000095581E080937D0402C010927D04C701F9
:1027E000DF91CF911F910F91FF90EF90DF90CF90ED
:1027F000BF90AF909F908F9008957E01A6CF0F93CA
:10280000772767FD7095552747FD5095332727FD9E
:1028100030950E9449130F9108950F93772767FD14
:102820007095552747FD5095332727FD309502E0D9
:102830000E9449130F9108950F93772767FD7095B4
:10284000552747FD5095332727FD309501E00E941D
:1028500049130F910895E0917C04F0E0EE0FFF1F03
:10286000EC58FB4F80819181089590917C049923CD
:1028700019F4882331F418C0882319F4892F815062
:1028800001C080E080937C0487E10E946068E09151
:102890007C04F0E0EE0FFF1FEE58FB4F0190F0813B
:1028A000E02D8EEB099508958BE195E060E00E94A4
:1028B00018120895FC01A0917C04B0E0AA0FBB1F80
:1028C000AE58BB4F8D939C938FEB099587E10E9487
:1028D00060680895CF93DF93EC0180917C04982F7A
:1028E0009F5F90937C04953040F080937C0488E057
:1028F00095E060E00E9418120FC087E10E946068B6
:10290000E0917C04F0E0EE0FFF1FEE58FB4FD18307
:10291000C0838FEBFE010995DF91CF9108958DE281
:1029200094E00E94EC65882311F084E105C0809159
:102930009C04882321F0815080939C0407C09091CF
:10294000630081E091FF80E080939D0480919D046D
:1029500008951092870410928904109288041092AE
:102960008604089520918304309184042115310553
:1029700031F0215030403093840420938304882325
:1029800069F04091700150E084EF91E0489F900120
:10299000499F300D589F300D112402C020E030E0D7
:1029A00080918504882369F06091780170E044EF9C
:1029B00051E0649FC001659F900D749F900D11249C
:1029C00002C080E090E0409183045091840442175B
:1029D000530720F4309384042093830420918304CC
:1029E000309184042817390720F49093840480934D
:1029F00083040E94E0100895E82FF0E0E050FB4FC0
:102A0000E491F0E0EE0FFF1FE056FB4F2081318193
:102A1000C9010895CF92DF92EF92FF920F931F9317
:102A2000DF93CF930F92CDB7DEB720E0CC24DD2427
:102A3000822F29830E94FC14092F10E0C00ED11EA2
:102A400029812F5F2430A1F7C6010F90CF91DF912C
:102A50001F910F91FF90EF90DF90CF9008951F93FB
:102A60000E94F60D41E02091D3043091D4048217E6
:102A7000930709F440E0409382040E94F60D90937E
:102A8000D4048093D30489E095E060E00E949634FA
:102A900080918204882309F4CBC08091860480FF52
:102AA00014C080918704982F9F5F90938704943679
:102AB00060F0835680938704809188049091890404
:102AC0000196909389048093880480E00E941755B2
:102AD0000E94BB590E94375E0E948A12182F0E94E2
:102AE000B2142091E1043091E20480917E0490912F
:102AF0007F04821B930B60E270E00E94A6687093D3
:102B00008104609380046115710591F08091D10476
:102B10009091D204821B930B62E070E00E94A66841
:102B2000709381046093800430937F0420937E042B
:102B30003093D2042093D10480916E0185FF04C0AC
:102B40001092810410928004E0917C04F0E0EE0F7A
:102B5000FF1FEE58FB4F0190F081E02D812F09956A
:102B60000E94C55D0E948F14882321F0809165002A
:102B70008F7E03C0809165008061809365000E9414
:102B8000F60D8F7190708230910509F04FC087E08B
:102B90000E94FC149C01E4E0220F331FEA95E1F748
:102BA00068E070E00E94A66840915801552747FDF3
:102BB00050954A5F5F4F649FC001659F900D749F61
:102BC000900D1124820F931F20916E0126FD05C0E8
:102BD0006091090170910A0102C060EF70E02091DC
:102BE000080130E02F5F3F4F0E949268260F371F89
:102BF00035952795209308018091D004805E8093BD
:102C0000D004882399F480915701281778F422334F
:102C100068F081E10E94606880916E0183FF06C0C8
:102C200082E390E09093840480938304109285045F
:102C30001F910895A0EAB4E0E0EBF4E060E0862F95
:102C4000806487B9369A408951898D919C911197FA
:102C500096958795840F951F8E7F11969C938E93E2
:102C600020813181C901840F951F96958795918B9D
:102C7000808B349BFECF349A84B195B1820F931F21
:102C800096958795819391936F5F12966830B9F608
:102C90000895EF92FF920F931F93CF93DF9380914C
:102CA0006E0184FD44C00E94E0100E94BB5980E088
:102CB00060E045ED50E020E000E00E94C6598091C0
:102CC000740184FD08C080E068E349E751E02AE030
:102CD00000E10E94E85A0E94C55D809156010E9461
:102CE000BB5D0E94D91000E20E941A160150E1F764
:102CF0000E940A158C010E94F60DEC01C057DE4FB0
:102D00000DC00E941A160E940A157C010E94D5105F
:102D1000882369F4E016F10651F406C00E94F60D0E
:102D2000C817D90771F703C00E94E010F7CFDF91F1
:102D3000CF911F910F91FF90EF900895E0EAF4E09A
:102D400040E012C067B9369A349BFECF349A24B162
:102D500035B1820F931F5150A9F7969587958193AE
:102D600091934F5F483031F054E080E090E0642F61
:102D70006064E8CF0895E0EAF4E020E0822F806408
:102D800087B9369A349BFECF349A84B195B1880FB7
:102D9000991F819391932F5F283081F70895FF92B7
:102DA0000F931F93CF93DF9380916B0180FD3AC007
:102DB00080916C0190E08170907002E010E0081B3F
:102DC000190BF801EE0FFF1FE85DFE4FC181D281A4
:102DD000609687859089C81BD90B0E94BB16F02E80
:102DE000802F0E94FC14C817D907E4F40E94D51064
:102DF0008823C1F40DC00E94BB168F2D0E94FC14C5
:102E0000C817D9077CF40E94D510882341F00AC066
:102E10008BED95E06CEC75E00E94F210ECCF0E9417
:102E2000E010E9CFDF91CF911F910F91FF900895AE
:102E30008EE587B9369A349BFECF349A84B195B12A
:102E400004964091090150910A019A0163E0220F12
:102E5000331F6A95E1F7241B350B820F931F23E084
:102E6000969587952A95E1F790930A018093090139
:102E7000089578941F920F920FB60F9211248F939A
:102E800080919B048F5F80939B048F910F900FBE66
:102E90000F901F90189578941F920F920FB60F9273
:102EA00011242F933F934F935F936F937F938F934F
:102EB0009F93AF93BF93EF93FF93F89487B78D7F62
:102EC00087BF789481B78E5F81BF90912F048091E6
:102ED0003104882379F080917701882349F081308B
:102EE00051F48091590E890F8093590E87FF02C0CB
:102EF0001B9A01C01B9880910B01982F91509093C1
:102F00000B01882371F48DE480930B018DE294E032
:102F10000E9400660E94355F80914B0E8260809314
:102F20004B0EF89487B7826087BF7894FF91EF913A
:102F3000BF91AF919F918F917F916F915F914F91D1
:102F40003F912F910F900FBE0F901F90189578947E
:102F50001F920F920FB60F9211241F932F933F933E
:102F60004F935F936F937F938F939F93AF93BF9391
:102F7000EF93FF932091800030918100F89480912D
:102F80007D008F7D80937D00789480919E04909148
:102F90009F04A901481B590BCA0196958795309348
:102FA0009F0420939E0410919A04212F21502830D1
:102FB00058F59C012152334055E02737350708F575
:102FC000E12FF0E0EE0FFF1FE857FB4FAC014C5D27
:102FD000554020917201332727FD3095265F3F4FE2
:102FE000429FC001439F900D529F900D11246AE0B3
:102FF00070E00E94A668718360831F5F10939A043B
:103000000CC010929A0409C0815A9F402EE28F3D55
:10301000920718F481E080939A04F89480917D00DF
:10302000806280937D007894FF91EF91BF91AF9182
:103030009F918F917F916F915F914F913F912F91D0
:103040001F910F900FBE0F901F901895EBE5FEE0BB
:103050009F0181918535E1F32A553E40C9010895CC
:10306000CF93DF930E94D30DEC0180916F018130EB
:1030700019F40E941A1607C0823019F40E949E1695
:1030800002C00E94BB168EE587B90E942F150E94D0
:10309000181780914B0E833019F4A89510924B0E9F
:1030A0000E94D30D8C1B9D0B2091AB063091AC067A
:1030B0002817390720F49093AC068093AB06DF9174
:1030C000CF9108951F938FEF8ABB1BBA91E897BBEE
:1030D0009EE798BB9EE394BB91EC95BB11BA82BB73
:1030E00088E082B987EF83B9109261001092620084
:1030F00084E1809364008BEF809365000E94855D7E
:1031000080E487B985E886B987E083BF8CE981BF11
:1031100087B7836087BF1FBC8AE08EBD10928B008B
:1031200082E880938A0080917D00806280937D0098
:10313000EDB7FEB7329785E502C0808331979EE0F8
:10314000EA35F90709F0C8F7789484E79EE390938D
:1031500073048093720489E10E94BB5D0E94C25493
:10316000109155010E94BA11809156010E94BB5DD9
:103170005091700140917801451778F4652F70E007
:1031800024EF31E0629FC001639F900D729F900D0C
:1031900011249093840480938304541770F450E0B6
:1031A00024EF31E0429FC001439F900D529F900D4C
:1031B000112490938404809383040E94E0108091F2
:1031C0007701813039F480916E0184FD03C087E07E
:1031D0000E9460680E9449160E947B120E94BB16E2
:1031E0000E94CF160E9424110E946F120E9460124A
:1031F0000E94D91080EF90E090930A01809309011A
:103200000E9457642DE088E190E00FB6F894A895ED
:1032100081BD0FBE21BD89E095E060E00E9496343B
:1032200084E590E30E946A1481E00E943514809145
:1032300056010E94BB5D80915501181729F081E06D
:103240000E9409550E94A55580ED97E09BBD8ABD5F
:1032500080E186BF87B7806187BF0E943018FDCFAD
:103260008DE294E00E94E965089529E282029001CE
:103270001124359527953595279587FD815C86FB2B
:10328000880F880B80F9992787FD9095281B390BAB
:10329000C90108959C01E5E035952795EA95E1F788
:1032A000AC01440F452F441F550B280F391F892FA0
:1032B000990F990B8595280F391F241B350BC901D0
:1032C0000895F8942091B70D3091B80D7894C90104
:1032D0000895AC0180E060E021E00E94185B089551
:1032E0000F931F93CF93DF93182F83E198E00E94F1
:1032F0006919113658F0133628F0133639F48BE07B
:103300009AE102C084E79EE30E945A1486E068E0D6
:103310004BE058E00E94475B409123065091240601
:103320008AE268E020E000E00E941A0E4091250643
:10333000509126068EE468E020E00E941A0E86E096
:1033400060E143E058E00E94475B409127065091BE
:1033500028068AE260E120E00E941A0E40912906C8
:1033600050912A06F4E056954795FA95E1F78EE4D8
:1033700060E120E00E941A0E86E660E04FEF57E021
:103380000E94475B40912106509122068EE460E046
:1033900020E00E941A0E8091A7069091A806893716
:1033A000910528F08091A606C82FD0E002C0C0E0A9
:1033B000D0E082E06CE34EE70E94C55B85E06CE103
:1033C00043E20E94C95B1BE0812F6BE343E00E9454
:1033D000C95B1A5F1338C1F716E00CE3FE01E25D2A
:1033E000F94F4081602F641B812F0E94C95B219699
:1033F000C837D10510F0C0E0D0E02091A60630E03B
:10340000C217D30719F01F5F1E3741F7DF91CF9125
:103410001F910F9108951F93182F88E698E00E943E
:1034200069191236E1F0133628F4103631F01136EE
:10343000E9F418C01336D1F415C08FEF97E09093DC
:103440000D0180930C011092AA061092A906109209
:10345000AC061092AB0687E10E94606807C080E767
:1034600099E102C084E79EE30E945A1488E069E56E
:1034700078E00E943F5B4091A9065091AA065695BC
:10348000479584E568E00E946B5D80E16AE478E03E
:103490000E943F5B40910C0150910D01569547955C
:1034A00084E560E10E946B5D88E16BE378E00E9457
:1034B0003F5B4091A9065091AA0680910C01909122
:1034C0000D01481B590B5695479584E568E10E940C
:1034D0006B5D80E262E378E00E943F5B2091AB0687
:1034E0003091AC0684E690E0289FA001299F500D02
:1034F000389F500D1124A4E056954795AA95E1F701
:1035000084E560E220E30E945B5D88E26AE278E0A5
:103510000E943F5B0E942618AC018FE368E20E9484
:103520004B5B82E168E348E158E00E94475B1F91F2
:10353000089585E39FE008950F9393E0499FA001CC
:103540001124425D504F01E0222309F400E023E002
:103550000E94E85A0F9108950F9393E0499FA001AC
:103560001124495D504F01E0222309F400E023E0DB
:103570000E94E85A0F910895FF920F931F93F82E1F
:10358000062F142F80E860E0402F50E0212F0E948A
:103590005B5D0A3010F00FE601C005E7802F60E0A8
:1035A0004FE2212F0E94255A4F2D50E04F5F5F4F71
:1035B000802F60E0212F0E945B5D1F910F91FF9093
:1035C00008956F927F928F929F92AF92CF92DF92E7
:1035D000EF92FF920F931F93CF93DF93EC01162F7F
:1035E000D42E49016090DD047090DE048091A8081B
:1035F0009091A9088619970920E430E0B9010E944A
:10360000A668462F60930705E091DF04F091E0047F
:103610008091A6089091A7088E1B9F0BB9010E946C
:10362000A668862F60930805442321F07092A908AC
:103630006092A808882321F0F093A708E093A608D9
:1036400080910605882321F480916E0185FF06C0D4
:103650001092070510920805109206056091070563
:10366000662351F480910805882331F48091800409
:1036700090918104009781F04091700150E024EF17
:1036800031E0429FC001439F900D529F900D112445
:1036900090938404809383048114910409F456C0A8
:1036A0008881882309F04BC0662331F1809104059D
:1036B000882311F5ED2DE61BE7FDE0E0202F30E03B
:1036C0008E2F992787FD90958217930714F0E02F8E
:1036D000E150FF27E7FDF0958D2D90E0E817F90701
:1036E00049F0EE0FFF1FE80DF91D25913491C90136
:1036F0000E945A1410920705153641F4DD2011F08E
:10370000ED2D01C0E02FF0E031970FC01436C9F461
:103710002D2D30E0802F90E00197281739071CF4F9
:10372000ED2DEF5F01C0E0E0F0E0EE0FFF1FE80DD0
:10373000F91D25913491C9010E945A1402C040E03C
:1037400001C041E08D2D602F0E94BC1AE114F104EC
:1037500051F098818C2D9C1508F4892FF701E80F02
:10376000F11D549101C050E080910405882309F0B7
:103770004FC080910805882329F14881481B47FDE7
:1037800040E0242F332727FD30958A2D90E028171D
:1037900039070CF04A2D48838981E114F10459F06E
:1037A000C41608F44C2DF701E40FF11DE4918E17B7
:1037B00018F4E82F01C0E0E0E98380E68093B90DBA
:1037C000109208058881882319F1909107059923A3
:1037D000F9F04981E114F104B1F0491B47FD40E0E3
:1037E0009C2D8C1508F4982FF701E90FF11DE49139
:1037F000242F332727FD30958E2F90E02817390787
:103800001CF04E2F01C040E0498380E68093B90D43
:10381000103651F1113690F4133409F480C0143489
:1038200030F4113279F1123409F09CC06AC01434BA
:1038300009F43FC0153409F095C04FC01436E9F1C2
:10384000153638F4123609F45FC0133609F08AC011
:1038500069C01138A1F01F3B21F0153609F082C074
:1038600040C01982188212C0552309F47BC081E040
:1038700090910405911180E08093040573C010922B
:1038800004050DC080910405882319F010920405E9
:1038900069C08881882319F08114910421F480E0A3
:1038A0000E9435145FC087E10E9460681982188207
:1038B00056C08981851709F455C0E114F10409F453
:1038C00051C080910405882309F04CC08981851777
:1038D00010F48F5F12C0198242C08981882309F4D5
:1038E00041C0E114F10409F43DC08091040588232E
:1038F000C9F58981882319F08150898330C05983A3
:103900002EC088818A1571F180910405882351F5B4
:1039100088818A1510F48F5F0DC018820EC08881CF
:10392000882301F1809104058823E1F488818823AC
:1039300019F08150888301C0A8828981E114F104C3
:1039400061F098819C1508F4C92EEC0CF11CF7016C
:103950009491891718F4982F01C090E0998380E61C
:103960008093B90DDF91CF911F910F91FF90EF9050
:10397000DF90CF90AF909F908F907F906F90089541
:103980004F925F926F927F928F929F92AF92BF926F
:10399000CF92DF92EF92FF920F931F93DF93CF931B
:1039A0000F92CDB7DEB7D82E80E69AE00E94691953
:1039B0008EE298E06D2D41E02FED37E006E058E60D
:1039C000E52E5AE0F52E15E0C12EB6E0AB2E0E9492
:1039D000E11A80902E0890902F088091630081FF5B
:1039E00007C08AE268E14AE55AE00E94475B60C18D
:1039F00082E168E04BE45AE00E94475B8A94809140
:103A00000405882319F0A2E0CA2E02C0CC24C39476
:103A1000EE24FF2410E1A82CBB24A7FCB094F4E012
:103A20006F2E712C2701440C551C82E691E0480E44
:103A3000591E4E2D4F5F80E0612F20E00E949F0EA7
:103A4000AE14BF0411F491E0911090E0F2012181D5
:103A5000229526952695237030E0A901440F551F25
:103A6000420F531F4F5B554F992311F400E001C0E3
:103A70000C2D88E1612F23E099830E94E85A9981F7
:103A80009923C1F0809104058823A1F0F20161819E
:103A900062956695669563708D2D40E022E00E94E8
:103AA0001C148295880F880F807CF20191819F738E
:103AB000982B9183AE14BF0421F401E0F92DF1306D
:103AC00009F000E0F2018181880F880F85958595C6
:103AD000FDE08F02C0011124B3010E94A668AB0172
:103AE000002311F420E001C02C2D82E4612F0E94FC
:103AF0005B5D0023A9F080910405882389F0F20121
:103B00006181660F660F659565958D2D41EE2FE1FC
:103B10000E941C148F73F2019181907C982B9183E9
:103B2000AE14BF0421F491E0F92DF23009F090E0D9
:103B3000F2012081277030E0A901440F551F420F88
:103B4000531F4C5C554F992311F400E001C00C2D1C
:103B500088E4612F23E099830E94E85A9981992390
:103B600091F080910405882371F0F2016081677003
:103B70008D2D40E023E00E941C148770F20190819B
:103B8000987F982B9083AE14BF0421F401E0F92DA7
:103B9000F33009F000E0F2014081459545954595E7
:103BA000002311F420E001C02C2D8AE5612F0E9432
:103BB000EB0E0023B1F080910405882391F0F2010F
:103BC00060816595659565958D2D4AEE26E10E948B
:103BD0001C14880F880F880FF20190819770982B22
:103BE0009083185F0894E11CF11C103309F01ACF80
:103BF00080E369E27AE00E943F5B409172015527C1
:103C000047FD5095465F5F4FF82DF43011F421E2E7
:103C100001C020E28EE460E30E945B5D282D243029
:103C200049F48D2D6091720146EF28E20E941C1428
:103C300080937201EE24E394882D853009F0EE2400
:103C400080E068E345E25AE02E2D0E94185B4AE8C6
:103C5000A42E44E0B42E0AE511E090E3F501419171
:103C600051915F01F801219131918F01421B530B5A
:103C7000440F551F892F68E320E299830E945B5D02
:103C80009981985E903951F7EE2091F0FD2DF03634
:103C900079F4AAE5B1E0EAE8F4E088E001900D9259
:103CA0008150E1F781E00E94095587E10E94606838
:103CB0000F90CF91DF911F910F91FF90EF90DF90C8
:103CC000CF90BF90AF909F908F907F906F905F90BC
:103CD0004F900895AF92CF92EF92FF920F93AE2C38
:103CE000EE24FF24CC240E94E11A0F91FF90EF9064
:103CF000CF90AF900895EF920F93DF93CF930F92F1
:103D0000CDB7DEB7682F8EE69AE069830E94691905
:103D100080E398E0698142E02FED37E006E0EE2491
:103D20000E946A1E80E167E677E00E943F5B88E1BF
:103D300064E377E00E943F5B80E267E477E00E9403
:103D40003F5B88E268E577E00E943F5B80E367E7DE
:103D500077E00E943F5B0F90CF91DF910F91EF9042
:103D60000895CF92DF92EF92FF920F931F93DF930C
:103D7000CF9300D0CDB7DEB7682F8DE99AE0698385
:103D80000E94691982E398E0698143E02FED37E0F2
:103D900006E0EE240E946A1EEEE0CE2ED12C00E05A
:103DA00010E0143020F078EFF72EF00E01C0F02E66
:103DB000C6010E94C55EE82E1F5F8AE26F2D412F6B
:103DC00020E00E94EB0E4E2D405D84E46F2D2E2DE1
:103DD0000E94255A085F0894C11CD11C193009F7AC
:103DE00008E3CC24DD2410E0812F90E00E94C55E22
:103DF000F82EA6014258554F80E0602F25E00E9422
:103E0000125B4F2D405D80E2602F2F2D0E94255ABE
:103E10001F5F85E090E0C80ED91E0850163021F7CC
:103E200084E568E146E75AE027E00E94125B66E01D
:103E3000E62EF12C10E230E084E5612F44E857E0F3
:103E4000232F00E03A830E94C659C7010E94C55E35
:103E5000282FC701019629830E94C55E082F29815A
:103E6000422F405D8CE6612F0E94255A402F405D15
:103E700088E7612F202F0E94255A3A813F5F185F03
:103E8000E2E0F0E0EE0EFF1E3430B1F60F900F903E
:103E9000CF91DF911F910F91FF90EF90DF90CF9026
:103EA00008958F929F92AF92BF92DF92EF92FF920E
:103EB0000F931F93CF93DF93D82E85EA9AE00E9449
:103EC000691984E398E06D2D44E02FED37E006E0BA
:103ED000EE24E3940E946A1EF0903408C5EDD4E00D
:103EE00010E000E0812CF4E09F2EA12CB12C88E1A1
:103EF000612F41E40E94E45A402F4F5C8EE1612F14
:103F00000E94E45A802F0E94FC14AC018AE2612FC7
:103F10000E944B5B0730B1F068817981882777FD7B
:103F20008095982F24E630E040E050E00E946768DA
:103F3000A50194010E94DB688AE5612FA9010E9416
:103F40006B5D0AC08F2D813011F040E201C041E26B
:103F50008AE5612F0E94990E0F5F185F2296083044
:103F600031F68CE668E242EA5AE022E00E94125BF7
:103F70004091090150910A0188E760E320E00E9426
:103F80005B5D8F2D813059F4F09206058D2D609187
:103F9000580141E82FE70E941C1480935801DF91DB
:103FA000CF911F910F91FF90EF90DF90BF90AF9056
:103FB0009F908F900895EF920F93E42E40E020E0C1
:103FC00030E000E00E946A1E0F91EF900895AF92DA
:103FD000BF92CF92DF92EF92FF920F931F93DF93E6
:103FE000CF9300D0CDB7DEB78FE161E247E10E9409
:103FF000C95B8FE167E347E10E94C55B85E361E24E
:1040000047E10E94C95B8FE161E247E10E94C55B25
:104010008BE461E247E10E94C95B8BE467E347E11F
:104020000E94C55B81E661E247E10E94C95B8BE4C7
:1040300061E247E10E94C55B8AE26BE243E00E94D5
:10404000C95B89E26CE243E00E94C55B86E56BE2F6
:1040500043E00E94C95B85E56CE243E00E94C55BDA
:104060008091D5049091D60451E7C52ED12CB6018C
:104070000E94A668262F8091D7049091D8040FE85B
:104080001FEFB8010E94A668362F48E2E42EE20E28
:104090009AE2F92EF60E8E2D6F2D45E02A83398394
:1040A0000E94C95B3981632F625D8E2D45E00E94BD
:1040B000C55B2A81822F845D6F2D45E00E94C95B1C
:1040C0008E2D6F2D45E00E94C55B8091DB049091A1
:1040D000DC04B6010E94A668262F8091D904909135
:1040E000DA04B8010E94A668062F84E5F82EF20EC5
:1040F000162F165D8F2D612F45E02A830E94C95B24
:10410000602F625D8F2D45E00E94C55B2A81822F62
:10411000885A612F45E00E94C95B8F2D612F45E0D1
:104120000E94C55B1DEDA12E14E0B12EBAE3FB2E5B
:104130000DE510E0A8E3EA2EF501819191915F0170
:1041400080509C4FB8010E94A668D62ED394CE2CE6
:10415000CD188F2D6C2D4D2D0E94C95B8F2D8F5F3B
:104160006C2D4D2D0E94C95B8F2D8E5F6C2D4D2DBA
:104170000E94C95BF5E0FF0E8F2D8934E9F60F90A0
:104180000F90CF91DF911F910F91FF90EF90DF90F3
:10419000CF90BF90AF9008954F925F926F927F92B1
:1041A0008F929F92AF92BF92CF92DF92EF92FF9247
:1041B0000F931F93DF93CF930F92CDB7DEB7B82E37
:1041C0008AEF9AE00E94691981E698E06B2D45E03C
:1041D0002FED37E006E0EE24E3940E946A1E109271
:1041E000610815E4E12E18E0F12EB7E3CB2EB8E01C
:1041F000DB2E8601470160E0862F69830E94FC1454
:10420000D4014D915C911197282F392F6981421764
:1042100053070CF49A01F401219331934F01D80113
:104220004D915C911197282F392F241735070CF4E5
:104230009A01F801219331938F016F5F6730E1F6A6
:104240008091360880930605FB2DF03219F0FF3B74
:1042500071F40BC08F5F80933608833041F487E19F
:104260000E94606881E00E94095510923608809192
:1042700036088130B1F0813020F0823009F0A4C0DE
:104280003FC08CE060E148EE5AE021E100E00E948E
:10429000E85A82E168E148ED5AE02FE00E94E85ACE
:1042A00093C08EE160E14BEC5AE02CE000E00E940C
:1042B000E85A82E168E149EA5AE020E10E94E85ABE
:1042C000A3E58A2EA8E09A2E20E008E91AE3F8E692
:1042D000AF2EF5ECBF2ED7010D931D937D01F60196
:1042E000A192B1926F01822F29830E94FC14D40104
:1042F0008D939D934D0129812F5F273061F764C015
:1043000082E160E14AEB5AE020E100E00E94E85AD5
:1043100082E168E149EA5AE020E10E94E85AE3E5D7
:10432000AE2EE8E0BE2E79E2472E71E0572EF20164
:1043300060E4862E912CD7018D919D917D01D6014F
:104340006D907D906D019C012619370937FF03C0E0
:10435000309521953F4F23333105DCF0D5012D9168
:104360003C91318320838901081B190BC801B401DA
:104370000E94A668061B170B17870687C301821BBE
:10438000930B9C01B4010E94A668261B370B358F46
:10439000248FA2E0B0E0AA0EBB1E3296B3E5EB1666
:1043A000B8E0FB0641F680E090E0F2012191319106
:1043B0002F01820F931FF1E44F16F1E05F06A9F77A
:1043C00090935401809353010E94E71F0F90CF9167
:1043D000DF911F910F91FF90EF90DF90CF90BF90F2
:1043E000AF909F908F907F906F905F904F900895C7
:1043F000282F30E0C901880F991FA90163E0440FFD
:10440000551F6A95E1F7840F951FA9014F5F5F4F14
:10441000BA01660F771FA3E0440F551FAA95E1F775
:10442000640F751F6E557E4F20953095205E3F4F6F
:10443000A901440F551FE3E0220F331FEA95E1F76E
:10444000420F531F8E559E4F0E940B698AE0E8ED84
:10445000F2E0DF011D928A95E9F782E00E9409559A
:104460000E94A55508950F931F93CF93DF93282F94
:1044700030E0E901CC0FDD1FC90113E0880F991F5F
:104480001A95E1F7C80FD91F8E010E551E4FA901CD
:104490004F5F5F4FCA01880F991FA3E0440F551F5C
:1044A000AA95E1F7840F951F20953095205E3F4F28
:1044B000A901440F551FE3E0220F331FEA95E1F7EE
:1044C000420F531F8E559E4FB8010E940B698AE020
:1044D000D8011D928A95E9F780918308C857DE4F6D
:1044E0008A8F8B8F84E68C8F82E00E9409550E9410
:1044F000A555DF91CF911F910F910895FF920F93D2
:104500001F9385EFE9E2F5E0DF011D928A95E9F757
:1045100080911E06A2EAB1E050E021E030E060E0C8
:104520007C91772311F0472F01C040E1641738F5E3
:10453000F22E032F162F1F5F802F90E0FC01EE0F4D
:10454000FF1FEE0FFF1FE80FF91FE75DFA4F912FD6
:104550009F738081807C892B80648083F182F394B7
:1045600053830F5F141738F3962F9095642F822F83
:104570008F5F890F390F340F290F240F840F772392
:1045800059F1832F90E0FC01EE0FFF1FEE0FFF1F8C
:10459000E80FF91FE75DFA4F4F738081807C5483E9
:1045A000842B8068808322832F5F1A968C911A97C0
:1045B000781719F41182138205C021832F5F852F8C
:1045C0008F5F8383822F5F5F1A96503219F4209396
:1045D0001E0604C03F5FA4CF80931E061F910F915B
:1045E000FF900895E2EAF1E080E0908191509031EF
:1045F00008F48F5F3A9692E0E23EF907B1F708952A
:104600001F93182F80E162E77DE00E943F5B0E94CC
:10461000F222482F88E760E150E020E00E945B5DD5
:1046200080E26CE57DE00E943F5B113651F481E64B
:104630000E94245F81E00E94351480EC93E20E9486
:104640006A141F9108950E94F222803230F080E0B7
:1046500093E20E946A1481E0089580E00895EF9249
:10466000FF920F931F93DF93CF9300D0CDB7DEB7A8
:10467000182F813208F07BC0882319F4442341F4B9
:1046800076C0803219F4442331F071C0442319F00C
:10469000012F0F5F02C0012F0150812F4A836983D0
:1046A0000E94FE0D7C01802F0E94FE0DFC01D701AF
:1046B0008C91982F91504A816981903108F057C0B0
:1046C0002081213108F053C06623A1F10E942323E9
:1046D000882309F04CC0212F30E0A9014F5F5F4FC4
:1046E000CA01880F991F13E0440F551F1A95E1F76F
:1046F000840F951FB901660F771FA901A3E0440F2E
:10470000551FAA95E1F7640F751F6E557E4F2095D2
:104710003095205E3F4FA901440F551FE3E0220F63
:10472000331FEA95E1F7420F531F8E559E4F0E94AB
:104730000B691DC0281759F0442331F08031B8F4BB
:104740008F5FF701808313C0D7019C9310C0D701FE
:10475000CF010A9604C020813C9131932D93E81734
:10476000F907C9F782E00E9409550E94A5550F90EC
:104770000F90CF91DF911F910F91FF90EF900895CF
:104780006F927F928F929F92AF92BF92CF92DF9261
:10479000EF92FF920F931F93CF93DF93182F86E52D
:1047A0009DE00E946919E0901E06EA9486E898E070
:1047B000612F43E02FEC37E008E00E946A1EC090B2
:1047C0008608CC2011F4109285081236D9F11336E0
:1047D00070F41334A9F1143420F4123409F070C0C9
:1047E00031C01036C1F0113609F06AC045C010382A
:1047F00009F452C0113820F4133609F061C020C00A
:104800001E3BB9F11F3B09F05BC081E08093840837
:10481000109285082EC01C143CF481E0909185080C
:10482000911180E0809385088091850880938408A9
:1048300080918108882309F443C01092850840C004
:1048400010928408809185088823D1F141E01236C6
:1048500009F040E080918208609184080E942F2333
:1048600080918408882319F0133609F4CA941092B1
:1048700084080E947E2224C080918508882301F14B
:10488000809182080E94F821109285080E947E2261
:1048900081E60E94245F14C01C1494F48091810866
:1048A000882341F00E942323882321F480918208E9
:1048B0000E943322109285088FE79FE40E946A14B9
:1048C00038E0D32E77247A9423E6822E9924BB24D1
:1048D000BA9466246394E0900305E90CFF24F70181
:1048E000EE0FFF1FEE0FFF1FEE0DFF1DE75DFA4FEE
:1048F0004081842F807C09F462C146FF06C04F735B
:1049000080E06D2D20E00E94CB0E1C14E4F4E70142
:10491000CC0FDD1FCC0FDD1FCE0DDF1DC75DDA4FC5
:104920008981C81681F46D2D695F80E048E10E949D
:10493000C55B8B818093820888818F738093830805
:1049400060928108B92CF701EE0FFF1FEE0FFF1FD9
:10495000EE0DFF1DE75DFA4F808187FF05C1948151
:10496000C92FDD27C7FDD095AA24A3949281C9122F
:10497000AA2486FD1FC0FE01EE0FFF1FCE01A3E09B
:10498000880F991FAA95E1F7E80FF91FE755FE4F29
:1049900040814695477050E04E5A524F80918508AD
:1049A000882311F400E001C00A2D82E16D2D21E081
:1049B0000E94E85AFE01EE0FFF1FCE0163E0880F50
:1049C000991F6A95E1F7E80FF91FE857FE4F448DEC
:1049D000552747FD50958DE26D2D2A2D0E945B5D78
:1049E00080918508882311F420E001C02A2D8DE2F2
:1049F0006D2D45E20E94255AFE01EE0FFF1FCE01EC
:104A000043E0880F991F4A95E1F7E80FF91FE8572F
:104A1000FE4F438D80918508882311F420E001C06A
:104A20002A2D86E36D2D0E949F0EFE01EE0FFF1FC3
:104A3000CE0123E0880F991F2A95E1F7E80FF91FAF
:104A4000E857FE4F458D442359F08091850888230F
:104A500011F420E001C02A2D8EE46D2D0E94EB0E92
:104A6000FE01EE0FFF1FCE01B3E0880F991FBA952C
:104A7000E1F7E80FF91FE857FE4F468D442391F008
:104A800023E0429FA00111244B5C504F8091850888
:104A9000882311F400E001C00A2D86E66D2D23E085
:104AA0000E94E85AFE01EE0FFF1FCE0173E0880F4F
:104AB000991F7A95E1F7E80FF91FEE55FE4F21E0B7
:104AC0008581882309F420E0FE01EE0FFF1FCE014F
:104AD00053E0880F991F5A95E1F7E80FF91FEE553B
:104AE000FE4F8681882329F0222309F498C04AE2E8
:104AF00003C0222361F044E480910405882311F46B
:104B000020E001C02A2D89E76D2D0E94255A8A2DAB
:104B1000813051F55E01AA0CBB1C33E0CC0FDD1FC8
:104B20003A95E1F7AC0EBD1EE8E8F1E0AE0EBF1E0F
:104B3000812FF501648D43E82DE70E940D14F501E6
:104B4000848FF701EE0FFF1FEE0FFF1FEE0DFF1D0D
:104B5000E75DFA4F84818093820880818F73809310
:104B6000830810928108B92CF701EE0FFF1FEE0F9A
:104B7000FF1FEE0DFF1DE75DFA4F8181882331F0A5
:104B800088150CF4882E87150CF0782EF701EE0F9F
:104B9000FF1FEE0FFF1FEE0DFF1DE75DFA4F828135
:104BA000882331F088150CF4882E87150CF0782EA8
:104BB0009394F8E0DF0E292D273009F08CCECC201D
:104BC000A1F08B2D8F3FF9F4C81464F48091030594
:104BD00090E00197EFEF8F3F9E0711F480E090E0A7
:104BE000809303057C14ECF414C0FB2DFF3F59F4B3
:104BF0008091030590E001972FEF8F3F920761F4BA
:104C000080E090E009C08B2D86305CF0992D9830C3
:104C100040F0809103058F5F8093030502C043E558
:104C20006BCFDF91CF911F910F91FF90EF90DF90AD
:104C3000CF90BF90AF909F908F907F906F9008958E
:104C40002F923F924F925F926F927F928F929F929C
:104C5000AF92BF92CF92DF92EF92FF920F931F938A
:104C60005C01CC24DD243B018824992464E6262EB3
:104C7000312C412C512CC201B101661977098809E8
:104C80009909A60195010E9467687B018C0182E366
:104C900090E0A0E0B0E0E80EF91E0A1F1B1FC6015D
:104CA000B5010E9467680E946768BC018827992740
:104CB000A40193010E94676844E0969587957795D3
:104CC00067954A95D1F7E60EF71E081F191FC80110
:104CD000B701A20191010E94B968C9011F910F910A
:104CE000FF90EF90DF90CF90BF90AF909F908F900C
:104CF0007F906F905F904F903F902F9008951F93FB
:104D0000CF93DF939C016115710511F1132F111FD2
:104D10001127111F19F0309521953F4F77FF0EC0D5
:104D2000C0E0D4E0709561957F4FCE01821B930B5C
:104D30000E9420269E01281B390B05C0C9010E9434
:104D40002026282F392F112319F0309521953F4F18
:104D5000C901DF91CF911F9108956F927F928F9239
:104D60009F92AF92BF92CF92DF92EF92FF920F93FA
:104D70001F93DF93CF93CDB7DEB7982E962F322FA8
:104D8000802F6E2D222359F0442361F4409180043A
:104D9000509181044115510539F421E001C020E012
:104DA000FF2405C022E001C021E0FF24F394332357
:104DB00011F0911121E04A2D433679F44C2D50E049
:104DC000440F551F8A0173E0000F111F7A95E1F718
:104DD000041B150B025C1C4F11C0FA2DF236D9F4DE
:104DE0004C2D50E0440F551F8A0193E0000F111F16
:104DF0009A95E1F7041B150B015C1C4FF8014081EB
:104E00000E94EB0EFF2009F463C0F8016081892D38
:104E10004AEE26E159C069887724BB24882051F5E1
:104E20004C2D50E0440F551F6A01B3E0CC0CDD1C43
:104E3000BA95E1F7C41AD50AAA0CBB1CAA0CBB1C74
:104E4000CA0CDB1CC60CD71C42E353E0C40ED51EB3
:104E5000F6014081552747FD50950E945B5DFF207C
:104E6000B9F1F6016081892D4CE924E60E940D1408
:104E7000F6012DC0DD24AA0CBB1CA601E3E0440F03
:104E8000551FEA95E1F74C195D09A40EB51EA80C53
:104E9000B11CAA0CBB1CF301EA0DFB1DEE5CFC4F20
:104EA0004081552747FD50954C595F4F0E945B5DEF
:104EB000FF2071F08501060D171D0E5C1C4F892D1A
:104EC000F80160814CE920E00E940D14F801808314
:104ED000CF91DF911F910F91FF90EF90DF90CF90D6
:104EE000BF90AF909F908F907F906F9008952F927A
:104EF0003F924F925F926F927F928F929F92AF926A
:104F0000BF92CF92DF92EF92FF920F931F93DF93A6
:104F1000CF93CDB7DEB72A970FB6F894DEBF0FBE9A
:104F2000CDBFD82E89E49DE00E9469198FE798E0F3
:104F30006D2D40E020E030E000E071E5E72E7DE0FF
:104F4000F72ECC2453E0A52E0E94E11A4091770859
:104F50004F5F80E360E020E00E949F0EF0907F08AA
:104F60008091770890E0880F991FFC0123E0EE0FF5
:104F7000FF1F2A95E1F7E81BF90BE25CFC4F8081EB
:104F800060E040E00E94C90F8823C1F0809177085B
:104F900090E0880F991FFC0113E0EE0FFF1F1A9598
:104FA000E1F7E81BF90BE15CFC4F808160E040E039
:104FB0000E94C90F882321F411E003C010E001C052
:104FC00012E060917708462F50E0FA01EE0FFF1FC4
:104FD000EB52FB4F808191818A3191051CF0109238
:104FE0007E0807C02FEF873E92071CF481E0809374
:104FF0007E0820916C0130E02170307082E090E0FA
:10500000821B930B8417950741F4643030F4809130
:105010009901807F11F010927E0880E164E47DE0C8
:105020000E943F5B0F92EDB7FEB7319621E0F11081
:1050300020E080917E0880838D2D61E041E006E3D1
:10504000A0E1EA2EC0907708A12E88240E94AD2608
:105050000F9088E16DE37DE00E943F5B0F92EDB71A
:10506000FEB7319621E03F2D313009F020E08091EC
:105070007E0880838D2D61E041E006E3F8E1EF2EAC
:10508000C0907708A12E882483940E94AD260F90AB
:1050900080E267E37DE00E943F5B0F92EDB7FEB7D1
:1050A000319621E08F2D823009F020E010828D2D85
:1050B00061E041E00EE1E0E2EE2EC090770873E699
:1050C000A72E88240E94AD260F9088E261E37DE040
:1050D0000E943F5B0F92EDB7FEB7319621E09F2D06
:1050E000933009F020E010828D2D61E041E00EE167
:1050F00058E2E52EC090770832E6A32E88240E945D
:10510000AD260F90113019F0123049F404C080E33D
:105110006AE27DE007C080E363E27DE003C080E3F4
:105120006BE17DE00E943F5B00917708402F50E0EB
:10513000812F90E0880F991F880F991FBA01660F81
:10514000771F9B01B3E0220F331FBA95E1F7261BAF
:10515000370B820F931F88579E4FFC01E655FE4F79
:10516000A081A983FC01E555FE4FB081BA83FC0103
:10517000E455FE4F9080E4E69E0E83559E4FDC0181
:105180008C908E0E20916C0130E02170307082E0A6
:1051900090E0821B930B8417950709F062C00430DE
:1051A00008F05FC080919901807F09F45AC0EE2415
:1051B000FF24870120E030E0B9816B2E772467FC63
:1051C0007094A1E24A2E512C292C332427FC3094D0
:1051D000F0E4CF2ED22ED801C701B595A7959795AB
:1051E0008795B30129873A870E947F26880F991FE8
:1051F000B2010E94A668629DC001639D900D729DE0
:10520000900D11246FE3A62EAD0C64E670E00E94B1
:105210009268EC2DE61B6E2F8A2D0E94795B298502
:105220003A85C90183709070009761F48A2D6FE30D
:105230000E94795B6D2D6695605E8FE30E94795BBD
:105240003A8529852F5F3F4F81E290E0A0E0B0E0F2
:10525000E80EF91E0A1F1B1F2E33310509F0BACFC5
:105260007CC0DD249981492E552447FC509401E2ED
:1052700010E0A92DBB27A7FDB095BC83AB8354E6F6
:10528000652E712C40E2A42EBA812B2E332427FCEC
:105290003094E82DFF27E7FDF095FE83ED83FD2D8B
:1052A00021E2F29F70011124C701B2010E947F2602
:1052B000B8010E94A668AB81BC816A9FC0016B9F48
:1052C000900D7A9F900D11243EE5C32ECD0CB301B5
:1052D0000E949268BA2DB61B6B2F8C2D0E94795BB1
:1052E000ED2DF0E0E370F070F887EF83309749F42C
:1052F0008C2D60E20E94795B6D2D605E8EE50E94D0
:10530000795BC701B1010E947F26B8010E94A6689F
:105310002D813E81629FC001639F900D729F900D11
:1053200011242EE5F22EFD18B3010E949268605EF2
:105330008F2D0E94795B8F819885009749F48F2D7E
:1053400060E20E94795B6A2D6D198EE50E94795B9F
:10535000D3949D2D9F3109F0A2CFE0917708F0E022
:10536000EE0FFF1FEB52FB4F408051805201CC24C7
:10537000B7FCC094DC2CC601B50121E230E040E06E
:1053800050E00E94DB68822F825A61E04EE30E9467
:10539000C95B4091770820916C0130E0217030703A
:1053A00082E090E0821B930B242F30E0821793075A
:1053B00009F050C0443008F04DC080919901807FC1
:1053C00009F448C0C601B50160507C4F8F4F9F4F14
:1053D00022E030E040E050E00E94DB68A9816A2FC3
:1053E000772767FD7095C9010E947F26BC01660F73
:1053F000771F882777FD8095982F292D97FC2D5FA3
:1054000025952595332727FD3095432F532F0E944F
:10541000676829E130E040E050E00E94DB687901F4
:105420008A01CA01B9012FED3FEF4FEF5FEF0E94F4
:10543000DB68622F605C8FE34EE30E94C55BC801AE
:10544000B70122E030E040E050E00E94DB687901E3
:105450008A013CC01A141B041C041D0414F4698145
:1054600001C06A81772767FD7095C2010E947F267F
:105470009C01442737FD4095542F1A141B041C042B
:105480001D0414F4692D01C0682D67FD6D5F6595DD
:105490006595772767FD7095872F972F0E9467681E
:1054A00029E130E040E050E00E94DB6879018A01A8
:1054B000CA01B9012FED3FEF4FEF5FEF0E94DB68AC
:1054C000622F605E8FE34EE30E94C55BC601B501AB
:1054D00029E130E040E050E00E946768612CB1E0D3
:1054E0007B2E812C912CA40193010E94DB6882E722
:1054F00060E3A90120E00E945B5DC801B70129E1DA
:1055000030E040E050E00E946768A40193010E94EF
:10551000DB6884E568E0A90120E00E945B5D1A1465
:105520001B041C041D0474F4B9816B2F772767FDDD
:105530007095C20144970E947F26F701E81BF90B82
:10554000CF010BC0FA816F2F772767FD7095C201DD
:1055500044960E947F268E199F099C01220F331FBB
:10556000220F331F280F391F442737FD4095542F32
:1055700084E560E100E3F3E0EF2E0E94255C2A96CB
:105580000FB6F894DEBF0FBECDBFCF91DF911F9154
:105590000F91FF90EF90DF90CF90BF90AF909F90D2
:1055A0008F907F906F905F904F903F902F900895D5
:1055B0002F923F924F925F926F927F928F929F9223
:1055C000AF92BF92CF92DF92EF92FF920F931F9311
:1055D000DF93CF93CDB7DEB72F970FB6F894DEBF2A
:1055E0000FBECDBF982E81E19DE00E9469198CE726
:1055F00098E0692D42E02FEC37E008E0F9E1EF2E6A
:10560000FDE0FF2ECC24C394E4E0AE2E0E94E11A0C
:10561000F0907C08FA9430907D08292D203841F4D0
:10562000F7FC06C0F092770887E797E20E946A14B9
:1056300085E168E041E05DE00E94475B8EE393E036
:105640009C838B8378E7472E78E0572EE5EDF4E0D6
:10565000FB87EA8710E1662477242F2D332727FD67
:1056600030953A832983C901880F991FFC0153E0C3
:10567000EE0FFF1F5A95E1F7E81BF90BFE83ED8350
:10568000F62CEB81FC81808160E040E00E94C90F34
:10569000882361F0EB81FC81818160E040E00E9421
:1056A000C90F882329F4BB24B39404C0BB2402C0CF
:1056B00042E0B42E2B2D30E038872F83C901880FAC
:1056C000991F880F991FA301440F551F9A0103E0EA
:1056D000220F331F0A95E1F7241B350B820F931F0E
:1056E00088579E4FDC01A355BE4FFC01E455FE4F89
:1056F0003C912081321751F4FC01E555FE4F86554F
:105700009E4F41E02081FC018081281340E0EA8522
:10571000FB8581919191FB87EA879C0197FF04C0EB
:1057200022273327281B390B2A3131050CF040E0A2
:10573000242E8A3191051CF0F201108207C0FFEF80
:10574000873E9F071CF421E0F201208380916C01C9
:1057500090E081709070E2E0F0E0E81BF90BE61554
:10576000F70551F480919901807F31F0F301E858F9
:10577000F74F1082222423944F2D4F5F80E0612F3A
:1057800020E00E949F0E5D864C86F2013081F1E0A0
:10579000F9873111198680910405882351F4DD249D
:1057A000D3948091800490918104009721F4DD24AA
:1057B00002C0DD24D39489819A818615970511F45E
:1057C00021E0311020E00F92EDB7FEB73183892D33
:1057D00060E04D2D07E2E12ECF2CAB2C88240E94F7
:1057E000AD260F9029813A812615370509F0D2C0E0
:1057F000332009F0CBC0DD2009F4CCC0222009F40D
:10580000C9C08F819885880F991F880F991FED81D6
:10581000FE818E0F9F1F88579E4FF9858F0F911D18
:1058200086559E4F9F878E87892DEE85FF856081E7
:105830004CE924E60E940D14EE85FF858083AAC002
:1058400021E00F92F2018081EDB7FEB78183892DAF
:1058500060E04D2D09E3E12ECF2CAB2C88248394FE
:105860000E94AD260F9029813A812615370509F04F
:1058700097C0332D313009F08FC0DD2009F490C07E
:10588000222009F48DC08F819885880F991F880F79
:10589000991FED81FE818E0F9F1F88579E4FF985BE
:1058A0008F0F911D84559E4F98878F83892DEF818F
:1058B000F88560814CE920E00E940D14EF81F885A5
:1058C00080836EC021E00F92EDB7FEB71182892D63
:1058D00060E04D2D0FE3E12ECF2CF3E6AF2E8824B0
:1058E0000E94AD260F9029813A812615370521F4B3
:1058F00021E0332D333009F020E00F92EDB7FEB7F1
:105900001182892D60E04D2D07E5E12ECF2CE2E6D6
:10591000AE2E88240E94AD260894411C511C0F9085
:10592000EC85FD858081882319F4222031F008C0A0
:10593000222031F48AE34FE705C08BE34EE702C033
:105940008AE34DE2612F0E94E45AFB2DF13019F0F9
:10595000F23049F404C085E7612F4DE407C085E7C4
:10596000612F4CE403C085E7612F48E40E94E45AAC
:105970000894611C711C2B813C81225F3F4F3C834A
:105980002B83185F103309F07BCE0CC0332D3130E0
:1059900009F456CF20E055CF832D823009F492CF01
:1059A00020E091CF2F960FB6F894DEBF0FBECDBF8B
:1059B000CF91DF911F910F91FF90EF90DF90CF90EB
:1059C000BF90AF909F908F907F906F905F904F901F
:1059D0003F902F90089520E030E0F901E254F34F1A
:1059E000E491E81711F4822F08952F5F3F4FEE23C3
:1059F000A1F780E00895823430F4E82FF0E0E2541B
:105A0000F34F8491089580E20895EF92FF920F93EF
:105A10001F93182FF62EE22E862FBA010E943F5BAD
:105A200086E66F2D412F2E2D0E949C1AEE2039F014
:105A3000802F612F40E021E00E941C14182F812F3D
:105A40001F910F91FF90EF900895FF920F931F9376
:105A5000F82E10919301212F332727FD309537FF22
:105A600003C0309521953F4F022F25320CF43DC0E5
:105A700020912808309129088091260890912708C4
:105A8000282B392B80912A0890912B08282B392B11
:105A90008091250890E0282B392B4091220850E076
:105AA000242B352B2115310531F4812F881F8827B0
:105AB000881F8093220811161CF4812F845202C083
:105AC000812F8C5D60E040E00E94C90F882359F06F
:105AD00090912208992339F491E020912508211111
:105AE00090E0909325088093220820912808309117
:105AF00029082F5F3F4F30932908209328082091D1
:105B00002608309127082F0D311D30932708209348
:105B100026080E94F60D20912A0830912B08821B3E
:105B2000930B8436910508F471C12C593F4F309383
:105B30002B0820932A082091260830912708E0910D
:105B40002808F0912908C901BF010E949268F62E29
:105B5000462F50E04E9FC0014F9F900D5E9F900DCD
:105B60001124281B390B3093270820932608109204
:105B700029081092280800311CF4109225080FC043
:105B800005326CF411161CF4812F8F5002C0812F46
:105B9000815F60E040E00E94C90F809325088091FA
:105BA0002106909122060196909322068093210669
:105BB00040912306509124064F5F5F4F5093240677
:105BC00040932306FF2049F08091270690912806F4
:105BD00001969093280680932706809125088823B4
:105BE00049F080912506909126060196909326060D
:105BF00080932506F6942091290630912A062F0DD0
:105C0000311D30932A0620932906809195019091A9
:105C1000960190932D0680932C066091930177272F
:105C200067FD709577FF03C0709561957F4F662380
:105C300019F410922B061EC0613019F4841B950BC9
:105C400015C0603168F460FF06C0A4E03695279562
:105C5000AA95E1F709C0209127063091280604C0D3
:105C60002091250630912606821B930B90932D06DA
:105C700080932C0680912B06813051F0813018F0F2
:105C8000823049F514C080919301882321F120C00E
:105C900080912C0690912D0618161906E4F080913B
:105CA0009501909196010097B1F082E012C0809129
:105CB0002C0690912D062FEF853C92071CF483E073
:105CC00080932B068091950190919601009719F48D
:105CD00081E080932B0680912C0690912D062091D7
:105CE0002308309124082817390709F479C0209136
:105CF0002B06213009F065C020916E0122FF45C0BE
:105D0000209195013091960121153105F1F18E31E7
:105D1000910519F489E10E94606880912C069091A8
:105D20002D068431910519F48AE10E946068809102
:105D30002C0690912D068A30910519F48BE10E9472
:105D4000606880912C0690912D06843091051CF49A
:105D50008CE10E94606880916E0183FF16C0809183
:105D60002C0690912D068E31910549F084319105D4
:105D700031F08A30910519F08430910534F482E3D2
:105D800090E0909384048093830480916E0181FF5E
:105D900027C08091940120912C0630912D0680FF20
:105DA00007C08091950190919601821B930B01C0D1
:105DB000C9016CE370E00E949268009789F480E06A
:105DC00003C0223069F48CE10E94606880916E010A
:105DD00083FF06C082E390E0909384048093830461
:105DE00020912C0630912D0630932408209323080F
:105DF0008091940180FF0AC0809195019091960155
:105E0000821B930B90932D0680932C061F910F916C
:105E1000FF90089580919301992787FD909597FFB2
:105E200003C0909581959F4F982F823034F1803137
:105E300024F585959A3024F40E94EE5F90E003C02B
:105E4000992787FD90950197FC01EE0FFF1FEB52FC
:105E5000FB4F208131818091930187FF05C080E055
:105E600094E0821B930B03C0C90180509C4F26E035
:105E7000969587952A95E1F702C080E090E00E9410
:105E8000252D83E00E94EE5FE82FF0E0EE0FFF1F6C
:105E9000ED52FB4F8081918180509C4FB6E09695EA
:105EA0008795BA95E1F72091940122FF0AC08530C9
:105EB000910538F020918604222319F423E02093E1
:105EC000860420911E0830911F082F5F3F4F3093AA
:105ED0001F0820931E0820911C0830911D08280FD0
:105EE000391F30931D0820931C080E94F60D209145
:105EF000200830912108821B930B23E0883E9207F3
:105F0000E8F10E94F60D909321088093200880917B
:105F10009701823051F485E160E040E00E94C90FB2
:105F2000882319F087E00E94606880911C08909196
:105F30001D0860911E0870911F080E9492681092BF
:105F40001D0810921C0810921F0810921E088091C4
:105F5000A7069091A80601969093A8068093A7069D
:105F60008091A606E82FF0E0E25DF94F60838F5F35
:105F70008093A606883710F01092A6060895109216
:105F80002B061092240610922306109228061092D7
:105F90002706109226061092250610922A061092C5
:105FA000290608950F931F93182F80911F068823A9
:105FB00019F06EEA7CE002C061EA7CE088E00E94B1
:105FC0003F5B81E060E148E851E02AE000E10E94A7
:105FD000E85A82E460E14FE30E94E45A82E168E219
:105FE0004AE95CE00E94475B82E160E34BE85CE0E9
:105FF0000E94475B113609F44AC01F3B21F010365E
:1060000009F04FC004C080E00E9460684AC08091DF
:106010001F068823A9F089E79CE00E94FF11809168
:1060200020060E947154882339F087E10E9460683D
:1060300082E080931F0629C080E00E94606825C02E
:10604000809155018F5F0E9435571091550108C00E
:106050001150113108F01FE080915501181739F0E7
:10606000812F8F5F0E94E856882391F301C010E0D2
:106070001093550181E00E9409550E94A555809119
:1060800055010E943A540E94BF2F80E601C081E66C
:106090000E94245F81E00E94351484E590E30E9411
:1060A0006A141F910F910895AF92BF92DF92EF9201
:1060B000FF920F931F93CF93DF93182F8BE09BE0FA
:1060C0000E946919809104058823A1F4E0910705D5
:1060D000E7FF10C0E195E83008F0E7E0F0E0EE0FF0
:1060E000FF1FE153F84F25913491C9010E945A14C2
:1060F00010920705F090730883E798E0612F4FE056
:106100000E94DB1F86E360E046E05BE00E94475BA5
:106110000E942A56AC0186E660E020E00E945B5DAA
:1061200080E068E041E00E94BC1AD0907308809142
:106130001F06823021F41092720810921F06163644
:1061400048F4143690F5103609F456C0113609F0AB
:1061500075C00AC0113809F456C01F3B09F465C068
:10616000103809F06BC053C0809172088823E9F0A1
:106170001092720887E10E94606881E60E94245FA5
:106180000E94A55580917308809355010E943A544E
:106190000E94BF2F81E00E9409550E94A55582E010
:1061A0000E9409550E94A55549C0809155018D1541
:1061B000B9F0812F0E94245F80917308809355016C
:1061C0000E94A555809155010E943A540E94BF2F0C
:1061D00081E00E9409550E94A55581E00E946068F7
:1061E000153619F48FE398E404C0143639F581E7C5
:1061F00091E40E945A1422C081E08093720887E1E2
:106200000E9460681BC081E00E94351417C0809115
:106210007208882399F081E080931F06D0922006AF
:1062200082ED9FE20E946A1409C010927208809168
:1062300055018093730881E00E9417558091720880
:10624000882341F0FD1431F06D2D6F5F8F2D8F5F2E
:106250000E94F656CD2DDD27C7FDD0958091030510
:106260009E01281B3109C901181619065CF0CE01E0
:10627000019797FF02C080E090E08093030510E152
:10628000DD240BC025303105D4F3CE0104978B30CB
:1062900091059CF38AE090E0F0CFF0900305FD0CAF
:1062A000AF2CBB2495012F5F3F4F442737FD40950E
:1062B000542FCA15DB0511F401E101C000E182E1B0
:1062C000612F72E0E72E0E94255C80915501F8163F
:1062D00029F481E0612F4AE20E94E45A8F2D63E69F
:1062E00078E04FE00E94F253CA15DB0531F480914B
:1062F0007208882311F001E101C000E188E1612FFB
:1063000043E658E02FE00E94E85AD394185F3D2DF1
:10631000363019F6DF91CF911F910F91FF90EF90DA
:10632000DF90BF90AF900895AF92BF92CF92DF926F
:10633000EF92FF920F931F93CF93DF935B016C015A
:1063400010E1E12EF12CC0E0D0E800E010E89E0161
:1063500040E050E0CA01B9010E946768A616B7067E
:10636000C806D90610F4C027D127169507950894BA
:10637000E108F108E114F10461F4CE01DF91CF915D
:106380001F910F91FF90EF90DF90CF90BF90AF9053
:106390000895C02BD12BDBCFE1E0683068F4E0E05A
:1063A00070E09B01220F331F220F331F260F371F70
:1063B000A90142595C4F0EC070E0685070409B01CB
:1063C00053E0220F331F5A95E1F7260F371FA9011B
:1063D0004A565C4FDA012C9180509C4F97FD0FC0BC
:1063E000B8E080309B078CF0EE2319F028E030E015
:1063F00002C024E030E0240F351FF901208133274B
:1064000027FD3095322F222730C0EE2329F0692F47
:106410009070880F991F03C0692F66959170262F81
:1064200030E0FA01E20FF31F6181772767FD709575
:10643000AC0155954795649F9001659F300D749F01
:10644000300D11246081772767FD709540E052E0A0
:10645000481B590B55954795649FC001659F900D4A
:10646000749F900D1124280F391FC90169E170E054
:106470000E94A668CB0108952F923F924F925F929F
:106480006F927F929F92AF92BF92CF92DF92EF92E4
:10649000FF920F931F93DF93CF9300D00F92CDB74E
:1064A000DEB7182F9924939480918808883008F4D7
:1064B00099248FE19FE00E946919992011F05AE018
:1064C00001C056E084EA98E0612F40E020E030E02F
:1064D00000E075E2E72E7FE0F72ECC24C394A52ED2
:1064E0000E94E11A4091880850E04F5F5F4F84E2BC
:1064F00060E021E00E945B5D80918808992079F03E
:1065000090E008977C0103E0EE0CFF1C0A95E1F790
:10651000E80EF91E26E933E0E20EF31E0CC090E00F
:106520007C01EE0CFF1CEE0CFF1CE80EF91E8EE643
:1065300093E0E80EF91E0091A4080150D090A50840
:10654000113661F0123628F41434D1F0153471F597
:106550000EC01436A9F0153649F509C0DD2031F119
:106560001092A50881E60E94245FDD241FC080915F
:1065700004058823D9F01D14CCF48D2D815014C04E
:1065800080910405882391F02D2D332727FD309528
:10659000992019F089E090E002C085E090E028178A
:1065A000390724F48D2D8F5F8093A5088091A5086D
:1065B00080930405CE2C4F2C6E2C7F2C90E122244E
:1065C0003324A02EBB24A7FCB094F30141913F01DA
:1065D000552747FD509521E0A214B30409F020E0AF
:1065E00088E1692F99830E945B5D0894211C311C0E
:1065F0009981985F983349F7992001F1A5E06A2EB7
:10660000712C6E0C7F1C90E1F5E02F2E312CF301E4
:1066100041913F01552747FD509521E0A214B30455
:1066200009F020E080E3692F99830E945B5D089464
:10663000211C311C9981985F903349F70F3F11F469
:1066400021E0D11020E08CE068E048E15FE00E94AA
:10665000185B992019F089E090E002C085E090E095
:1066600021E0A816B90609F020E08CE068E341E1DA
:106670005FE00E94185B992019F089E090E002C069
:1066800085E090E0A816B90694F407FD4EC0A02E50
:10669000BB24A7FCB094AE0CBF1C812FF501608118
:1066A0004CE924E60E940D14F50180833EC01016CB
:1066B000E4F5812F6091A3084CEF24E000E00E94F4
:1066C000FF138093A30890917D04992371F1992081
:1066D00021F050E194E049E003C058E092E045E049
:1066E00024E6820230011124892F90E09095819553
:1066F0009F4F869D9001879D300D969D300D1124F2
:10670000EC2DF42DA52E00E0C9016A2D702F0E94FA
:10671000A6686193260D371D8E2F8C198417A0F360
:1067200082E00E9409550E94A555809104058823A6
:1067300051F0AA24ECE92E2EEFEF3E2E4D2C5524DD
:1067400047FC5094A5C000E01CEFAA24BB2470E2D3
:10675000D72EACC0C90165E0880F991F6A95E1F793
:10676000992019F064E070E002C062E070E00E94DD
:10677000A668462F062F055C37016A0C711CF301D1
:106780008081992787FD909555E0880F991F5A952C
:10679000E1F7B1010E94A668562F90E2D92ED60EDD
:1067A0002F5F3F4F8D2D90E09B838A8342165306C7
:1067B00009F050C082349105ACF48AE3C82EC40EAF
:1067C000625E8C2D45E059830E94C55B5981EA8148
:1067D000FB81E134F10531F0652F615E8C2D45E0E0
:1067E0000E94C55BFD2DF03430F4802F81506D2D5B
:1067F00045E00E94C55B2A813B812F33310594F42B
:1068000001506D2D6F5F802F45E00E94C55B8A812E
:106810009B818E33910531F06D2D6E5F802F45E0A9
:106820000E94C55B8091800490918104009741F49F
:10683000123631F0133621F0123411F0133439F5D9
:10684000812FF30160814CE924E60E940D14F301CD
:1068500080831DC02A813B81213431052CF4615E87
:10686000802F43E00E94C55B3D2D303428F4802FFB
:106870006D2D43E00E94C55B8A819B818F3391051A
:1068800034F46D2D6F5F802F43E00E94C55BA394AD
:106890002A2D30E0992019F089E090E002C085E0CF
:1068A00090E0281739070CF455CF4DCFC8016091FF
:1068B00088080E94CC31BCE3EB2EEA0C9C01A5E0D9
:1068C00036952795AA95E1F76D2D621B8E2D0E94B6
:1068D000795B9501237030702115310521F48E2DDF
:1068E00060E20E94795B0894A11CB11C005E1F4FFE
:1068F00090E4A916B104D1F68CE560E040E40E9472
:10690000C95B0F900F900F90CF91DF911F910F9166
:10691000FF90EF90DF90CF90BF90AF909F907F90CF
:106920006F905F904F903F902F9008952F923F92DD
:106930004F925F926F927F928F929F92AF92BF928F
:10694000CF92DF92EF92FF920F931F93DF93CF933B
:10695000CDB7DEB7A2970FB6F894DEBF0FBECDBF9E
:106960008F8F98A36A8B80918204882309F474C066
:1069700080910505882319F0815080930505809149
:10698000AF069091B0062091AD063091AE06820F11
:10699000931F2091B1063091B206820F931F209170
:1069A000B3063091B406820F931F209138073091BF
:1069B00039072C01421A530A920157FE03C0309541
:1069C00021953F4F41E0213034073CF09093390747
:1069D0008093380781E08093850480916D01863F24
:1069E000D9F1909108019233B8F1909135079F5FEA
:1069F00090933507903160F020913607309137073A
:106A00002F5F3F4F3093370720933607109235079B
:106A100090918504992321F0109237071092360740
:106A20002091360730913707992787FD90950A9670
:106A300067E771E0869FA001879F500D969F500DDC
:106A400011244217530740F4237030702130310570
:106A500019F480E10E94606880916C01582F517098
:106A60005F5F598781FF02C01D8602C063E06D87AA
:106A70006090A001662009F44AC08985E82FF0E003
:106A8000EE0FFF1FEB52FB4FA080B180CC24B7FC70
:106A9000C094DC2C9D85E92FF0E0EE0FFF1FEB5238
:106AA000FB4F20813181442737FD4095542FCA0187
:106AB000B9010E9467687B018C01C601B501A6017E
:106AC00095010E946768E60EF71E081F191F662DC4
:106AD00070E080E090E0EAE0660F771F881F991F62
:106AE000EA95D1F724E630E040E050E00E94DB6810
:106AF000B901CA010E9467686E157F05800791077A
:106B000030F4C801B7010E9494314C0102C08824BE
:106B10009924B40180E090E024E630E040E050E0C9
:106B20000E9467686B8F7C8F8D8F9E8F68E2662EC8
:106B300061E0762EADEAB6E0BE8BAD8BFE013196FC
:106B4000F88FEF8B50E0252E51E0352E28E831E00C
:106B50003F872E8745ED54E05A8F498F2901F98BE5
:106B6000E88BBC8BAB8BEE24FF241B865A895170BB
:106B700059A3AE2C8E2D0E94FC149C01D3011196BA
:106B80008D919C911297281B390BB901882777FDAD
:106B90008095982F4AE0660F771F881F991F4A95A6
:106BA000D1F7121613062CF45D962D913C915E9749
:106BB00003C0F301278530892436310514F424E617
:106BC00030E0442737FD4095542F0E94DB6889014F
:106BD000FCEF21303F072CF024E00030120724F4B2
:106BE00005C000E01CEF02C000E014E080916E01DF
:106BF00080FF0FC080916C0190E08170907042E046
:106C000050E0481B590BE416F50619F41095019550
:106C10001F4FA98DBA8D0D931D93BA8FA98FC801EF
:106C20000F968F319105F0F4B4E0EB16F1047CF48B
:106C30008A2D8F5F0E94EE5F90E00197E1E0F0E027
:106C400002C0EE0FFF1F8A95E2F7CF0108C081E076
:106C500090E00E2C02C0880F991F0A94E2F7FB8582
:106C6000F82BFB872A2D243008F07AC139A1332371
:106C700009F05FC08091940181FF5BC06701CC0C7B
:106C8000DD1C42E651E0C40ED51ED60111968C9152
:106C90001197807C09F44DC08C91859585958595DB
:106CA00061E040E00E94C90F882309F442C0D60188
:106CB000EC91E770F0E0DF01AA0FBB1FA657BB4FB6
:106CC000EE0FFF1FE65AFE4F8D919C911197208188
:106CD0003181821B930B62E070E00E94A668F7018D
:106CE000EE0FFF1FED59FE4F2081422F440F440F3E
:106CF00045954595552747FD5095649FC001659F73
:106D0000900D749F900D11246FE170E00E94A668B1
:106D1000660F771F660F771F22952695269523709D
:106D2000213019F0223029F403C0060F171F01C0CB
:106D30008B018114910409F1B985AB1619F0ED8529
:106D4000AE16D9F46091A00170E080E090E04AE0D6
:106D5000660F771F881F991F4A95D1F7980144271E
:106D600037FD4095542F0E9467682B8D3C8D4D8DCB
:106D70005E8D0E94DB68022F132FF201EA54FE4F52
:106D8000808160E040E00E94C90F882369F0F20131
:106D9000E954FE4F808160E040E00E94C90F8823E3
:106DA00029F4CC24C39404C0CC2402C032E0C32E06
:106DB00080916C0190E08170907022E0A22EB12C45
:106DC000A81AB90AAE14BF0469F580919901807FB1
:106DD00049F1C80180509C4F62E070E00E94A668B3
:106DE0009B01EC2DF0E0EE0FFF1FEE0FFF1FA70140
:106DF000440F551FCA01A3E0880F991FAA95E1F718
:106E0000841B950BE80FF91FEE5CFC4F6081772720
:106E100067FD7095C9010E947F26AC01440F551F84
:106E200030E028C031E0101611060CF430E08C2D53
:106E300090E0A701440F551FFA0163E0EE0FFF1F1A
:106E40006A95E1F7E41BF50B880F991F880F991FCE
:106E5000E80FF91FE857FE4FE30FF11DE655FE4F0F
:106E60006081772767FD7095C8013AA30E947F264D
:106E7000AC013AA1EC2DF0E0EE0FFF1FEE0FFF1F6B
:106E8000B701660F771FCB0113E0880F991F1A9582
:106E9000E1F7861B970BE80FF91FE857FE4FE30F4A
:106EA000F11DE455FE4F6081772767FD70956C59A1
:106EB0007F4F882777FD8095982FDA019D01442721
:106EC00037FD4095542F0E94676824E630E040E08B
:106ED00050E00E94DB68022F132FAE14BF0499F517
:106EE00080919901982F907F09F466C60050144054
:106EF00063C6D101ED91FC911197608180916E0183
:106F000080FD6195772767FD7095872F972F6358D0
:106F10007F4F8F4F9F4F20E034E0201B310B4427E1
:106F200037FD4095542F0E94676820E038E040E02C
:106F300050E00E94DB682030B8E03B07B0E04B0730
:106F4000B0E05B0739F4D101ED91FC91208133274A
:106F500027FD3095220F331FE889F989318320837B
:106F6000AB89BC890D931D93BC8BAB8B0894E11C42
:106F7000F11CE2E0F0E06E0E7F1E288939892E5F59
:106F80003F4F398B288B2E0E3F1E4EE050E0440EB3
:106F9000551E57E0E516F10409F0EBCD00919D0177
:106FA0006B85062380913A078095802319F088E14C
:106FB0000E94606800933A0780E094E09093BC06DA
:106FC0008093BB069093BE068093BD06EAE8F4E08A
:106FD0002AE531E0A5ECB6E0BD0181919191D9019E
:106FE0004D915D919D01841B950B880F991FDB01CD
:106FF0008D939D93BD01B4E0E239FB0771F7809159
:10700000920490919304880F991F9093CE068093D9
:10701000CD068091940490919504880F991F9093C8
:10702000D0068093CF068091960490919704880FA4
:10703000991F9093D2068093D106809198049091E5
:107040009904880F991F9093D4068093D306E5EF97
:10705000F6E0FC87EB8725ED36E041915191619197
:107060007191D9014D935D939D01B7E0E533FB0725
:10707000A1F7C090A001CC2009F47AC0E985AE2E1A
:10708000BB24AA0CBB1C2DEA422E26E0522EA40CD7
:10709000B51CD5012D903C90442437FC4094542CD1
:1070A000BD850B2F10E0000F111F0355194FF8017C
:1070B00020813181442737FD4095542FCA01B90101
:1070C0000E9467683B014C01C201B101A20191011C
:1070D0000E946768660E771E881E991EDD24EE24C6
:1070E000FF248AE0CC0CDD1CEE1CFF1C8A95D1F736
:1070F000C701B60124E630E040E050E00E94DB68C2
:10710000B901CA010E946768661577058805990567
:1071100078F5C401B3010E949431BC0180E090E095
:1071200024E630E040E050E00E9467683B014C01FB
:10713000C201B101A70196010E946768A4019301F1
:107140000E94DB68D5012D933C93F8016081718129
:10715000882777FD8095982FA70196010E94676880
:10716000A40193010E94DB68D80111963C932E93F1
:10717000E0909E018E2D807E09F4DEC0B9852B2F14
:1071800030E0220F331FF901E355F94F408151815F
:10719000CE010196280F391FD901ED91FC91BD85D3
:1071A0006B2F70E0660F771FDB01A355B94F2D9150
:1071B0003C91860F971FDC018D919C91BA89B1FD9E
:1071C00005C0E40FF51F280F391F04C020E030E090
:1071D000E0E0F0E0A0919F01AA2349F0B0E0AA0FFF
:1071E000BB1FA555B94F0D911C91119702C000E02E
:1071F00010E0E2FE03C0F095E195FF4FE3FE03C00F
:10720000309521953F4FE4FE03C0109501951F4F27
:1072100080919E01829586958770823071F18330CE
:1072200020F4813009F088C007C0833009F459C0C8
:10723000843009F081C06CC0C90168E070E00E9430
:10724000A6687B01C90160E870E00E94A668290178
:107250004E185F087201E61AF70AC90160E072E091
:107260000E94A668E61AF70AC8018E1B9F0B90932E
:10727000C0068093BF06CF0120C0CF0168E070E058
:107280000E94A6687B01CF0160E870E00E94A668BA
:107290003F016E187F087301E61AF70ACF0160E01C
:1072A00072E00E94A668E61AF70AC801821B930BD7
:1072B0009093C0068093BF06C90162E070E00E940F
:1072C000A668600F711FCB018E0D9F1D9093C206A3
:1072D0008093C1066E197F097093C4066093C3063C
:1072E0002BC0C8018E1B9F0B9093C0068093BF06D6
:1072F000E00FF11FCF01820F931F9093C20680937E
:10730000C106E21BF30BF093C406E093C30614C05E
:10731000C8018E1B9F0B9093C0068093BF06C801C7
:10732000820F931F9093C2068093C106021B130B1A
:107330001093C4060093C30680918204882311F041
:107340000E940A2F80E4E5EFF6E0DF011D928A95A6
:10735000E9F7BA89B1FF2DC080916C0190E081708E
:10736000907022E030E0281B390B80E090E0ED893E
:10737000FE89AF89B88D2817390729F0118210824C
:1073800011961C921E9201963296129684309105A7
:1073900091F71092C6061092C5061092C806109278
:1073A000C7061092CA061092C9061092CC06109217
:1073B000CB068AE693E090930101809300019C0143
:1073C0002F5F3F4F30930301209302019C012E5FFA
:1073D0003F4F3093050120930401039690930701DA
:1073E000809306012BEF422E27E0522E9BE7692E59
:1073F00097E0792E8BE3282E87E0382E19861D869C
:1074000089850E94FE0D7C01FC01808181508031C4
:1074100008F0ADC2838161E040E00E94C90FD20153
:107420009C918823A1F4292F1C92F7019181892F27
:107430008850823008F08AC287818E70843009F4C7
:1074400085C2993009F04BC000E01CEF4AC021E032
:10745000911120E081E0D2018C93D7011196EC913B
:107460003E2F3150832F90E0DC01AA0FBB1FA355A4
:10747000B94F0D911C911197343160F0B9853B17CC
:1074800048F4DC01AA0FBB1FAA0FBB1FAB50B94FBA
:107490000D911C91D70117963C911797832F8073FC
:1074A00081F0832F8295837090E0019741E050E056
:1074B00002C0440F551F8A95E2F7CA015D85582B1B
:1074C0005D8736FF0EC0E53060F4F0E0EE0FFF1F81
:1074D000E250FF4FC70108969183808302C000E00D
:1074E00010E0D7011796CC901797C6FC0BC01896E2
:1074F0008C911897882331F02AA30E94E10D080F80
:10750000191F2AA1F7018681882321F48581882308
:1075100009F458C1D3016D917D918D919C91139780
:10752000222389F420E031E040E050E00E94DB6853
:1075300050954095309521953F4F4F4F5F4F4801F3
:10754000820E931E5AC08C2D8E70843051F5D70157
:10755000EC91F0E0EE0FFF1FED52F94F6081718169
:10756000882777FD8095982F20E034E640E050E0B2
:107570000E946768F3016083718382839383D701DC
:1075800012962C911297222361F0332727FD309514
:10759000432F532F0E94DB68F30120833183428302
:1075A0005383D3016D917D918D919C91139720E030
:1075B00031E040E050E00E94DB6850954095309506
:1075C00021953F4F4F4F5F4F4801820E931E81140C
:1075D000910499F0F701258197FE22952F7030E0F4
:1075E00044E650E0249FC001259F900D349F900DEC
:1075F0001124D10111969C938E93F1018081918188
:10760000009799F020918204222319F00197918329
:107610008083D1018D919C911197009731F0F301F6
:107620006081718182819381B7C08114910409F4D2
:10763000C9C0D70116968C911697882309F4B4C057
:1076400080918204882309F476C012962C911297B7
:107650002223B1F0332727FD309537FF03C0309543
:1076600021953F4F332727FD3095432F532F60E05F
:1076700070E080E293E00E94DB6859016A0106C075
:10768000A12CB12CF0E2CF2EF3E0DF2EF7018681A2
:1076900018141904FCF48F7090E00097F1F144E69F
:1076A00050E0849F9001859F300D949F300D1124F0
:1076B000442737FD4095542FC601B5010E94DB6871
:1076C000F30180819181A281B381280F391F4A1F64
:1076D0005B1F2CC082958F7090E00097F1F044E61C
:1076E00050E0849F9001859F300D949F300D1124B0
:1076F000442737FD4095542FC601B5010E94DB6831
:1077000059016A01D3012D913D914D915C911397DF
:107710002A193B094C095D0909C09801442737FD26
:107720004095542F542F432F322F2227F3012083CB
:10773000318342835383D3016D917D918D919C91CF
:1077400020E031E040E050E00E94DB68C801AA2759
:1077500097FDA095BA2F1814190434F482179307D3
:10776000A407B50734F012C0281739074A075B078A
:107770006CF4222717FD2095322F322F212F102F46
:107780000027F3010083118322833383D3016D919A
:107790007D918D919C91139720E031E040E050E085
:1077A0000E94DB6889010EC0C801AA2797FDA09539
:1077B000BA2FBA2FA92F982F8827F301808391839E
:1077C000A283B383D70114966C911497633061F14F
:1077D000643028F4613051F06230A0F444C0653068
:1077E00069F1653038F1663081F52BC0F701818190
:1077F000893029F417FD35C0005012400EC017FF24
:1078000032C02CC0D70111968C911197893041F468
:107810001016110604F100501E4F000F111F23C057
:1078200010161106DCF01FC017FF1DC01095019542
:107830001F4F19C01016110674F010C017FF0EC0AC
:1078400010C0101611063CF00CC06750C8010E9411
:10785000CC318C0108C000E014E005C000E010E06D
:1078600002C000E01CEFF701878180FD13C0E181B9
:10787000EE2381F0E53070F4F0E03197EE0FFF1F5A
:1078800021E030E02C0F3D1FE20FF31F808191813A
:10789000080F191FB801882777FD8095982FD70109
:1078A00012962C911297332727FD3095432F532F93
:1078B0000E946768F701008110E0015010402781A5
:1078C00026952770213071F0F801EE0FFF1FEE0FA3
:1078D000FF1F223069F5EB50F94F6083718382837B
:1078E000938334C024E630E040E050E00E94DB683F
:1078F000E22EC32EDA01000F111F000F111F0B50D3
:10790000194FF80120813181428153816E2D7C2DE8
:10791000CD010E94676820E034E040E050E00E9422
:10792000DB68D8012D933D934D935C9313970EC064
:10793000EB50F94F2081318142815381260F371F4F
:10794000481F591F2083318342835383B985BF5F0A
:10795000B9870894411C511CE4E0F0E06E0E7F1ED4
:1079600022E030E0220E331EB03209F049CD0E94F1
:10797000F60D8C01ED84E0FE05C0882319F48EE13C
:107980000E946068E1FE0BC0C801907080349105D0
:1079900019F08834910519F48FE10E946068E2FEC5
:1079A0000DC010700038110531F00838110519F0BC
:1079B0000039110519F480E20E946068B3EE4B2E85
:1079C000B4E05B2E3F8D28A1832F922F9A87898761
:1079D00022243324598A488AAB85BC85ED90FD90DA
:1079E0000D911C91C801B70124E630E040E050E061
:1079F0000E94DB68EB85FC852083318342835383BF
:107A0000A889B9892D933D93B98BA88BEE85FF8505
:107A1000E35AFE4F80819181EE85FF85E55AFE4F46
:107A20002081BAE02B0260011124E8EEF3E0CE0ED3
:107A3000DF1EEE85FF85E65AFE4F20812B025001A6
:107A40001124A8E14A2EACEF5A2EA40CB51C9601C5
:107A50004C2D232F8C159D0514F4482F292F842E8F
:107A6000922E8A149B040CF44501E114F1040105E3
:107A7000110569F19401442737FD4095542F1E14D8
:107A80001F041006110654F4B601882777FD80956F
:107A9000982F621B730B840B950B0DC0C501AA2791
:107AA00097FDA095BA2F29013A01481A590A6A0A86
:107AB0007B0AC301B201A80197010E94676820EA0E
:107AC00036E841E050E00E94DB6879018A01C40198
:107AD0000E944A193C01882477FC8094982C6E0CF3
:107AE0007F1C801E911EC6010E944A198C01C5018F
:107AF0000E944A19222717FD2095322F06151705D7
:107B00002805390514F438014901AA2797FDA095E5
:107B1000BA2F84017301681679068A069B0614F44D
:107B20007C018D01EE85FF85E45AFE4F808188231C
:107B300041F010950095F094E094E11CF11C011DBA
:107B4000111DF8E8CF2EF1E0DF2EC20CD31CF60198
:107B5000E358FD4F8081882389F060E040E00E9477
:107B6000C90F882359F0F601E258FD4F80810E9429
:107B7000E10D7C010027F7FC0095102FF894A985F2
:107B8000BA85ED92FD92BA87A9877894EB85FC853A
:107B90003496FC87EB87E2E04E2E512C240C351CEA
:107BA0002E853F852B5F3F4F3F872E8730E2231680
:107BB000310409F011CF04C08F7009F09AC9C3C90C
:107BC000A2960FB6F894DEBF0FBECDBFCF91DF9166
:107BD0001F910F91FF90EF90DF90CF90BF90AF90EB
:107BE0009F908F907F906F905F904F903F902F90DD
:107BF0000895EF92FF920F931F93DF93CF93CDB72A
:107C0000DEB7C054D0400FB6F894DEBF0FBECDBF74
:107C10008E010F5F1F4FC80163E00E94963481E21E
:107C2000E82EF12CEC0EFD1EC70161E00E94963497
:107C3000E4EEF2E0418152816081D8012D913C91C6
:107C4000D7018D919C911197662329F0B901681B8A
:107C5000790BCB0102C0821B930B840F951F73E03D
:107C6000883E97072CF4ACEF89319A0724F005C0C1
:107C700088EE93E002C088E19CEF92838183359681
:107C80000E5F1F4F62E070E0E60EF71E73E0E43314
:107C9000F70781F680916C0190E08170907022E08E
:107CA00030E0281B390B80E090E02817390721F0DD
:107CB000FC01E659FC4F1082019684309105A9F72A
:107CC00086E00E94095581E00E946068C05CDF4F39
:107CD0000FB6F894DEBF0FBECDBFCF91DF911F91DD
:107CE0000F91FF90EF9008952F923F924F925F92E5
:107CF0006F927F928F929F92AF92BF92CF92DF92BC
:107D0000EF92FF920F931F93DF93CF930F92CDB714
:107D1000DEB710916A011F70813809F475C082388E
:107D200088F48332F1F1843230F48032E1F082322F
:107D300009F07CC045C0813609F45BC0803809F089
:107D400075C01BC08438F9F0853838F4823809F4DE
:107D50004AC0833809F06AC040C08538E1F08F3BE3
:107D600009F064C057C0153009F060C080918604E6
:107D700091E08927809386044BC00E942B140E94B7
:107D80006A1480E805C084E590E30E946A1484E8E0
:107D90000E94245F4BC084EE98E40E946A1485E838
:107DA000F7CF812F8F5F80936A01863010F0109299
:107DB0006A0181E00E94095583E10E94606836C033
:107DC000112319F0812F815001C085E080936A0151
:107DD00081E00E94095584E1F0CF80E799E10E949B
:107DE0005A1483E8D5CF8BE09AE10E945A1482E8B6
:107DF000CFCF80912B06823021F483E080932B0635
:107E000007C0153099F402C00E94BF2F0E94A91428
:107E100087E1D3CF81E00E94245F83E00E94245F4A
:107E200082E00E94245F81E080931B0880919C0186
:107E300060E040E00E94C90F882331F080911B0868
:107E4000882311F40E94F93D80919C0160E040E09C
:107E50000E94C90F80931B0880916A01803108F04D
:107E6000D3C09091080180915701981710F496E0C3
:107E700001C094E0B8E8EB2EB1E0FB2E0AE0D70198
:107E80004D917D01802F60E024E099830E94255A66
:107E9000055F9981083799F7492F406884E260E1CE
:107EA0000E94990E84E268E146E50E94E45A8091BE
:107EB0002B06882399F0823011F406E001C004E01B
:107EC00040912C0650912D068EE560E1202F0E94F6
:107ED0001A0E83E368E140E00E943E0F40919A0150
:107EE00083E04802A00111244151584F84E260E12F
:107EF00023E000E00E94E85A809199018F7031F0F0
:107F000089E360E14BEE57E00E94475BAEE0EA2E6A
:107F1000A1E0FA2EF0E0CF2EF1E0DF2E66247724E8
:107F2000EFE19E2EF70101917F01D601ED91FD91C8
:107F30006D01808187FD8D5F85958595843E0CF46C
:107F400084EEA82E8D3114F07CE1A72E862D815071
:107F50008230F8F4802F64E046E30E94C95B2091F0
:107F60006C0130E02625372520FD04C08091990161
:107F70008F7061F4802F81506EE143E00E94C95BF5
:107F8000802F8F5F6EE143E00E94C95B992D9A19A3
:107F900014C0802F8B516BE346E30E94C55B802E9B
:107FA0008A94882D6AE343E00E94C55B882D6CE3C8
:107FB00043E00E94C55B0A0D9BE36DEF862E800EA9
:107FC0005DEFA52EA90E882D6A2D47E099830E94AA
:107FD000C95B9981692F6D5F882D47E00E94C55B61
:107FE000802F8D5F6A2D47E00E94C95B882D6A2D26
:107FF00047E00E94C55B0894611C711CB4E06B16DD
:10800000710409F08FCF27C080E060E048E851E0BC
:108010002AE001E10E94E85A9091080180915701FD
:10802000981710F442E001C040E084E560E00E944F
:10803000990E80912B06882371F0823011F402E0B2
:1080400001C000E040912C0650912D068FE660E0C3
:10805000202F0E941A0E123008F085C049E0E42E4D
:1080600045E0F42E00E039E1A32EB12C2BE1922E55
:1080700090E2692E712C80E8482E512CF701219056
:1080800031907F01113011F1802F8370899DC02CB8
:108090001124D02ED694D694DD0CDD0CDD0CF8E244
:1080A000DF0EC101B3010E94A6689B01C101B201AC
:1080B0000E94A668AB01421B530B420D531D8C2D31
:1080C0008F5D6D2D20E20E945B5D48C0043018F486
:1080D000B2E2CB2E02C0AEE5CA2E802F8370D82E1E
:1080E000DD0CDD0CD80E26E2D20EC10137FE04C035
:1080F00088279927821993098A9DA0018B9D500D8D
:108100009A9D500D112440505E4F452F550F550B31
:1081100045954595842E4A3114F0E9E18E2E8C2D3B
:1081200089516D2D43E325E50E94975B6D2D6250CB
:108130008C2D45E00E94C95B1214130414F4C394FF
:1081400001C0C8186D2D6F5F8C2D482D0E94C55B36
:108150006D2D61508C2D482D0E94C55B0F5F08303E
:1081600009F08CCF8AC0153008F07DC00E94E71F4F
:10817000123061F0812F880F810F880F8950912F65
:108180009150192F110F190F110F02C080E016E046
:10819000C82E992787FD90952C01440C551C480E3C
:1081A000591E60E2D62EEE24FF2452E0852E912C3B
:1081B000880E991E3C011AC00E943B0F5C018C2D59
:1081C00060E040E00E94C90F082FA501440D551D35
:1081D0008AE06D2D23E00E94E85A0894E11CF11C0E
:1081E00083E090E0480E591E98E0D90EC394C70171
:1081F000860D971D88169906FCF6812F992787FD15
:1082000090952C01440C551C480E591E30E2D32E7B
:10821000EE24FF2422E0822E912C880E991E3C0130
:108220001AC00E943B0F5C01812F60E040E00E9479
:10823000C90F082FA501440D551D85E66D2D23E0BE
:108240000E94E85A0894E11CF11CA3E0B0E04A0E39
:108250005B1EB8E0DB0E1F5FC701860D971D8816F9
:108260009906FCF60AC040918804509189048CE379
:1082700068E224E004E00E941A0E0F90CF91DF9193
:108280001F910F91FF90EF90DF90CF90BF90AF9034
:108290009F908F907F906F905F904F903F902F9026
:1082A000089518161CF0109203050895282F3327FF
:1082B00027FD309590910305291B3109462F50E089
:1082C0004217530724F4861B8093030508954650F4
:1082D00050402417350724F48A5F861B80930305DA
:1082E0000895AF92BF92CF92DF92EF92FF920F93D9
:1082F0001F93DF93CF930F92CDB7DEB7D82E87E6CB
:108300009CE00E94691985E798E06D2D41E02FEC13
:1083100037E008E07DE6E72E7CE0F72E5BE0C52E37
:1083200010E1A12E0E94E11A10917508F0907608D4
:10833000812F67E00E9451412091550130E02F5F6D
:108340003F4F442737FD4095542F8AE260E001E11A
:10835000B2E0EB2E0E94255C2D2D253451F0263401
:1083600018F4243401F511C03D2D343671F0353642
:10837000D1F41130C1F4FF20B1F0809104058823BD
:1083800091F08091760881500CC0113061F44F2D2E
:10839000493048F480910405882329F080917608BB
:1083A0008F5F8093760880910305882309F088C049
:1083B00088E062E67CE00E943F5B113031F481E0AE
:1083C00090E020910405222311F080E090E0082F36
:1083D00000618CE368E048E851E02AE00E94E85A36
:1083E00080910405882359F48091070587FF07C011
:1083F00081E0809304051092070510927608809121
:108400000405882381F020910705332727FD309547
:108410008F2D90E08217930734F410920405109288
:10842000070510927608113009F04DC080910405BF
:10843000882309F448C08091760890910705891B2C
:108440008093760887FF02C01092760880917608A4
:108450008A301CF089E08093760810920705AF2CD3
:10846000BB24F501E857FE4F80810E94EB2C682F5A
:1084700020918004309181042115310549F47D2D2E
:10848000723631F0733621F0723411F0733431F4F6
:108490008D2D40E021E40E940D14682F862F0E944C
:1084A000FB2C482FF501E857FE4F80838F2D880F56
:1084B0008F0D880F845C68E021E00E94255A03C07C
:1084C000A8E0EA2E02C0F0E1EF2E80910305823091
:1084D00008F084C08E2D6CE57CE00E943F5B4091EB
:1084E000950150919601123099F4FF2039F4809152
:1084F0000405882309F01AC421E019C48F2D8130A6
:1085000039F480910405882329F020E002E004C0BA
:1085100020E00DC420E001E087E46E2D0E941A0ED9
:10852000123009F059C080910405882339F48091F4
:10853000800490918104009709F44EC0FF2029F037
:108540009F2D913009F048C022C0809195019091F3
:108550009601ECE3AE2EB12CB5010E9492688D2DF0
:1085600040E02BE30E940D142CE3482F42039001BE
:1085700011248091950190919601B5010E94926815
:10858000280F391F309396012093950125C08091C3
:108590009501909196016CE370E00E949268082F1B
:1085A0000E5F8D2D602F41E02EE30E940D14081BFD
:1085B000602F772767FD7095209195013091960186
:1085C000261B370B309396012093950137FF04C08B
:1085D000109296011092950168E0E60E80910305D5
:1085E0008330F8F48E2D64E57CE00E943F5B01E06F
:1085F000133009F000E08CE36E2D402F0E943E0FF7
:10860000002349F08D2D6091930147EC29E30E94EE
:108610000D148093930178E0E70E8E2D893308F0D6
:1086200088C3809103058430C8F58E2D6DE47CE00D
:108630000E943F5B91E0143009F090E0809194013A
:10864000282F217030E0A901440F551F63E0220F4D
:10865000331F6A95E1F7420F531F485C534F8CE379
:108660006E2D2AE0092F99830E94E85A9981992357
:1086700079F06091940161708D2D40E021E00E94BD
:108680000D148170909194019E7F982B909394018A
:1086900098E0E90EEE2DE93308F04BC38091030515
:1086A000853030F5009199010F708E2D61E37CE0EB
:1086B0000E943F5B21E0153009F020E08CE36E2D35
:1086C000402F0E949C1A153069F48D2D602F40E0D8
:1086D00021E00E940D148F7090919901907F982B4A
:1086E00090939901F8E0EF0E2E2D293308F021C365
:1086F00080910305863040F50091990102950F7035
:108700008E2D6AE27CE00E943F5B21E0163009F08A
:1087100020E08CE36E2D402F0E949C1A163071F4DD
:108720008D2D602F40E021E00E940D148295807F06
:10873000909199019F70982B9093990138E0E30EE6
:108740004E2D493308F0F5C280910305873050F56E
:108750008E2D61E27CE00E943F5B91E0173009F0D2
:1087600090E040919A0186E04802A00111244E5FFA
:10877000534F8CE36E2D26E0092F99830E94E85A0F
:108780009981992349F08D2D60919A0140E024E070
:108790000E940D1480939A0168E0E60E7E2D7933D5
:1087A00008F0C7C280910305883008F58E2D6AEF66
:1087B0007BE00E943F5B01E0183009F000E086E3B7
:1087C0006E2D40919C01202F0E94EB0E002349F05A
:1087D0008D2D60919C014AEE26E10E940D1480933C
:1087E0009C0188E0E80E9E2D993308F0A2C280918A
:1087F0000305893008F051C08E2D61EF7BE00E94A7
:108800003F5B9CE3AA24BB24A5014751544FFA14B3
:1088100011F4193061F020919D0130E00A2C02C062
:10882000359527950A94E2F7022F017001C002E006
:10883000892F6E2D21E099830E94E85A0894A11C8B
:10884000B11C99819A5F9636F9F6193001F5ED2D34
:10885000E03631F080918004909181040097B9F066
:108860008D2D0E94245F1092040581E090E00F2C72
:1088700002C0880F991F0A94E2F720919D012827D2
:1088800020939D0182E00E9409550E94A555F8E0C1
:10889000EF0E2E2D293308F04CC2809103058A304B
:1088A00008F0E3C08E2D63EE7BE00E943F5B4091B9
:1088B000970186E0489FA00111244653544F1A3077
:1088C00041F4FF2031F480910405882321F002E077
:1088D00003C000E001C001E084E26E2D26E00E94AA
:1088E000E85A80919701882321F0833009F04DC028
:1088F00009C086E66E2D45EC5BE020E00E94185B27
:108900009CE308C082E76E2D42EC5BE020E00E9411
:10891000185B98E440919801552747FD5095440F06
:10892000551F440F551F4355544F1A3049F43F2DDE
:10893000313031F480910405882321F002E003C036
:1089400000E001C001E0892F6E2D24E099830E9490
:10895000E85A9981892F865D40919B0192E34902F3
:10896000A0011124445D5E4F1A3049F46F2D62302E
:1089700031F490910405992321F022E003C020E016
:1089800001C021E06E2D0E945B5D809197018130D6
:1089900001F582E46E2D4EE95BE020E00E94185B59
:1089A00040919801552747FD50954F5F5F4F1A3012
:1089B00049F47F2D713031F480910405882321F032
:1089C00022E003C020E001C021E08EE76E2D0E946E
:1089D0005B5D1A3009F043C080910405882331F4AF
:1089E00080918004909181040097C9F18F2D81308E
:1089F00079F0813018F0823091F522C08D2D609190
:108A0000970140E023E00E940D148093970127C056
:108A100080919701882311F0833031F48D2D60917E
:108A200098014EEF24E007C08130C9F48D2D60918C
:108A3000980140E02CE70E940D14809398010FC02C
:108A400080919701882311F0833049F48D2D609136
:108A50009B014CEF2AE00E940D1480939B0198E04B
:108A6000E90EEE2DE93308F064C1809103058B30E7
:108A700008F07AC080919701882311F0833019F5AE
:108A80008E2D6FE87BE00E943F5B4091A10185E065
:108A90004802A00111244F515F4F1B3011F421E215
:108AA00001C020E28EE46E2D0E945B5D1B3009F058
:108AB00055C08D2D6091A1014CEE24E10E940D1452
:108AC0008093A1014BC08130B9F401E01B3009F063
:108AD00000E080E06E2D49E75BE0202F0E94185BEC
:108AE0000023E1F1FD2DF038C9F581E080934D0EB2
:108AF00080E00E94606832C08E2D60E77BE00E94BB
:108B00003F5B8091980187FD03C083301CF403C054
:108B100080E001C082E08093980149E08402A001D6
:108B200011244C5A544F1B3031F480910405882392
:108B300021F002E003C000E001C001E08CE36E2DF3
:108B400029E00E94E85A1B3049F48D2D609198016C
:108B500040E022E00E940D148093980128E0E20E8C
:108B60003E2D393308F0E5C0809103058C3098F52F
:108B70008E2D6AE47BE00E943F5B31E01C3009F0FF
:108B800030E080919E01817090E0AC01440F551F50
:108B9000480F591F4D5B544F8CE36E2D23E0032F7C
:108BA00039830E94E85A3981332379F060919E011C
:108BB00061708D2D40E021E00E940D148170909134
:108BC0009E019E7F982B90939E0148E0E40E6E2DAF
:108BD000693308F0AEC0809103058D3040F50091F7
:108BE0009E01069501708E2D69E37BE00E943F5B3C
:108BF00021E01D3009F020E08CE36E2D402F0E9413
:108C00009C1A1D3071F48D2D602F40E021E00E94F0
:108C10000D148170880F90919E019D7F982B9093E9
:108C20009E0178E0E70E8E2D893308F082C0809196
:108C300003058E3040F500919401069501708E2D4C
:108C400061E37BE00E943F5B21E01E3009F020E001
:108C50008CE36E2D402F0E949C1A1E3071F48D2DD6
:108C6000602F40E021E00E940D148170880F9091E8
:108C700094019D7F982B9093940198E0E90EEE2D3E
:108C8000E93308F056C0809103058F3048F5009114
:108C900094010695069501708E2D68E27BE00E9496
:108CA0003F5B21E01F3009F020E08CE36E2D402F68
:108CB0000E949C1A1F3079F48D2D602F40E021E036
:108CC0000E940D148170880F880F909194019B7FF2
:108CD000982B90939401F8E0EF0E2E2D293348F550
:108CE00080910305803128F580910505882319F4CA
:108CF00021E0103109F020E080E06E2D44E15BE0DE
:108D00000E94185B1031A9F43D2D303891F4109277
:108D1000040589E18093050580E80E94245F109294
:108D20001F0682ED9FE20E946A1403C022E000E069
:108D3000F3CB0F90CF91DF911F910F91FF90EF90A8
:108D4000DF90CF90BF90AF9008956F927F928F92F7
:108D50009F92AF92BF92CF92DF92EF92FF920F93CA
:108D60001F93DF93CF930F92CDB7DEB7B82E82EB70
:108D70009EE00E9469198BE898E06B2D46E02FEC8D
:108D800037E008E0E2ECEE2EEEE0FE2ECC24C394B9
:108D90007CE0A72E0E94E11A80908B088A94D090E4
:108DA0008C08882D66E00E94514118E0CC2499245B
:108DB00087FC9094909103059C0D9C3009F44FC161
:108DC000E92EFF248E149F0439F480910405882332
:108DD00029F062E0A62E04C0AA2402C0AA24A3940B
:108DE00080E0612F4FEA5EE022E000E099830E947C
:108DF000E85A9981993010F048E301C041E3490FE6
:108E00008CE0612F0E94E45AF701EE0FFF1FEE0D78
:108E1000FF1DE052FC4F408187E0489FA0011124D4
:108E2000445B514FDD2011F000E001C00A2D88E1C4
:108E3000612F27E00E94E85AC701880F991F8E0D05
:108E40009F1D88579E4FFC01E85AFD4F2081253019
:108E500008F4F6C0FC01EA5AFD4F283008F4F9C0C6
:108E600040819D2D9130D1F53BC020E001C02A2DDD
:108E700088E4612F0E949F0EF701EE0FFF1FEE0D99
:108E8000FF1DE152FC4F4081552747FD5095ED2DC8
:108E9000E23011F020E001C02A2D88E7612F0E9406
:108EA0005B5D00E035C020E001C02A2D88E4612F21
:108EB0000E94EB0EF701EE0FFF1FEE0DFF1DE152BA
:108EC000FC4F4081FD2DF23011F020E001C02A2D31
:108ED00080E6612F0E94EB0E01E01AC020E001C085
:108EE0002A2D88E4612F0E949F0EF701EE0FFF1FCD
:108EF000EE0DFF1DE152FC4F40818D2D823011F0AF
:108F000020E001C02A2D86E6612F0E949F0E02E01C
:108F100080910405882339F4809180049091810424
:108F2000009709F486C0AA2009F483C09D2D9130D2
:108F3000D1F1913020F0923009F07BC046C037016A
:108F4000660C771C6E0C7F1CE0EEF3E06E0E7F1E4D
:108F50008B2DF301608140E02DE00E940D14F301A0
:108F60008083202F30E0853028F0883030F481E095
:108F700090E005C080E090E002C082E090E0281719
:108F8000390709F456C0C701880F991F8E0D9F1D20
:108F900088579E4FFC01EA5AFD4F1082895A9D4F17
:108FA000FC01108246C0013041F0C701880F991FB3
:108FB000E80EF91E8EED93E031C03701660C771C88
:108FC0006E0C7F1C8EED93E01AC0013089F0C70152
:108FD000880F991F0230F1F0E80EF91E8FED93E033
:108FE000E80EF91E8B2DF701608143E82DE71DC0C7
:108FF0003701660C771C6E0C7F1C8FED93E0680EBA
:10900000791E8B2DF30160814AEE26E10E940D143A
:10901000F3010EC0E80EF91E8FED93E0E80EF91E85
:109020008B2DF701608140E024E20E940D14F701CE
:109030008083C394185FFC2DF73009F0BBCE0FC0BE
:109040008A5A9D4FFC014081FD2DF13009F00DCF72
:109050000ECF40818D2D813009F025CF26CF0F9086
:10906000CF91DF911F910F91FF90EF90DF90CF9004
:10907000BF90AF909F908F907F906F9008956F9268
:109080007F928F929F92AF92BF92CF92DF92EF9298
:10909000FF920F931F93CF93DF93982E84EC9EE063
:1090A0000E9469198DE898E0692D47E02FEC37E0C0
:1090B00008E054EDE52E5EE0F52ECC24C39410E1DB
:1090C000A12E0E94E11A60908D086A9480908E080B
:1090D000862D66E00E945141B8E0FB2EDD24772406
:1090E00067FC7094409103054D0D403109F45DC05B
:1090F000A42EBB244F5F80E06F2D20E00E94CB0E9A
:10910000EE24E501CC0FDD1FCA5FDB4F8501000FA8
:10911000111F0B5F1B4F6A147B0471F48E1461F4F2
:1091200080910405882359F48091800490918104F2
:10913000009739F421E001C020E0CC2405C022E0F2
:1091400001C021E0CC24C394EE2091F48EE16F2D78
:10915000F80140810E94EB0ECC20D9F0892DF80156
:1091600060814AEE26E10E940D14F801808311C04F
:109170004881552747FD509580E66F2D0E945B5D25
:10918000CC2039F0892D688143E82DE70E940D1429
:109190008883E394FE2DF33009F0BDCFD39488E0AB
:1091A000F80EED2DE73009F09DCFDF91CF911F91A3
:1091B0000F91FF90EF90DF90CF90BF90AF909F9076
:1091C0008F907F906F900895AF92BF92CF92DF9271
:1091D000EF92FF920F931F93DF93CF9300D0CDB701
:1091E000DEB7182F80917701813019F0B8E1CB2ECE
:1091F00002C0AAE1CA2EFBEFBF2EBC0C89E19AE0A7
:109200000E9469198CE298E0612F40E02FED37E071
:1092100006E0EC2C0E946A1EF0902C08D0902D08DD
:109220008F2D67E00E945141609103058C2D90E0E5
:10923000462F50E09C01275030404217530761F4FD
:109240002F2D30E004972817390714F48FEF01C051
:1092500081E0680F60930305113629F1123678F426
:10926000143409F448C0153420F4123408F46AC0E8
:1092700063C0153419F1103609F064C009C0143602
:1092800008F45AC01436B9F1153609F05BC016C09F
:10929000FF2009F457C081E090910405911180E00E
:1092A000809304054FC080910405882309F44AC0C7
:1092B0001092040581E60E94245F44C02F2D2130C6
:1092C00059F4DD2049F080910405882329F080912C
:1092D0002D08815080932D082F2D30E08B2D99275C
:1092E00087FD90952817390769F5DD2059F18091A0
:1092F0002D0881501EC03F2D313061F48D2D8930F5
:1093000048F480910405882329F080912D088F5F0F
:1093100080932D082F2D30E08B2D992787FD909578
:109320002817390779F49D2D973060F480912D0826
:109330008F5F80932D0806C080910405882311F467
:1093400010922D0880910305882309F089C088E0D8
:109350006EE07AE00E943F5BEF2DE13031F481E076
:1093600090E020910405222311F080E090E0082F86
:10937000006182E468E049E751E02AE00E94E85A8F
:1093800080910405882359F48091070587FF07C061
:1093900081E0809304051092070510922D088091BA
:1093A0000405882381F020910705332727FD309598
:1093B0008D2D90E08217930734F4109204051092DB
:1093C000070510922D08FF2DF13009F04CC0809157
:1093D0000405882309F447C080912D089091070562
:1093E000891B80932D0887FF02C010922D08809161
:1093F0002D088A301CF089E080932D081092070513
:10940000AD2CBB24F501E758FE4F80810E94EB2C68
:10941000682F20918004309181042115310541F499
:10942000123631F0133621F0123411F0133431F4C6
:10943000812F40E021E40E941C14682F862F0E9497
:10944000FB2C482FF501E758FE4F80838D2D880FA8
:109450008D0D880F8E5B68E021E00E94255A03C0C5
:10946000E8E0EE2E02C070E1E72E80910305823025
:10947000A0F5C0906B01C694C694C69427E0C222A2
:109480008E2D67E07AE00E943F5B91E03F2D323005
:1094900009F090E046E08C2D849FA00111244452F5
:1094A000564F8CE56E2D26E0092F9A830E94E85ACC
:1094B0009A81992381F0812F6C2D40E026E00E9453
:1094C0001C148770880F880F880F90916B01977C10
:1094D000982B90936B0198E0E90E809103058330FF
:1094E00058F5C09077018E2D61ED79E00E943F5BC9
:1094F00091E0EF2DE33009F090E046E0FC2DF49F81
:10950000A00111244C53564F8CE56E2D26E0092FF7
:109510009A830E94E85A9A81992341F0812F6C2DF9
:1095200040E021E00E941C148093770128E0E20EC5
:109530003E2D393308F0FFC380917701813041F52A
:1095400080910305843030F58E2D66EB79E00E9422
:109550003F5B409175018F2D843011F421E401C0EF
:1095600020E486E66E2D50E00E945B5D9F2D9430D6
:1095700049F4812F6091750141E024E60E941C149A
:1095800080937501E8E0EE0EFE2DF93318F0D3C399
:1095900004E001C005E0809177018150823038F508
:1095A00080910305801710F58E2D66EA79E00E9400
:1095B0003F5B40917601F01611F421E401C020E4F4
:1095C00086E66E2D50E00E945B5DF01649F4812F17
:1095D0006091760140E025E00E941C1480937601A2
:1095E00028E0E20E3E2D393308F0A5C30F5F8091CD
:1095F0000305801720F58E2D6DE979E00E943F5B11
:1096000040915601F01611F421E401C020E486E6F1
:109610006E2D50E00E945B5DF01659F4812F609131
:1096200056014AE02DE20E941C14809356010E94CC
:10963000BB5D88E0E80E9E2D993308F07CC3C02EF8
:10964000C394809103058C1508F58E2D6DE879E0A3
:109650000E943F5B40915701FC1411F421E401C0CA
:1096600020E486E66E2D0E94850EFC1449F4812FBD
:109670006091570148E228E70E941C14809357012B
:10968000E8E0EE0EFE2DF93308F055C3C394809147
:1096900003058C1560F58E2D6CE779E00E943F5B29
:1096A00040916D01552747FD5095465F5F4FFC1473
:1096B00011F421E401C020E486E66E2D0E945B5D7A
:1096C0008091890D6E2D4DE60E94E45AFC1449F4F8
:1096D000812F60916D0146EF2EE60E941C1480934D
:1096E0006D0128E0E20E3E2D393308F024C3C39407
:1096F000809103058C1550F58E2D61E779E00E946D
:109700003F5B91E0FC1090E040916F0150E0440F0E
:10971000551F440F551F4C59564F86E66E2D24E0B9
:10972000092F9A830E94E85A9A81992349F0812F40
:1097300060916F0140E022E00E941C1480936F0151
:1097400088E0E80E9E2D993308F0F5C2C39480910D
:1097500003058C15C8F480916E01817021E0FC1026
:1097600020E06E2D43E559E0012F0E94052D817008
:1097700090916E019E7F982B90936E01E8E0EE0E23
:10978000FE2DF93308F0D7C2C394809103058C15E0
:10979000D8F480916E018695817021E0FC1020E064
:1097A0006E2D47E459E0012F0E94052D8170880F2E
:1097B00090916E019D7F982B90936E0128E0E20EB0
:1097C0003E2D393308F0B7C2C394809103058C1540
:1097D000E8F480916E0186958695817021E0FC10F9
:1097E00020E06E2D48E359E0012F0E94052D817085
:1097F000880F880F90916E019B7F982B90936E013C
:1098000088E0E80E9E2D993308F095C2C3948091AC
:1098100003058C15F8F480916E01869586958695E2
:10982000817021E0FC1020E06E2D4AE259E0012F0A
:109830000E94052D8170880F880F880F90916E010E
:10984000977F982B90936E01E8E0EE0EFE2DF93392
:1098500008F071C2C394809103058C1500F58E2D1C
:109860006DE179E00E943F5B01E0FC1000E080E6E2
:109870006E2D40915901202F0E94EB0E002349F0DC
:10988000812F609159014AEE26E10E941C148093B9
:10989000590128E0E20E3E2D393308F04CC2C39442
:1098A000BB24809103058C1508F048C0BB2019F437
:1098B0006DE079E002C06DEF78E08E2D0E943F5B95
:1098C000BB2019F4A090700102C0A0907801AA20DA
:1098D000A9F08A2D95E0899FA0011124FC1411F4B0
:1098E00021E401C020E486E66E2D0E945B5D80913C
:1098F000890D6E2D43E70E94E45A0AC001E0FC1076
:1099000000E086E66E2D49EF58E023E00E94E85A19
:10991000FC1439F4812F6A2D40E028E70E941C14C2
:10992000A82EBB2019F4A092700102C0A092780169
:10993000E8E0EE0EFE2DF93308F0FDC1C394B394B8
:109940002B2D223009F0ADCF809103058C15F8F452
:1099500080916E0182958F708095817021E0FC105E
:1099600020E06E2D4BEE58E0012F0E94052D8095D2
:1099700081708295807F90916E019F7E982B90934D
:109980006E0138E0E30E8E2D893308F0D4C1C39404
:10999000809103058C15F8F48091740182958F7085
:1099A0008095817021E0FC1020E06E2D4FED58E095
:1099B000012F0E94052D809581708295807F909166
:1099C00074019F7E982B9093740198E0E90EEE2D20
:1099D000E93308F0B0C1C394809103058C15D8F425
:1099E00080916B018095817021E0FC1020E06E2D4C
:1099F0004EEC58E0012F0E94052D809581709091CA
:109A00006B019E7F982B90936B01F8E0EF0E2E2D4B
:109A1000293308F090C1C394809103058C15E8F4B4
:109A200080916B0186958095817021E0FC1020E08B
:109A30006E2D4FEB58E0012F0E94052D809581700F
:109A4000880F90916B019D7F982B90936B0138E06C
:109A5000E30E8E2D893308F06EC1C3948091030507
:109A60008C1508F086C08E2D64EB78E00E943F5B79
:109A700092E4AA24BB24A5014555574FE0918301E8
:109A8000F0E00A2C02C0F595E7950A94E2F7E17040
:109A9000F070892F6E2D21E00E2F9A830E94E85AD4
:109AA0000894A11CB11C9A819A5F923721F7FC148B
:109AB00009F059C080912D0890910705891B80936A
:109AC0002D0887FF02C010922D0880912D088A3042
:109AD0001CF089E080932D08109207058D2D880FCA
:109AE0008D0D880F4D2D50E04E55574F8E5B6E2DCE
:109AF00021E002E00E94E85A103631F080918004A3
:109B000090918104009779F1812F0E94245F109237
:109B1000040581E090E002C0880F991FDA94E2F713
:109B200090918301982790938301803151F0803286
:109B300071F0883099F493FF02C09F7C0DC098604B
:109B40000BC094FF02C0977D07C0906105C095FFD0
:109B500002C0977E01C090629093830181E00E94D1
:109B600009550E94A55598E0E90EEE2DE93308F05D
:109B7000E2C0C394809103058C15F8F480916B01C9
:109B8000869586958095817021E0FC1020E06E2DF1
:109B900043E958E0012F0E94052D80958170880FC0
:109BA000880F90916B019B7F982B90936B01F8E04D
:109BB000EF0E2E2D293308F0BEC0C394809103050B
:109BC0008C1500F590916B01991F9927991F81E0E1
:109BD000891B21E0FC1020E06E2D45E858E0012FA4
:109BE0000E94052D809587958827879590916B0118
:109BF0009F77982B90936B0138E0E30E8E2D89337D
:109C000008F099C0C394809103058C1508F58091E4
:109C10006E018295869587708095817021E0FC1099
:109C200020E06E2D4BE758E0012F0E94052D809516
:109C300081708295880F807E90916E019F7D982B18
:109C400090936E0198E0E90EEE2DE93308F073C0B1
:109C5000C394809103058C1518F580916E0182954F
:109C60008695869583708095817021E0FC1020E0B8
:109C70006E2D43E758E0012F0E94052D80958170DD
:109C80008295880F880F807C90916E019F7B982B26
:109C900090936E01F8E0EF0E2E2D293308F04BC0A3
:109CA000C394809103058C1508F045C086E06E2DA5
:109CB0004EE658E00E94475B3E2D383390F434E284
:109CC00090E0832F6E2D44E857E0292F00E0398380
:109CD0009A830E94C6599A819F5F3981385E943079
:109CE00081F788E0E80E9E2D993328F5DD24D39482
:109CF000FC10DD2440916C014F5C82E16E2D2D2D16
:109D00000E94255A94E200E00F5F892F6E2D402FAC
:109D100020E09A830E949F0E9A81985E0430A1F7FA
:109D2000DD2049F0812F60916C0140E023E00E942A
:109D30001C1480936C010F900F90CF91DF911F91B5
:109D40000F91FF90EF90DF90CF90BF90AF9008956C
:109D50004F925F926F927F928F929F92BF92CF921B
:109D6000DF92EF92FF920F931F93DF93CF9300D078
:109D7000CDB7DEB7182F8AE09FE00E94691981EA0B
:109D800098E0612F45E02FEC37E008E050E1E52E48
:109D90000E946A1E6090A1086A94862D66E00E9467
:109DA0005141103611F0143641F467FC06C0609240
:109DB00088088CE392E30E946A14CC24DD24EE240C
:109DC000E39428E0F22E772467FC70943091030529
:109DD0003C0DBB24B394383028F4BB248E2D88303E
:109DE00028F074C09E2D973008F070C0032F10E04B
:109DF00091E06016710609F090E0DD2019F0DD2495
:109E0000D39401C0D92E80E06F2D47E05FE0292F69
:109E10003A8399830E94185B3A819981393010F412
:109E200082E101C087E1A8014F5F5F4F6F2D292FAD
:109E30000E945B5DBB2079F008501040280193E040
:109E4000440C551C9A95E1F7400E511EE6E9F3E0EB
:109E50004E0E5F1E0BC02801440C551C440C551CB3
:109E6000400E511E8EE693E0480E591E42010AE252
:109E7000F40141914F01552747FD5095802F6F2DDB
:109E800020E00E945B5D0B5E033991F7F8E0FF0E66
:109E9000E394BB20B1F085E090E0480E591E0AE241
:109EA000F20141912F01552747FD5095802F6F2DCD
:109EB00020E00E945B5D0B5E0E3791F7F8E0FF0E2D
:109EC000E394C3948C2D873009F080CFDD2029F4F2
:109ED000809103058F5F809303050F900F90CF91C2
:109EE000DF911F910F91FF90EF90DF90CF90BF9087
:109EF0009F908F907F906F905F904F900895AF925A
:109F0000BF92CF92DF92EF92FF920F931F93CF9366
:109F1000DF93F82E89E898E06F2D4DE00E94DB1F5B
:109F200080918108882319F080E49EE002C086E3D6
:109F30009EE00E946919182F809182080E94FE0DF0
:109F4000EC01812F8A5F60E0488120E00E94CB0E07
:109F5000A09089088A2D66E00E94514118E0EE2405
:109F6000BB24A7FCB094209103052E0D822F90E016
:109F7000DD24D394A816B90609F0DD24263009F4AF
:109F8000FAC0273090F4223009F457C0233030F45F
:109F9000222309F1213009F0E8C134C0243009F44A
:109FA00099C0253008F0BAC069C02A3009F46BC1E5
:109FB0002B3038F4283009F420C1293008F044C18E
:109FC000F1C02C3009F49CC12C3008F47AC12D303A
:109FD00009F0CBC1B2C18CE0612F4FE25EE00E947C
:109FE000475B84E5612F49812D2D0E949F0EDD2066
:109FF00009F4BBC18F2D698141E024E20E940D1458
:10A000008983B3C18CE0612F48E25EE00E94475B28
:10A010004A81552747FD50952D2D206484E5612FF9
:10A020000E945B5DDD2009F4A0C18F2D6A8143E8A9
:10A030002DE70E940D148A8398C18F8186FF03C08B
:10A040004EE15EE002C047E15EE08CE0612F0E94DD
:10A05000475B4885552747FD50952D2D206484E5A5
:10A06000612F0E945B5DDD2009F47FC18F2D688523
:10A0700043E82DE70E940D14888777C1CF80C294F2
:10A08000C694C694E3E0CE2281E0C8228CE0612F22
:10A090004CE05EE00E94475B43E09C2D949FA00152
:10A0A00011244B5F514F84E5612F23E00D2D0E9459
:10A0B000E85ADD2009F459C18F2D6C2D40E021E0D4
:10A0C0000E940D1481708295880F880F807C9F817B
:10A0D0009F7B90C08CE0612F40E05EE00E94475B78
:10A0E0008F81817090E0AC01440F551F480F591FBC
:10A0F0004750524F84E5612F23E00D2D0E94E85A0E
:10A10000DD2009F432C16F8161708F2D40E021E0C4
:10A110000E940D1481709F819E7F6CC08CE0612F26
:10A1200042EF5DE020E00E94185B4C8183E0489F95
:10A13000A00111244B5C504F84E5612F23E00D2DCD
:10A140000E94E85ADD2009F410C18F2D6C8140E097
:10A1500026E10E940D148C83873008F406C19F2DE0
:10A16000903609F002C18750809388088CE392E30F
:10A170000E946A14FAC08CE0612F4BEE5DE00E94F1
:10A18000475B8EE4612F4B812D2D0E94EB0EDD206D
:10A1900009F4EBC08F2D6B814AEE26E10E940D146D
:10A1A0008B83E3C08CE0612F43EE5DE00E94475B50
:10A1B0000F810295037049F02D2D206484E5612FF5
:10A1C000402F50E00E945B5D07C084E5612F4FED9A
:10A1D0005DE02D2D0E94185BDD2009F4C6C08F2D97
:10A1E000602F40E023E00E940D1483708295807FF1
:10A1F0009F819F7C982B9F83B8C08CE0612F48ED96
:10A200005DE00E94475B4F814695477050E063E0F8
:10A21000440F551F6A95E1F74154524F84E5612F71
:10A2200028E00D2D0E94E85ADD2009F49EC06F81C0
:10A23000669567708F2D40E022E00E940D148770B4
:10A24000880F9F81917FD6CF8CE0612F44EB5DE03A
:10A250000E94475B4D8142954F7080E6612F50E030
:10A260002D2D0E945B5DDD2009F47FC06D8162951C
:10A270006F708F2D40E02FE00E940D148295807F3B
:10A280009D819F701BC08CE0612F4BEA5DE00E94B6
:10A29000475B4D814F7080E6612F50E02D2D0E946D
:10A2A0005B5DDD2009F461C06D816F708F2D40E032
:10A2B0002FE00E940D148F709D81907F982B9D83BD
:10A2C00054C08CE0612F40EA5DE00E94475B4E8104
:10A2D00042954F7080E6612F50E02D2D0E945B5D0E
:10A2E000DD2009F442C06E8162956F708F2D40E0D1
:10A2F0002FE00E940D148295807F9E819F701AC06E
:10A300008CE0612F47E95DE00E94475B4E814F7012
:10A3100080E6612F50E02D2D0E945B5DDD2029F14C
:10A320006E816F708F2D40E02FE00E940D148F70B2
:10A330009E81907F982B9E8318C08CE0612F45E80A
:10A340005DE02D2D0E94185BDD2079F08F2D803887
:10A3500061F40E94245F809182080E94F82181E0CC
:10A360000E94606880E00E943514E394185F9E2D7F
:10A37000973009F0F8CDDF91CF911F910F91FF90A9
:10A38000EF90DF90CF90BF90AF9008955F926F9263
:10A390007F928F929F92AF92BF92CF92DF92EF9275
:10A3A000FF920F931F93CF93DF93D82E8EEE9EE0F4
:10A3B0000E9469198FE998E06D2D44E02FEC37E099
:10A3C00008E075EFE72E7EE0F72E51E1C52E11E192
:10A3D000A12E0E94E11AF0909F08FA948090A008A4
:10A3E0008F2D66E00E9451418D2D803821F59F2DE3
:10A3F000903108F5EF2DFF27E7FDF09580910305DB
:10A40000E81BF109EE0FFF1FE75FFA4FC081D18112
:10A410008F2D0E940E0EFC01882069F48281882312
:10A4200019F0D095C195DF4FD483C38382E00E9499
:10A4300009550E94A55518E09924552453946F2C72
:10A44000772467FC709400910305090D003109F42D
:10A45000E1C0802F0E940E0EEC018A816B817C810D
:10A46000882319F0709561957F4FA02EBB24F501CC
:10A47000EE0FFF1FE75FFA4F20813181261B370B5C
:10A480002333310524F0F501E157F74F08C09FEF62
:10A490002E3C39072CF4F501E157F74F85258083D1
:10A4A000402F4F5F80E0612F20E00E94CB0EF5012E
:10A4B000E157F74F8081882311F04FE701C04EE745
:10A4C0008BE4612F20E00E94255AEE246A147B045D
:10A4D00071F48E1461F480910405882359F48091FD
:10A4E000800490918104009739F401E001C000E0FC
:10A4F000CC2405C002E001C001E0CC24C3948E2D21
:10A50000823009F43FC0833009F45DC08130C1F06E
:10A510004B815C81202F206280E3612F0E945B5D74
:10A52000CC2009F46BC06B817C818D2D48E15CEF00
:10A5300028EE33E002E00E9449139C838B835EC0C7
:10A5400048814456552747FD509588E4612F202FB8
:10A550000E945B5DCC2009F451C068816456688319
:10A5600080919E0181FF04C08D2D43E82DE703C03B
:10A570008D2D4CE924E60E940D14888388818C5926
:10A5800088833CC049814C59552747FD509586E644
:10A59000612F202F0E945B5DCC2081F169816C5975
:10A5A000698380919E0181FF04C08D2D43E82DE7D2
:10A5B00003C08D2D4CE924E60E940D148983898106
:10A5C000845689831BC08A8190E0AC01440F551FDB
:10A5D000480F591F4951514F8CE6612F23E00E94CB
:10A5E000E85ACC2059F08D2D6A8140E021E00E948C
:10A5F0000D1491E0882309F490E09A83E3949E2D52
:10A60000943009F063CF9394185F892D873009F057
:10A610001ACF1FC001E09F2D903109F000E080911A
:10A620000505882311F020E001C0202F82E1612F71
:10A6300046ED5EE00E94185B002359F08D2D8038B6
:10A6400041F489E18093050580E80E94245F0E941F
:10A65000F93DDF91CF911F910F91FF90EF90DF9027
:10A66000CF90BF90AF909F908F907F906F905F90B2
:10A670000895F8942091B70D3091B80D7894C901E0
:10A680000895CF93DF93C8E2D1E080E6FE011192F6
:10A690008A95E9F78AE08093280189E18093560141
:10A6A0008AE58093570181E080936C012196FE0139
:10A6B00020E032E080E891E0219331939587848710
:10A6C000938F828F41E0E733F407B1F789E791E098
:10A6D00067ED7FE04AE050E00E94FC6880E090E097
:10A6E00029913991820F931FE1E0C134DE07C1F750
:10A6F0009093540180935301DF91CF9108951F935C
:10A70000CF93DF938AEA98E060E00E94655768E2A1
:10A7100071E080E6FB0111928A95E9F78AEA98E0F8
:10A7200040E650E00E94F157182FC9E7D1E0888138
:10A730000E94EB2C0E94FB2C8993F1E0C338DF07C9
:10A74000B1F7809128018A3028F4809165048160F6
:10A75000809365048AE0809328011D3468F0E9E263
:10A76000F1E020E030E081919191280F391F81E0E4
:10A77000E134F807C1F702C020E030E081E0409109
:10A780005301509154014217530709F080E0DF91C3
:10A79000CF911F9108951F93182FE8E8F1E025EA63
:10A7A00032E0DF01C9011D920197E9F7CF016CEC9E
:10A7B0007FE04AE050E00E94FC68812F90E0019623
:10A7C0006AE070E00E94A668605D60938D01805D24
:10A7D00080938E018AE08093920180E00E94FB5F6B
:10A7E0001F910895CF92DF92EF92FF920F931F93E4
:10A7F000DF93CF930F92CDB7DEB76B01803160F559
:10A80000682F6F5F8AEA98E049830E946557498103
:10A81000042F10E0C60160E270E050E00E941D6964
:10A820008AEA98E0B6014AE050E00E94F1578A3087
:10A83000910591F48AEA98E00E945757F601E00FDB
:10A84000F11F2AE030E006C0B9010E949268805DE5
:10A850008293CB010097C1F70F90CF91DF911F91A9
:10A860000F91FF90EF90DF90CF9008958F5F0E943F
:10A87000E85608951F93CF93DF93182F803168F522
:10A88000682F6F5F8AEA98E00E94655768E871E078
:10A8900025EA32E0FB01C90111920197E9F78AEA42
:10A8A00098E045EA52E00E94F1578F3F910509F088
:10A8B00018F4812F0E94CB53C8E8D1E088810E9410
:10A8C000EB2C0E94FB2C899391E0C239D907B1F798
:10A8D0008AE0809392010E94A914DF91CF911F9189
:10A8E00008950F931F93DF93CF93CDB7DEB7609793
:10A8F0000FB6F894DEBF0FBECDBF682F6F5F062F77
:10A900000AC0102F1F5F812F688B0E94E85668894C
:10A91000882329F0012F0031A0F3003139F18AEAB0
:10A9200098E00E946557602F6F5F83EB98E042E0EC
:10A9300028E532E00E94D7588E010F5F1F4F06C0F6
:10A9400083EB98E0B8010E945258A8958AEA98E0F3
:10A95000B8014FE050E00E948057482F882381F7CC
:10A9600083EB98E00E94005981E001C080E060968E
:10A970000FB6F894DEBF0FBECDBFCF91DF911F9110
:10A980000F910895EF920F931F930E94D35688233F
:10A9900041F00E943E5687FD04C00E947F538823E9
:10A9A00081F58CEB9FE061E00E9418128AEA9FE03B
:10A9B0000E94FF110E94AD560E9441538AEA98E01E
:10A9C00060E041E028E231E000E610E078ECE72EBC
:10A9D0000E942F598036910529F08BE99FE060E0B5
:10A9E0000E94181280E00E94CB538AEA98E061E04E
:10A9F00042E028E831E005EA12E058ECE52E0E943A
:10AA00002F59809155010E943A541F910F91EF9058
:10AA10000895882359F09091C608982B9093C60802
:10AA20000E94F60D9093C8088093C7080895EF928E
:10AA30000F931F93CF93DF931091C608112309F44E
:10AA40007EC0882309F076C00E94F60D2091C708C9
:10AA50003091C808AC01421B530B4436510508F431
:10AA60006EC068C081E08093C508812F90E0EC0142
:10AA7000C470D07012FF03C023E02093C508109269
:10AA8000C60880FF1CC08CEB98E061E141E028E241
:10AA900031E000E610E0F4E1EF2E0E942F598036FD
:10AAA000910511F480E020C08091C208823021F429
:10AAB0008091C608816029C08BE89FE035C081FF86
:10AAC00036C08CEB98E061E142E028E831E005EA2D
:10AAD00012E0E4E1EE2E0E942F5952E0853A9507EC
:10AAE00039F4809155018F5F61E10E94F6561FC0D5
:10AAF0008091C2088230A1F48091C608982F92609C
:10AB00009093C608209719F086608093C6080E942B
:10AB1000F60D845690409093C8088093C70807C0EC
:10AB2000209729F48BE79FE060E00E9418121092B2
:10AB3000C50805C08091C508882309F493CFDF912B
:10AB4000CF911F910F91EF9008950AC081E00E946C
:10AB5000175580914B0E833019F4A89510924B0E27
:10AB60008091C608882391F70895DF93CF930F92C1
:10AB7000CDB7DEB7682F70E084E0660F771F8A9547
:10AB8000E1F7CE01019641E050E00E9424698981FD
:10AB90000F90CF91DF910895DF93CF930F92CDB7B0
:10ABA000DEB76983682F70E094E0660F771F9A958F
:10ABB000E1F7CE01019641E050E00E94F85D0F9070
:10ABC000CF91DF91089589EC98E060E070E040E477
:10ABD00050E00E94F85D08958BEC98E062E070E030
:10ABE00041E050E00E94F85D08950F931F93182FE5
:10ABF000082F04C0802F0E94B555082F802F0E9477
:10AC0000B5558823B9F7802F6091CB080E94CC55A9
:10AC10001093CB080E94EC551F910F9108951F933C
:10AC20001091CB08112359F0812F0E94B5558093C4
:10AC3000CB080E94EC55812F60E00E94CC55812FFB
:10AC40001F910895F8942091B70D3091B80D789424
:10AC5000C9010895EF92FF92CF93DF938091CB08C3
:10AC6000C0E0D0E003C02F960E94B5558823D9F7E5
:10AC7000CE01DF91CF91FF90EF900895CF92DF92B8
:10AC8000EF92FF920F931F93CF93DF9380E8E9E059
:10AC9000F9E0DF011D928A95E9F70DEC18E0C0E0BC
:10ACA000D0E08C2FC43139F4D090CB083BECE32EAC
:10ACB00038E0F32E0BC07E01EE0CFF1CEC0EFD1EE7
:10ACC0002DEC38E0E20EF31ED801DC9090E0C82EA7
:10ACD000C3941DC08D2D84508C3738F4ED2DF0E0D9
:10ACE000E75FF64F8081882361F0992329F0892F4F
:10ACF00060E00E94CC550DC0F70110820E94E35520
:10AD000008C0C0828D2D0E94B5559D2DD82EDD2006
:10AD100009F721960D5F1F4FC531D10511F604E0EB
:10AD2000E02FF0E0E75FF64F8081882349F4802F21
:10AD30006091CB080E94CC550093CB080E94EC5543
:10AD40000F5F003869F780E0DF91CF911F910F917D
:10AD5000FF90EF90DF90CF9008951F9380E4E9EC8F
:10AD6000F8E0DF01982F1D929A95E9F794E090930F
:10AD7000C9088093CA0880E18093CC0884E001C0B0
:10AD8000812F182F1F5F612F0E94CC551038C1F7FB
:10AD90008FE760E00E94CC5584E08093CB080E944E
:10ADA000E3551F91089589EC98E060E070E040E47D
:10ADB00050E00E9424698091C908843039F481E010
:10ADC0009091CA08903419F080E0089580E00895C9
:10ADD00090E0FC01EE0FFF1FE80FF91FE753F74F5C
:10ADE00081E09481992309F480E00895DF93CF9363
:10ADF00000D00F92CDB7DEB790E0FC01EE0FFF1F41
:10AE0000E80FF91FDE011196E353F74F23E001909D
:10AE10000D922150E1F770E0DC01AA0FBB1FA80FD3
:10AE2000B91FFB01EE0FFF1FE60FF71FA353B74F2C
:10AE3000E353F74F83E001900D928150E1F7FB015E
:10AE4000EE0FFF1FE60FF71FE353F74FDE011196DA
:10AE500083E00D9001928150E1F70E94E3550F903D
:10AE60000F900F90CF91DF910895DF93CF930F92C2
:10AE7000CDB7DEB790E09C01220F331F280F391F9A
:10AE8000F901E753F74F84812353374F93E0D901FA
:10AE90001D929A95E9F789830E94E3558981882359
:10AEA00011F00E94F5550F90CF91DF910895FC01AC
:10AEB000808190E0FC01EE0FFF1FE80FF91FE253C5
:10AEC000F74F918180819F700895FC016083128209
:10AED000118270E0CB01880F991F860F971FDC014C
:10AEE000A753B74F14962C9114972383148215827D
:10AEF00016828153974FFC01808182958F7008954F
:10AF00008F929F92AF92BF92CF92DF92EF92FF9279
:10AF10000F931F93DF93CF930F92CDB7DEB78C01C2
:10AF20005B01FC01808190E0FC01EE0FFF1FE80F48
:10AF3000F91FE253F74F80812181922F9F70F80112
:10AF400021813281821B930BE42EF52E8E159F05F5
:10AF500008F47C0167014E010894811C911C25C0F6
:10AF6000F8016381662321F184818F5F848370E01F
:10AF7000B4E0660F771FBA95E1F7680F711DC40141
:10AF800041E050E00E9424698981F50181935F01CD
:10AF9000F80184818F3030F0148283810E94B5558E
:10AFA000F80183830894C108D108C114D104C1F603
:10AFB000F801818192818E0D9F1D8C199D099283CC
:10AFC00081838E2D8C190F90CF91DF911F910F915E
:10AFD000FF90EF90DF90CF90BF90AF909F908F90B9
:10AFE00008958F929F92AF92BF92DF92EF92FF925D
:10AFF0000F931F93CF93DF938C015B017A01C0E025
:10B00000D0E045E0842E912C880E991E3BC0F801BB
:10B01000858190E08F779070009741F4C801B4016A
:10B0200041E050E00E948057813079F5F801458178
:10B030003FE7D32ED4222D2D30E0C7018C1B9D0B72
:10B040008217930710F4DE2CDC1AB5016C0F7D1FFC
:10B0500047FF08C0CB0160E070E04D2D50E00E943A
:10B060001D690AC0C8014D2D50E00E9480578D1502
:10B0700019F0C80FD11D09C0CD0DD11DF801858172
:10B080008D198583CE15DF0510F2CE01DF91CF91AA
:10B090001F910F91FF90EF90DF90BF90AF909F9026
:10B0A0008F9008959F92AF92BF92CF92DF92EF92CE
:10B0B000FF920F931F93CF93DF93EC018B01C42E6C
:10B0C0008B81882389F489819A81009769F4E880CB
:10B0D000FF240E940F568B83F701EE0FFF1FEE0D2A
:10B0E000FF1DE753F74F8483DC2C6FE0962E44C09E
:10B0F000EF80F8840E94F60DE81AF90AF7FE02C004
:10B1000082E004C08B81882319F481E08E8337C0EC
:10B110009C819F3080F01C820E94B555882339F4B1
:10B12000EB800E940F56682F8E2D0E94CC558B818C
:10B130000E94B5558B838B81882339F36C81992DBF
:10B14000961BED2C9D1508F4E92EAE2CBB2470E067
:10B150006F5F7F4F90E054E0880F991F5A95E1F799
:10B16000680F791FC801A5010E94F85D0A0D1B1D1B
:10B170008C818E0D8C83DE18DD2009F0B9CF2C2D4B
:10B1800030E02D19310989819A81820F931F9A83AA
:10B1900089838C2D8D19DF91CF911F910F91FF9095
:10B1A000EF90DF90CF90BF90AF909F9008950F9356
:10B1B0001F93CF93DF93EC01890168831A82198270
:10B1C00070E0CB01880F991F860F971FFC01E75392
:10B1D000F74F24812B831C821D821E82FC01E253C7
:10B1E000F74F10824295407F41830E94F60D080F71
:10B1F000191F18870F83DF91CF911F910F91089529
:10B200001F93CF93DF93EC01888190E0FC01EE0F58
:10B21000FF1FE80FF91FE253F74F898180839A815E
:10B220009F708181807F892B81838B81882389F026
:10B230000E94B555182F882361F08B8160E00E9431
:10B24000CC550E94E355112331F0812F0E94F55512
:10B2500002C010E0F6CFDF91CF911F9108954F9279
:10B260005F926F927F929F92AF92BF92CF92DF9246
:10B27000EF92FF920F931F93DF93CF930F92CDB76F
:10B28000DEB75C01290168012E2D30E00E94D758FD
:10B290001982720100E010E081E03E010894611C17
:10B2A000711CF70191917F01992341F4882349F49E
:10B2B0009081992349F4992493941EC0882371F4B2
:10B2C00003C09924939401C0992499819F3718F45D
:10B2D0000C151D0561F5882379F001C09924898139
:10B2E000882321F180688983C501B30141E00E9470
:10B2F00052588130D1F025C089818823B9F0C50129
:10B30000B30141E00E9452588130D9F44981B8011B
:10B31000641B7109640D751DC5010E945258998105
:10B32000891719F0981B99830CC01982892D99816E
:10B330009F5F99830F5F1F4FC016D10608F0B1CFF2
:10B3400005C089818F776801C81AD108C5010E949C
:10B350000059C6010F90CF91DF911F910F91FF907F
:10B36000EF90DF90CF90BF90AF909F907F906F90C5
:10B370005F904F90089580E094E0E9E8F9E0DF0104
:10B380009C011D9221503040E1F708950F931F93C7
:10B39000CF93DF93DA011196FA014491ED012196E2
:10B3A000FD01A491B0E0179613E0B595A7951A9505
:10B3B000E1F71A2FDE011196FE019491929FE001B0
:10B3C0001124AC0FBD1F00FD08C001FF08C0909103
:10B3D000B90D51E096FD04C002C051E001C050E03B
:10B3E00066956695669570E09B013695322F22270B
:10B3F0003795279590E0280F391F610F711D7695BD
:10B40000762F662777956795680F791F042F10E0D0
:10B4100014C0E901C757D64F80E090E008C0FD0195
:10B42000E80FF91FE4915111E095E9930196841713
:10B43000B0F3A00FB11F20583F4F2617370749F729
:10B44000DF91CF911F910F910895FF920F931F935A
:10B45000CF93DF93942F46313CF4440F490F440FB0
:10B4600022FFABC0440FA9C0482F4A5F092F112704
:10B4700007FD109520FD09C021FF0AC03091B90DCC
:10B48000FF24F39436FD05C003C0FF24F39401C0EC
:10B49000FF2466956695669570E07695762F66270B
:10B4A00077956795680F711DEB01C757D64F22FF3F
:10B4B0004FC09E3209F04A5FC801809760E170E09A
:10B4C0000E94A66880EA90E0689F9001699F300D15
:10B4D000789F300D1124C801880F991F53E0000F89
:10B4E000111F5A95E1F7800F911F280F391F285718
:10B4F0003F4E85E0882369F0F9019491E056FF4FB3
:10B5000054912F5F3F4FF9016491E056FF4F7491C2
:10B5100004C060E050E090E070E0FF2021F09095E2
:10B52000609550957095DE01AF57BF4FFDE0A9388B
:10B53000BF0740F498836983FE01E058FF4F5083B2
:10B540007C93229681508F3FC1F12F5F3F4FD2CF26
:10B5500023FF0DC0FF2011F08FEF01C080E067577F
:10B56000764FFB01808321964F5F91E001C090E010
:10B570009801220F331F220F331F200F311F2B5B27
:10B58000304F85E0F9012F5F3F4FE491992311F08F
:10B59000843039F0FDE0C938DF0718F4F110E09588
:10B5A000E993815079F75DE0C938D50730F4FF2081
:10B5B00011F08FEF01C080E08883842FDF91CF915D
:10B5C0001F910F91FF90089520E00E94255A089541
:10B5D000CF92DF92EF92FF920F931F93CF93DF935F
:10B5E000162FF22EF0E1EF2EE022C42EE6016E01BE
:10B5F000D52EE6010CC0EE2011F0488102C0FE01FC
:10B600004491612F202F0E94255AFA942196FF2001
:10B6100091F7DF91CF911F910F91FF90EF90DF9005
:10B62000CF9008950F9300E00E94E85A0F9108957B
:10B63000CF92DF92FF920F931F93CF93DF93162F3A
:10B64000022FA0E1FA2EF222C42EE6016E01D52EC1
:10B65000E601FF2011F0488102C0FE0144912196CD
:10B66000442329F0612F202F0E94255AF2CFDF9129
:10B67000CF911F910F91FF90DF90CF900895982F59
:10B68000AB0180E0692F20E00E94185B089520E064
:10B690000E94185B0895EF92FF920F931F93DF9320
:10B6A000CF930F92CDB7DEB7182F062F7A01982FC0
:10B6B0009C5E95504E2D4F704A301CF0495C28E03E
:10B6C00002C0405D20E0892F602F99830E94255A97
:10B6D0009981911731F0B4E0F694E794BA95E1F7C7
:10B6E000E8CF0F90CF91DF911F910F91FF90EF90D6
:10B6F0000895E62FE695E695E695F0E0F695FE2F9F
:10B70000EE27F795E795E80FF11DE757F64F8DE027
:10B71000E938F80758F4677081E090E002C0880FBC
:10B72000991F6A95E2F7208128272083089547FF13
:10B7300002C0840F4195E62FE695E695E695F0E088
:10B74000F695FE2FEE27F795E795E80FF11DE757E1
:10B75000F64F6770A1E0B0E001C0AA0F6A95EAF762
:10B7600011C08DE0E938F80778F4822F90E09C0151
:10B770003595279580FF04C080818A2780832068C3
:10B7800041503196442369F708952FEF0E94975B4B
:10B7900008950F931F93CF93DF93C82FD0E0E62F28
:10B7A000E695E695E695F0E0F695FE2FEE27F795FF
:10B7B000E795EC0FFD1FE757F64F062F10E0242FFB
:10B7C000332727FD3095200F311FC90168E070E055
:10B7D0000E94A6687695762F6627779567956C0FF9
:10B7E0007D1F6757764F0770107081E090E002C0B0
:10B7F000880F991F0A95E2F781959081892708C0E3
:10B80000E058FF4F8DE0E938F807D0F4808180954B
:10B810008083E617F707A0F38DE0E938F80780F496
:10B82000C90168E070E00E94A66821E030E002C033
:10B83000220F331F8A95E2F721958081822780832A
:10B84000DF91CF911F910F9108952F923F924F92C8
:10B850005F926F927F928F929F92AF92BF92CF92A0
:10B86000DF92EF92FF920F931F93DF93CF9300D05D
:10B870000F92CDB7DEB7182F662E59016A01F02E50
:10B88000802F05FF04C004FF04C002E003C000E0F5
:10B8900001C001E0E7FE04C0E1942224239401C02A
:10B8A0002224D7FE0BC0D094C094B094A094A11CC5
:10B8B000B11CC11CD11C4424439401C0442482FF08
:10B8C00006C09CE09093890D3AE0932E05C096E067
:10B8D0009093890D25E0922E86FF2FC04110190DFF
:10B8E00028EEA21623E0B20620E0C20620E0D2062F
:10B8F00014F0190D06C034E6A316B104C104D10436
:10B9000014F0190D06C08AE0A816B104C104D104D0
:10B910000CF0190D002391F0023039F4E4E6AE1674
:10B92000B104C104D10454F4190DFAE0AF16B10406
:10B93000C104D1041CF4190D01C0191B8091890D9B
:10B94000810F8093890D023011F420EFF20E5524FF
:10B95000539492E0792E88242E2D332727FD30959D
:10B96000862D8A5F89833B832A8370C0C601B50117
:10B970002AE030E040E050E00E94DB68E62E80E301
:10B98000382E3E0C812F662D432D2F2D0E94255AD7
:10B990000515D9F5F2FE23C08E2D8150833008F4B1
:10B9A0007394C601B5012AE030E040E050E00E9407
:10B9B000DB68CA01B9012AE030E040E050E00E94B3
:10B9C000DB68623011F06430C1F4E32DE43319F424
:10B9D000812E839413C0812E8A9473940FC01250C9
:10B9E000812F8F5FF0FE05C0662D47E00E94C95B86
:10B9F00005C069810E94795B01C0812EFAE0AF1613
:10BA0000B104C104D1040CF000E0C601B5012AE084
:10BA100030E040E050E00E94DB6859016A012115E6
:10BA200031054105510581F4002331F0023059F40C
:10BA3000252D223040F408C0F4FE10C0222021F44D
:10BA400030EFF30E01C000E019195394852D90E0FA
:10BA5000EA81FB81E817F9070CF088CF882061F0B4
:10BA6000662D645F882D472D0E94C55B662D635F40
:10BA7000882D472D0E94C55B442039F0812F8919FC
:10BA8000662D4DE22F2D0E94255A0F900F900F909A
:10BA9000CF91DF911F910F91FF90EF90DF90CF90AA
:10BAA000BF90AF909F908F907F906F905F904F90DE
:10BAB0003F902F900895EF920F93022FFA019F016C
:10BAC000442737FD4095542F75E0E72E0E94255CF2
:10BAD0000F91EF90089520E00E945B5D0895A99872
:10BAE000AB98AC988BBBAD9AAD98AB9AA99A0895D8
:10BAF00020E030E006C045E04A95F1F700002F5FF6
:10BB00003F4F28173907BCF30895AA9885E08A9516
:10BB1000F1F7000085E08A95F1F70000AA9A8CED14
:10BB200095E00E94785D82EE0E946F5D8EEA0E9431
:10BB30006F5D81EA0E946F5D86EA0E946F5D84EA14
:10BB40000E946F5D82EA0E946F5D80EC0E946F5DD3
:10BB50008FE20E946F5D85E20E946F5D81E80E9426
:10BB60006F5D82E20E946F5D8FEA0E946F5D82E2EC
:10BB70008093560108951F93182F81E80E946F5DEE
:10BB8000812F0E946F5D1F9108951F93CF93DF93C4
:10BB900010E0C9E8D9E084E00E946F5D80E10E9476
:10BBA0006F5D812F806B0E946F5DA998AB9AAC98F6
:10BBB000FE0180E290819BBBAD9AAD9891819BBBC9
:10BBC000AD9AAD9892819BBBAD9AAD9893819BBB8A
:10BBD0003496AD9AAD98815069F7C058DF4FAB9A53
:10BBE000A99A1F5F1830B9F6DF91CF911F91089580
:10BBF000BF92CF92DF92EF92FF920F931F93CF935A
:10BC0000DF93EA01E82EF92E062F172F21C0F70146
:10BC1000B1907F0168010894C11CD11C04C0009739
:10BC200039F00E9430188091C50890E082709070C1
:10BC3000E199F5CF1FBB0EBBE09A8DB3B81631F07A
:10BC4000BDBA8FB7F894E29AE19A8FBF2197860127
:10BC50002097E9F6DF91CF911F910F91FF90EF9020
:10BC6000DF90CF90BF9008958093BA0D0895809192
:10BC7000BA0D1092BA0D0895FC018081982F990F8A
:10BC80009E70807F892B8083662321F09160807F66
:10BC9000892B808381818F5F81839281992391F0A9
:10BCA00020812F7079F4933659F0242F206220934D
:10BCB000BA0D903111F4803118F080818F7C80832F
:10BCC000118212828281883009F443C0893058F48D
:10BCD000813009F446C08130A0F08230D1F1843047
:10BCE00009F052C036C08F3549F1803620F48031DA
:10BCF00009F04AC02EC0813689F0823609F044C06E
:10BD00003DC08081982F9F709F30F1F591E692831E
:10BD100091819131E0F08F7C808319C0406640931F
:10BD2000BA0D9081892F82958F708F5F8370829575
:10BD3000807F9F7C982B90838FE508C0818188311C
:10BD400011F4406818C08832F9F480E182831182CE
:10BD500008959181903328F090E09595879582839E
:10BD60001182828190E00197218130E08223932328
:10BD7000009751F440644093BA0D08958181803456
:10BD800018F088E08283118208958E3091056CF45A
:10BD9000FC01EE0FFF1FE80FF91FE357F24F9081F0
:10BDA0009F7081E09F30E9F53FC0823129F18331F6
:10BDB00060F48F30C9F0803118F48E3091F529C0CD
:10BDC000803161F0813169F512C0843151F08431E4
:10BDD000C8F08531D9F0863121F51EC091B194703B
:10BDE0001DC091B192701AC09091630013C09091E0
:10BDF00063009095987012C08091630083FF13C018
:10BE000091B102C091B19095907408C091B19071B8
:10BE100005C091B1917002C091B1907281E09923F7
:10BE200019F480E0089580E008958F708E3058F402
:10BE300090E0FC01EE0FFF1FE80FF91FE357F24FF0
:10BE400082E68283118208958F708E3068F490E0CC
:10BE5000FC01EE0FFF1FE80FF91FE357F24F83E6D7
:10BE6000828380818F7C808308950F931F93CF936B
:10BE7000DF938091B70D9091B80D01969093B80D16
:10BE80008093B70D8091B90D8F5F8093B90D06B384
:10BE9000009540E050E010E001C0AE01EA012196BB
:10BEA000CA01880F991F840F951FB8010C2E02C07C
:10BEB000759567950A94E2F7617070708357924F99
:10BEC00050E00E943C5EC630D10539F700B30095C2
:10BED000C0E0D0E0FE01E85BF64EE4919E012A5FEF
:10BEE0003F4FC901880F991F820F931F8357924FAD
:10BEF000E02361E009F460E09E012A5F422F50E0F8
:10BF00000E943C5E2196C830D10521F7DF91CF9188
:10BF10001F910F910895FF920F931F93CF93DF937B
:10BF2000F82EE2EAF1E080E090E0582F9C01408199
:10BF3000F41638F0442329F001963A96813291059F
:10BF4000A1F75032B9F1E901CC0FDD1FC901A3E01F
:10BF5000880F991FAA95E1F7C80FD91F8E010E55BA
:10BF60001E4FA9014F5F5F4FCA01880F991FE3E081
:10BF7000440F551FEA95E1F7840F951F20953095E2
:10BF8000205E3F4FA901440F551F63E0220F331F6E
:10BF90006A95E1F7420F531F8E559E4FB8010E94DC
:10BFA0000B698AE0D8011D928A95E9F7C857DE4FE0
:10BFB000FA8E02C002EA11E0C801DF91CF911F9111
:10BFC0000F91FF90089580E491E0E2EAF1E0DF0153
:10BFD0009C011D9221503040E1F70895E0916C01E1
:10BFE000F0E0EE0FFF1FEE0FFF1FE80FF11DE15114
:10BFF000FB4F84910895EF92FF920F931F93DF936D
:10C00000CF9300D000D0CDB7DEB719821A821B8241
:10C010001C82E0917101F0E0E852FB4F26E030E035
:10C0200091E0E491EE2EFF24DE0111960FC06F5FC8
:10C030007F4F0617170711F4FA01908364307105DA
:10C04000B1F79F5F22503040953089F060E070E09A
:10C05000A701022E02C0559547950A94E2F7437056
:10C0600050708A010F5F1F4F4A0F5B1FE0CF88237C
:10C0700061F50E94E35F89810E948B5F8C0181E002
:10C080000E94EE5FF801818324E6F22EF2828A811B
:10C090000E948B5F8C0182E00E94EE5FF801818339
:10C0A000F2828B810E948B5F8C0183E00E94EE5FA5
:10C0B000F8018183F2828C810E948B5F8C0184E085
:10C0C0000E94EE5FF8018183F2820F900F900F9033
:10C0D0000F90CF91DF911F910F91FF90EF900895F6
:10C0E0006F927F928F929F92AF92BF92CF92DF9288
:10C0F000EF92FF920F931F93CF93DF9380919E0156
:10C1000081FF03C060E075E002C060E074E09091E0
:10C110009B0184E69802C0011124885A9D4FE0914A
:10C12000A101FF27E7FDF09548EE53E0E49F900161
:10C13000E59F300DF49F300D112428533045AA247B
:10C14000BB24A81AB90A281B390BF9E0EF2EF5E039
:10C15000FF2E40919801440F485F50E0440F551F57
:10C16000440F551F4554524FEBEBFDE0CC24DD242A
:10C17000C61AD70AA8E5B2E0A81BB90B1CC0E70194
:10C18000699079907E014B01661677060CF44301A5
:10C1900084018C149D040CF48601005A164FE501AD
:10C1A000C01BD10B2C0F3D1F0A0F1B1F11830083D7
:10C1B000938382833496E417F50709F7318320834C
:10C1C0009383828315821482DF91CF911F910F9107
:10C1D000FF90EF90DF90CF90BF90AF909F908F90A7
:10C1E0007F906F900895E0911201F0911301819377
:10C1F000F0931301E09312010895FF920F931F93A0
:10C20000CF93DF93B9E0FB2E90E120E0C82FD0E080
:10C210008E0101701070201711F4905F07C0892FF4
:10C2200090E001970E94F360202F90E1FA9431F0A2
:10C23000D595C795AE014068842FE8CF892F90E04F
:10C240000F960E94F360DF91CF911F910F91FF90A5
:10C2500008951F93CF93DF93182F2BEB3DE030937E
:10C2600013012093120180911801877471F080915D
:10C270009801882319F0813029F402C080E803C0B6
:10C2800080E901C088E9809318018091180187FF37
:10C290000BC086E190E00E94C55E882329F480915E
:10C2A00018018F77809318018091180187FD5AC07B
:10C2B00085E160E040E00E94C90F882309F452C084
:10C2C00080911801806280931801809155018F5FE1
:10C2D00080931901EAE1F1E0A9E0B5E080E01CC03B
:10C2E0002D913D913595279520503E4F37FD05C046
:10C2F00093E02F3F390724F405C020E030E002C06E
:10C300002FEF33E0932F9370482F440F440F942B5B
:10C31000908321838F5F3296811711F7C8E1D1E0B6
:10C3200089910E94FD6081E0C632D807C9F78091EB
:10C3300012019091130101979093130180931201C0
:10C340008FEF90E00E94F36080E090E00E94F36045
:10C350008BEB9DE09093170180931601DF91CF91B5
:10C360001F910895809118018F7DADCF1F920F927C
:10C370000FB60F9211242F938F939F93EF93FF93F8
:10C3800088B391E0892788BBE0911601F0911701ED
:10C390002191F0931701E0931601822F90E097BD51
:10C3A00086BD293C08F0C09A80914B0E8160809335
:10C3B0004B0EFF91EF919F918F912F910F900FBE98
:10C3C0000F901F9018951F920F920FB60F92112485
:10C3D0002F933F938F939F93EF93FF9388B391E0B5
:10C3E000892788BBE0911201F0911301208130E090
:10C3F00020FD04C088B599B5809603C088B599B56D
:10C40000409699BD88BDC90195958795009791F48F
:10C41000CF010196909313018093120181818823AB
:10C4200051F480917800909179008053984F99BD94
:10C4300088BD01C0808380914B0E816080934B0E3C
:10C44000FF91EF919F918F913F912F910F900FBE90
:10C450000F901F901895EDE7F0E08081857E808336
:10C4600017981F9AAAE8B0E01C9210928B0082E8FD
:10C470008C938081806280830895EDE7F0E0808175
:10C480008F7D8083179AAAE8B0E01C9210928B00EF
:10C490008AE08C9380818861808308951F920F9237
:10C4A0000FB60F9211248F939F93AF93BF93EF9387
:10C4B000FF938091570E882321F01F9A1092570EF8
:10C4C00004C01F9881E08093570EA0911401B09191
:10C4D0001501FD01819191919093870080938600D1
:10C4E000F0931501E093140180914E0E90914F0E40
:10C4F000909385008093840012968D919C91139760
:10C50000009759F483E09EE0909315018093140105
:10C5100080919E0181708093570E80914B0E8160B7
:10C5200080934B0EFF91EF91BF91AF919F918F91AF
:10C530000F900FBE0F901F901895AF92BF92CF92A1
:10C54000DF92EF92FF920F931F93CF93DF9380912F
:10C550009E0181FF03C040E055E002C040E054E08E
:10C56000F0909801FF0C80E1F80E20919B0184E689
:10C57000280290011124285A3D4FE091A101FF2784
:10C58000E7FDF09568EE73E0E69FC001E79F900D30
:10C59000F69F900D112488539045CC24DD24C21AB7
:10C5A000D30A821B930B68EFE62EEF0CE3E0FEE06C
:10C5B00000271127041B150B68E572E0621B730B43
:10C5C00021C0AE2DB0E0AA0FBB1FA75FBA4FAC9041
:10C5D0001196BC90D5014A175B070CF4DA01A0173D
:10C5E000B1070CF4D801A05AB64FE601CA1BDB0B09
:10C5F0008C0F9D1F31832083A60FB71FB383A283A7
:10C600003496E394EF14E8F231832083938382839A
:10C61000885E934090934F0E80934E0E1582148245
:10C62000DF91CF911F910F91FF90EF90DF90CF900E
:10C63000BF90AF9008951F920F920FB60F921124E2
:10C640002F933F934F935F936F937F938F939F931A
:10C65000AF93BF93EF93FF9378940E949D62FF91F5
:10C66000EF91BF91AF919F918F917F916F915F916A
:10C670004F913F912F910F900FBE0F901F901895E3
:10C680002091540E3091550E90E0822793279070A0
:10C69000880F991F805B964EFC0145915491232F82
:10C6A0003327422753275093550E4093540E089535
:10C6B0009091500E96959695982B9093500E809150
:10C6C000510E8F5F8093510E843068F0E091520ECE
:10C6D000F091530E9193F093530EE093520E1092FB
:10C6E000500E1092510E089503C080E00E945863CE
:10C6F0008091510E8823C9F7E091520EF091530EAC
:10C7000010820895882339F08091560E8F5F8093B0
:10C71000560E80E803C01092560E80EC0E945863BB
:10C720008091560E8530B8F708950F931F93182FF8
:10C730000E94406308E0812F81700E9482631695F9
:10C740000150C9F71F910F91089580EC0E94586322
:10C7500080E80E94586380E80E94586380E80E9445
:10C76000586380E80E94586380E80E94586380E81C
:10C770000E94586380EC0E9458630895AF92BF9264
:10C78000CF92DF92EF92FF920F931F93CF93DF939D
:10C790008BEB9DE090931301809312019093530EC5
:10C7A0008093520E1092550E1092540E1092500E0D
:10C7B0001092510E1092560E0E94A563809198011E
:10C7C0000E94956380914D0E0E94956380E00E94C7
:10C7D000956310924D0E09E015E054E0C52ED12C62
:10C7E000F80120813181C901880F991F820F931FA1
:10C7F000B6010E94A668EB0122813381C901880F2E
:10C80000991F820F931FB6010E94A66860507C4F4B
:10C81000C050DC4FF8E0C030DF0710F0CFEFD7E0BA
:10C820007B0128E06030720720F0AFEFEA2EA7E02E
:10C83000FA2E8C2F0E9495635E019B2D9F708E2D8A
:10C840008295807F892B0E949563C701F4E09695BD
:10C850008795FA95E1F70E9495630C5F1F4F25E0DD
:10C860000931120709F0BCCF0091550E8091540E8A
:10C870000E949563802F0E9495630E94A5630E9489
:10C8800074638091780090917900805C93469093D6
:10C89000790080937800C09ADF91CF911F910F911A
:10C8A000FF90EF90DF90CF90BF90AF900895809170
:10C8B000970190914C0E981709F494C080934C0EF8
:10C8C0008130F9F0813030F08230F1F1833009F0BD
:10C8D00089C05EC00E942B621EBC80E49CE99BBDA7
:10C8E0008ABD1DBC1CBC87B7837C87BF8CE386BF19
:10C8F0008FE380937C0087B7806187BF1FBC8AE08D
:10C9000021C00E942B621EBC1DBC1CBC80E797E1AD
:10C9100099BD88BD80EA9FE090937900809378006C
:10C9200087B7837C87BF8CE386BF8FE380937C00CF
:10C9300087B7886087BF80917D00816080937D008C
:10C940001FBC82E08EBD4EC00E942B621EBC88ECD4
:10C9500090E090937900809378008CE291E09DBD07
:10C960008CBD80EE9BEA97BD86BD87B7837C87BF71
:10C970008CE386BF8FE380937C0087B7806287BF9C
:10C9800080917D00816080937D001FBC8AE1DACFB9
:10C990001EBC80E49CE99BBD8ABD1DBC1CBC87B746
:10C9A000837C87BF80917D008E7F80937D008CE3A8
:10C9B00086BF8FE380937C0087B7806187BF1FBCF1
:10C9C0008AE08EBD0E949D6280E593EC9093870083
:10C9D0008093860088E893E190938500809384009B
:10C9E0000E943D6280919701813051F0813028F0A2
:10C9F000823051F0833079F40CC00E947060089549
:10CA000078940E94BE630895789486E00E9429611C
:10CA100008950E94706008951F920F920FB60F92B2
:10CA200011242F933F934F935F936F937F938F9333
:10CA30009F93AF93BF93EF93FF93809197018230C1
:10CA4000C1F480E492EA97BD86BD80917800909110
:10CA500079008F3F910538F488E598E99093790043
:10CA60008093780008C088EC90E0909379008093E0
:10CA700078000E945764FF91EF91BF91AF919F9111
:10CA80008F917F916F915F914F913F912F910F9077
:10CA90000FBE0F901F9018951F920F920FB60F9216
:10CAA00011242F933F934F935F936F937F938F93B3
:10CAB0009F93AF93BF93EF93FF938CB59DB5209158
:10CAC000580E222321F0C09A1092580E04C0C0982C
:10CAD00021E02093580EA0912601B0912701FD017D
:10CAE000219131913BBD2ABDF0932701E0932601AE
:10CAF0002091A9063091AA062817390720F49093AF
:10CB0000AA068093A90620910C0130910D0182178D
:10CB1000930720F490930D0180930C0112968D9150
:10CB20009C9113970097D9F48BEB9DE0909327018C
:10CB30008093260180919E01809581708093580E8C
:10CB400087B78F7E87BF0E945764809197018823A3
:10CB500011F0833021F487B7806187BF789480918A
:10CB60004B0E816080934B0EFF91EF91BF91AF917F
:10CB70009F918F917F916F915F914F913F912F91F5
:10CB80000F900FBE0F901F90189590916B019873A6
:10CB9000903121F463E00E9486680895983111F481
:10CBA00086950895983211F4880F0895903319F4FA
:10CBB000982F990F890F0895FC01A5E6B0E08C919C
:10CBC0008B7F8C93148215821082118216A617A671
:10CBD00008950E94DC65089521E0FC01848188238A
:10CBE00009F420E0822F0895FC0181819081891B46
:10CBF000877098E0981B81E0933008F480E00895F6
:10CC0000FC0184818823F9F081508483828193819F
:10CC1000890F828386A5882309F44CC087A5982FA5
:10CC2000915097A7882331F08091650084608093AC
:10CC300065000895809165008B7F809365008091E9
:10CC4000760187A708951B98809165008B7F80935C
:10CC500065008581882319F081508583089580813E
:10CC60009181891739F190E0DF01A80FB91F16965D
:10CC70002C911697228356962C91569724831E96B4
:10CC80002C911E9723835E962C915E972583D096D8
:10CC90002C91D09726A717A696962C919697322F6F
:10CCA000315096963C939697222321F401968770F3
:10CCB0009070808308958F929F92AF92BF92CF928F
:10CCC000EF92FF920F931F93DF93CF9300D0CDB7D6
:10CCD000DEB74C01122F4A8369830E94F4654A81B2
:10CCE0006981882331F180916B01887311F1F4011E
:10CCF000A180BB24C501019697E0F92EF82280811E
:10CD0000F816B9F0662329F080917501865F860FC9
:10CD100001C080E0A80CB91CF5018683842F0E9415
:10CD2000C565F501868B168FE0AA06A3C686F401B9
:10CD3000F1820F900F90CF91DF911F910F91FF9093
:10CD4000EF90CF90BF90AF909F908F900895AF924B
:10CD5000BF92CF92EF920F93DF93CF9300D00F92B9
:10CD6000CDB7DEB75C012B834A8369830E94F465EB
:10CD70002B814A816981882329F180916B01887315
:10CD800009F1662329F080917501865F860F01C045
:10CD900080E0F5018283842F2B834A8369830E947C
:10CDA000C565F50184832B812583E6A617A6C3827A
:10CDB000808181834A816981002321F00150C5016E
:10CDC0000E945B660F900F900F90CF91DF910F91B3
:10CDD000EF90CF90BF90AF900895CF92EF920F93C6
:10CDE000CF93DF93EC0180916B01869586958695B4
:10CDF000877028819981291709F05CC1E62FF0E03E
:10CE0000E132F10508F056C1EA5BFF4FEE0FFF1F5C
:10CE10000590F491E02D0994CE0166E44AE0DEC06D
:10CE2000CE0166E444E1DAC0CE0166E44EE1D6C04C
:10CE3000CE0164E64AE022E002E0EE24E39452E010
:10CE4000C52E36C1CE016FE545E022E00AE0EE24B2
:10CE5000E394CC240E945B66CE016FE545E02AE0B6
:10CE600001E00E945B66CE016FE545E022E00AE04A
:10CE70001FC1CE0160E54AE023E002E0EE24CC24AD
:10CE8000CA940E945B66CE016CE34AE023E0CC24A6
:10CE9000C3940E945B66CE0166E44AE021E000E0B4
:10CEA00032E0E32E96C0CE0166E445E021E001E0E9
:10CEB000EE24E394CC240E945B66CE0162E34FE053
:10CEC00022E00E945B66CE0160E54FE022E0F0C008
:10CED000CE016EE645E021E002E0EE24E394CC24AE
:10CEE0000E945B66CE016CE745E021E02AC0CE01DE
:10CEF00062E345E025E000E0EE24CC240E945B667E
:10CF0000CE016AE545E025E00E945B66CE016EE653
:10CF100043E024E002E0CCC0CE0160E545E02AE039
:10CF200003E0EE24E394CC240E945B66CE0160E52E
:10CF300045E024E101E00E945B66CE0160E545E04A
:10CF40002AE003E0B5C0CE016AE044E125E002E05A
:10CF5000EE24E394CC24C394ABC0CE0162E344E05E
:10CF60002AE002E0EE24E394CC240E945B66CE012A
:10CF700066E448E024E101E00E945B66CE0162E3E2
:10CF800048E02AE002E00E945B66CE0166E444E0ED
:10CF900024E101E08DC0CE0168E745E02AE00AE027
:10CFA00016C0CE0168E745E022E30AC0CE0160E08A
:10CFB00044E12AE001E00BC0CE0160E044E12AE058
:10CFC00002E005C0CE0160E044E12AE003E0EE2487
:10CFD000E394CC246DC0CE0166E448E221E000E099
:10CFE00048C0813009F466C0CE016BE405C08130D1
:10CFF00009F460C0CE0161E44AE021E000E041C0F4
:10D00000CE01642F46E0F9CFCE0166E44AE022E08B
:10D01000E6CF813009F44EC0CE0166E44AE022E05A
:10D02000EDCFCE0168E7E8CFCE0168E74AE021E026
:10D030001FC0CE016AE74AE021E00FC0CE016CE7D5
:10D040004AE021E004C0CE0168E74FE023E003E0BE
:10D0500010C0CE0168E74FE023E002E00AC0CE0135
:10D0600068E74FE023E004C0CE0166E444E129E133
:10D0700001E0EE24E39406C0CE0166E44AE022E03B
:10D0800002E0EE24CC240E94A76614C0CE016CE31B
:10D0900044E123E002E0EE24CC24C3940E945B66CA
:10D0A000CE0160E544E123E0EE24E394CC24CA946D
:10D0B0000E945B66DF91CF910F91EF90CF90089522
:10D0C000682F8DE294E046E40E94ED660895629F29
:10D0D000D001739FF001829FE00DF11D649FE00D70
:10D0E000F11D929FF00D839FF00D749FF00D659FD1
:10D0F000F00D9927729FB00DE11DF91F639FB00DD0
:10D10000E11DF91FBD01CF0111240895991B79E09C
:10D1100004C0991F961708F0961B881F7A95C9F7C7
:10D1200080950895AA1BBB1B51E107C0AA1FBB1F16
:10D13000A617B70710F0A61BB70B881F991F5A95A3
:10D14000A9F780959095BC01CD01089597FB092E14
:10D1500007260AD077FD04D0E5DF06D000201AF4B8
:10D16000709561957F4F0895F6F7909581959F4F43
:10D170000895A1E21A2EAA1BBB1BFD010DC0AA1F18
:10D18000BB1FEE1FFF1FA217B307E407F50720F030
:10D19000A21BB30BE40BF50B661F771F881F991FAB
:10D1A0001A9469F760957095809590959B01AC01F4
:10D1B000BD01CF01089597FB092E05260ED057FD1E
:10D1C00004D0D7DF0AD0001C38F450954095309534
:10D1D00021953F4F4F4F5F4F0895F6F790958095FB
:10D1E000709561957F4F8F4F9F4F0895EE0FFF1FF2
:10D1F0000590F491E02D0994FB01DC014150504071
:10D2000048F005900D920020C9F701C01D924150D1
:10D210005040E0F708956817790768F4FB01DC01D6
:10D22000E40FF51FA40FB51F02C002900E924150EB
:10D230005040D8F708950C943469DC0101C06D9317
:10D2400041505040E0F70895DC01CB01FC01E19929
:10D25000FECF06C0FFBBEEBBE09A31960DB20D9239
:10D2600041505040B8F70895FB01DC0102C0019025
:0ED270000D9241505040D8F70895F894FFCF2A
:10D27E006A036B036C036D034AF0004DFF07220433
:10D28E007C5EBB0D030EBB0DFF0000AA05FF09FF60
:08D29E000DFF135414AABB0D8F
:00000001FF
